:020000040800F2
:100000000050002069700108B915010859C30008A3
:10001000B7150108B5150108B31501080000000067
:10002000000000000000000000000000B115010801
:10003000AF15010800000000AD150108732B010881
:1000400005710108057101080571010805710108B4
:100050000571010805710108852E0108992E010816
:10006000952E0108912E01088D2E010811350108E9
:1000700001350108F1340108E1340108D1340108E7
:10008000BD340108AB340108057101080571010890
:100090007D1601080571010805710108892E010806
:1000A0000571010895CC00080571010885CC000890
:1000B00075CC000865CC000855CC00080571010816
:1000C0000571010805710108057101080571010834
:1000D00005710108B12B010805710108A52B010864
:1000E000812E01080571010859590108000000001E
:1000F0000000000000000000000000000000000000
:0C01000000000000000000005FF808F1A3
:100110002DE9FF47B0F908300646DDB2382D0C4610
:1001200017460B8100F0C48100F2A480042D00F07A
:100130003B8163D8022D00F0228100F22681012D3F
:1001400000F00E815C2D00F0CD8401F25E83362D2F
:1001500001F0F58401F2D8822C2D00F0728301F2B7
:100160008782222D01F0FD8401F274820A2D00F0B5
:100170009F82742D336800F0F584772D00F0FF84A2
:10018000F52D40F0328572689A420FBFFF23591C4B
:10019000316013F8021BAC4A16BF33601370117044
:1001A0001378FF2B4FF0000340F01985A74A18463B
:1001B0009046995801B108801833C02BF9D1002618
:1001C0004FF01809A24BA34D31462022A2481E70C1
:1001D0002E7019F09AFE8DF808609F4E9DF8083039
:1001E000072B40F2D58423682A78591C21601A70A5
:1001F000002F00F0A480994B3B60A0E0202D00F080
:100200007B8111D8052D9DD120460B2294490FF0FA
:100210001FFD2046082293490FF01AFD072292493C
:1002200020460FF015FD8AE0242D00F0DC80282DFB
:1002300088D101250B688D4E5A1C0A601D700B6811
:1002400020465A190A6006221A700B685A190A6069
:100250000A221A700B685A190A601D7031880FF053
:1002600015FD718820460FF011FD68B2658104B05C
:10027000BDE8F087802D64D02FD8522D00F05B812F
:1002800007D8442D7FF45EAF002A58D0784B136016
:1002900055E0542D00F055816E2D7FF453AF754B12
:1002A0000A681B88511CFF2BA8BFFF23724D2160D9
:1002B0001370A968204681F3100189B20FF0E6FCA3
:1002C0006E4B204619880FF0E1FC2968204601F3A7
:1002D0000F0189B20FF0DAFC31E0822D00F0898045
:1002E0000FD3A02D6FD0FE2D7FF42CAF0025644ED0
:1002F00036F81510204601350FF0C8FC042DF7D153
:100300001DE04FF6FF765F4B0A2519689F68B142E2
:10031000A8BF3146236821EAE1715A1C226089B2E4
:1003200020461D700FF0B2FC05FB07F1B142A8BFDB
:10033000314621EAE17189B220460FF0A7FC012580
:1003400093E70A68504B511C1B8821600A21FF2B40
:10035000A8BFFF2311702268511C21601370EEE7C3
:100360000B685A1C0A6000221A700B685A1C0A603B
:100370001D700B685A1C0A6024221A7075E704224B
:10038000424920460FF064FCD9E70B6801255A1C4E
:100390000A6002221A700B685A1C0A601D700B68F2
:1003A0005A190A600022E8E72A46394920460FF028
:1003B0004FFC002120460FF069FC23685A1C226084
:1003C00000221A70BBE7334B204619680FF04AFC35
:1003D000314B204619680FF045FC304B2046196818
:1003E0000FF040FCABE72E4B204619680FF03AFCAB
:1003F000A5E72C4B20461A780B681F4D591C21602D
:100400001A70294BD9880FF041FC1A4B22681B88BF
:10041000511CFF2BA8BFFF2321601370A968204641
:1004200081F3100189B20FF031FC2968204601F3F5
:100430000F0189B20FF02AFC1C4B1A782368591C53
:1004400021601A707BE700BF60060020502B00205F
:100450003A3A0020373A002050410020913F0108ED
:1004600040BE01084CBE010855BE0108D411002051
:10047000A9C20008681700206C1700204A1B002042
:100480003C170020C41000209010002036BE010848
:100490003BBE0108E8F7FF1FECF7FF1FF0F7FF1F57
:1004A000A82200207C200020521B00204D1B002091
:1004B00001250B685A1C0A601D700B685A190A60E6
:1004C00005221A700B685A190A600A221A700B6802
:1004D0005A190A6000221A70AD4B22681978501917
:1004E00020601170226859785019206011709A7834
:1004F00023685919216040E7A64D0B686A78591C9A
:1005000021601A7023682A78591C21601A702368A8
:10051000AA78591C21601A70E98820460FF0B6FBB2
:1005200023682A79591C21601A7023686A79591C3A
:1005300021601A7003E70B685A1C0A6000221A70C7
:10054000FDE60B685A1C0A6000221A700B68591CE1
:1005500021601A70F3E600264FF6FF788E4FDFF821
:1005600068920096019602960396F157481C0BD0AC
:1005700048FA06F3DA0707D5B9F800303341DB074C
:1005800002D502A811F043FF01360B2EEDD1002653
:100590000FF2F419D9E9008932464046494615F070
:1005A00071FD002100F0010050EA010307D0F0B214
:1005B00010F0F8FE18B1314602A811F028FF0136FC
:1005C000242EE9D1754BDFF804821B78DF074FF04A
:1005D00000073E4642BF029B43F0010302933946A7
:1005E000404611F020FF48B1394602A811F01BFF28
:1005F00018B13146684611F00AFF01360137242F41
:10060000EDD1674B2046B3F850100FF03FFB0021AF
:1006100020460FF03BFB634B20461968624F4A01AE
:10062000C1F3400302F020021343C1F3800243EA06
:100630004203C1F3C00243EA8203C1F3401243EA1A
:10064000C20301F0100119430FF020FB0422694698
:1006500020460FF0FDFA23683A78591C21601A7081
:10066000524B204619886429A8BF64210FF00EFB65
:10067000962D18D123685A1C226003221A70236811
:100680007A78591C21601A700822193E96FBF2F202
:10069000236882F30402591C216020461A7001A9C4
:1006A0000FF0D6FA4BE6002120460FF0EFFAEBE709
:1006B0003F4815F0DFFC00233B4998427FF73FAEEF
:1006C0005A18157922680133561C26601570F4E714
:1006D0001022384920460FF0BBFA30E600251826D4
:1006E000354FDFF8EC8006FB0573597C31B92046A5
:1006F00001350FF0CBFA082DF5D120E658F825008A
:1007000017F038F981B2F2E736F8151020460FF0ED
:10071000BDFA01353B789D42F6DB10E6274D2046B9
:1007200029880FF0B3FA698820460FF0AFFA0A2340
:10073000B5F90410204691FBF3F189B20FF0A6FA47
:10074000FDE5204600210FF08DFA002120460FF034
:100750009DFAF4E51A4D204629880FF097FAA988EA
:1007600020460FF093FA298920460FF08FFAE6E52C
:10077000144B22689978501C206011705A782368B5
:10078000591C21601A70DAE590E33FF4080000007C
:10079000D0110020521B002062A00108301B002055
:1007A0003800002060190020582000208020002000
:1007B0005C20002078170020502B002018330020E8
:1007C000000D002016120020141F0020940D0020A0
:1007D000481700200021AC48036801EB41029D5CF2
:1007E000236801315E1C26601D7003680A291344CA
:1007F0005D78236803F1010626601D7003681344C9
:100800009A78236803F1010525601A70E4D196E512
:100810002168481C20600A7013F8012F002AF7D1C4
:100820008DE5012523685A1C22601D701DE5974D3A
:100830002046A9890FF02AFA698920460FF026FA86
:100840007DE5934D23682A7A591C21601A70A98B83
:1008500020460FF01BFA298B20460FF017FA698B00
:1008600020460FF013FA2368EA7C591C21601A70A5
:10087000E98C20460FF00AFA298D20460FF006FA7F
:100880002368AA7F591C21601A70236895F82020DC
:10089000591C21601A70A98C20460FF0F7F92368C3
:1008A000EA7A591C21601A70E96820460FF0DAF9DB
:1008B00023682A7C591C21601A70236895F821202E
:1008C000591C21601A703AE5724D23682A78591C28
:1008D00021601A7023686A78591C21601A7069882F
:1008E00020460FF0D3F923682A79591C21601A7029
:1008F000E98820460FF0CAF923682A7A591C21603A
:100900001A701CE5236816F81510581C06EB4502F2
:10091000206019705178204601EB810101EB8101C3
:1009200001F2EE2189B20FF0B1F901353B789D4219
:10093000E8DB04E5564B5A7D2368591C21601A7088
:10094000FDE40025544E56F82510204601350FF0E1
:1009500089F9202DF7D1F2E44F4D002306272846D0
:10096000002107FB03F6226802F1010EC4F800E043
:100970001370226802F1010EC4F800E011708A19A8
:100980002A4492F8C0E02268013102F1010C0629E4
:10099000C4F800C082F800E0E5D10133062BDFD1B6
:1009A000002221684D1C25600B7021684D1C2560BC
:1009B0000A70811891F8E450216801324E1C0B2A0C
:1009C00026600D70EDD123685A1C226007221A7030
:1009D00023685A1C226000221A70236890F8F020C5
:1009E000591C21601A70AAE411F07EFD002814BF82
:1009F000032202222368294D591C21601A7029887C
:100A000020460FF02FF9E96820460FF02BF911F07E
:100A10004BFD014620460FF025F990E4012523689F
:100A20005A1C22601D701E4B226899785019206054
:100A30001170226819785019206011705A7857E5A2
:100A40000025236829465A1C22601D702368204611
:100A50005A1C22601D7023685A1C22601D700FF002
:100A600001F9294620460FF0FDF868E40D4D2046B7
:100A700029880FF00BF9698820460FF007F9A9883B
:100A800020460FF003F95AE42C19002020390020E9
:100A90003419002044330020B01900207C040020C9
:100AA0008C41002030390020B54B1A782368591C3E
:100AB00021601A70B34B9A782368591C21601A7010
:100AC000B14B9A782368591C21601A7037E4B278C8
:100AD000591C21601A70AD4B1A782368591C21608B
:100AE00000F073BEA64E23687279A94D591C21608F
:100AF0001A702B682046198C0FF0C8F82B68204616
:100B0000598C0FF0C3F8718920460FF0BFF8B189F6
:100B100020460FF0BBF82B682046998C0FF0B6F8F2
:100B20002B682046D98C0FF0B1F8F18920460FF0E0
:100B3000ADF8318A20460FF0A9F800E4914BDA783D
:100B40002368591C21601A70924B1A782368591C2B
:100B500021601A708C4BDA782368591C21601A7056
:100B6000FFF7EDBB72689A420FBF00215A1C32603A
:100B70001978894A20460BF0CBFBFFF7E0BB72687F
:100B80009A421DBF5A1C326019780021834AF1E74E
:100B90009DF8083009FB03835B7CC3B19DF80830E6
:100BA00009FB03835B6993B19DF808304A2109FB77
:100BB000038358692B7846F8230012F09FF82B78AE
:100BC00056F8230012F0C1F82B7801332B709DF8F2
:100BD00008300133DBB28DF80830FFF7FFBA226826
:100BE000511C21601370FFF7AABB472D4AD17268D0
:100BF0003046D51A0FF00BF8052D07463FD9304681
:100C00000FF01BF80026054694E80C009B1A103BD9
:100C1000634AAB42A846B8BF9DB2D3683946DB1BD6
:100C20009D42204688BF9DB291460FF01BF83EB909
:100C3000294620460FF02AF823685A1C22601E70AD
:100C4000D9F80C307A199A42D4F800A088BFDD1B7D
:100C500011F028FD2A465146384611F07FFD2368E1
:100C600003442360002E3FF46AAB002280457FF7E7
:100C700066AB23680130591C21601A70F6E7012623
:100C80008025C1E7292D2AD0392D1ED0212D35D11F
:100C90005A1C32601A46434D12F8021B30466970E6
:100CA00032605A782A70DA1C32609B78AB700EF092
:100CB000C4FF3368E8805A1C32601A4612F8021BDF
:100CC000297132605B786B7105E05A1C32601A78CA
:100CD0000A2A00F082874FF0FF35FFF7C6BA5A1C88
:100CE00032601B780A2BF6D130460EF0A6FF2E4D4F
:100CF000288030460EF0A1FF6880ECE777685D2D14
:100D0000A7EB030700F0A08300F25C81352D00F013
:100D1000808200F2B2802B2D00F035844CD8232D38
:100D200000F05F8217D80B2DD5D1002111221F486A
:100D300019F0EBF8102F4FF0000328BF10271C49C3
:100D4000BB42BFF4FCAA3268501C306010785A18BD
:100D500010710133F4E7252D00F00A84272DBAD154
:100D600030460EF06AFF134D286030460EF065FFE6
:100D7000686030460EF061FFA860FFF7E0BA00BF80
:100D8000963A0020203900200A120020BC320020B0
:100D90002C1900200212002087C20008F1C10008AF
:100DA0007C040020521B0020D41100205C20002075
:100DB00058200020000D00202F2D00F00E844FD869
:100DC0002D2D88D15A1C32601B78B74D30462B72BE
:100DD0000EF033FFA88330460EF02FFF28833046F5
:100DE0000EF02BFF336868835A1C32601B78082F83
:100DF000EB747FF6A4AA30460EF01FFFE88430465D
:100E00000EF01BFF0C2F28857FF699AA3368304619
:100E10005A1C32601A4612F8021BA97732605B78BE
:100E200085F820300EF009FF102FA8847FF687AADE
:100E3000336830465A1C32601B78EB720EF0E7FEC6
:100E40003368E8605A1C32601A78162F2A747FF6CD
:100E500076AA9A1C32605B7885F82130FFF76FBA6A
:100E6000312D00F0D383332D7FF435AF5A1C32601F
:100E70001A788D4B5A75FFF762BA482D00F07483CB
:100E800039D83C2D3FF45BAA23D8372D7FF423AF0C
:100E90000723B7FBF3F3C3EBC302BF1A7FF41BAF07
:100EA000DFF81CA25FFA83F8FBB243453FF447AA80
:100EB000002533685A1C326093F900300AEBC509EB
:100EC00099F902209A4200F0B2860135052DF5D13C
:100ED00001E73E2D00F07981412D7FF4FCAE002327
:100EE00071493268501C306012785A540133082B13
:100EF000F7D1FFF724BA4E2D00F04C8320D84C2DAB
:100F00007FF4E9AE5A1C32601A46684D12F8021B93
:100F10003046297032605B786B700EF08EFE33685D
:100F200068805A1C32601B7830462B710EF085FEAB
:100F30003368E8805A1C32601B782B72FFF7FFB9C8
:100F4000512D00F0FC825B2D7FF4C5AE5A1C32603F
:100F50001A46574D12F8021B564FA9703260597845
:100F6000554A30461170DA1C32609A783A711A1D6F
:100F70003260DB78042BA8BF0423BB700EF05DFE4B
:100F800096E80C009B1A012B388003DD30460EF0EA
:100F900054FEF881336872689A4206D05A1C326057
:100FA0001B78003318BF0123EB710BF0DDFA3368B7
:100FB00072689A423FF4C3A95A1C32601B78FB70D6
:100FC000FFF7BDB9D42D00F0948100F29780CC2DAD
:100FD00000F0468176D8612D00F07B8241D85F2DEC
:100FE0007FF479AE30460EF028FE30460EF025FE36
:100FF00030460EF022FE3368304D9A1CD5F8008042
:1010000032605A78304688F82F20DA1C32609A789D
:1010100088F83A201A1D3260DA78073388F83B20C6
:1010200033600EF00AFEA8F83E003046D5F8008086
:101030000EF003FE112FA8F83C002B460CD93268A5
:101040002868511C3160114611F8025B80F831505C
:101050003160527880F8322018680DF0CBFAFFF733
:101060006EB9C82D3FF46BA9CA2D7FF434AE134B73
:101070001868034600F11E0532680333511C3160C5
:10108000114611F8027B03F8037C3160517803F8B4
:10109000021CD11C3160927803F8012C9D42EBD1E7
:1010A0000DF0A8FAFFF74BB93419002044330020A3
:1010B000963A002098170020BC3200202C190020FE
:1010C0000E400020CE2D00F02E82C0F02182D02DC7
:1010D00000F01182D22D7FF4FEAD5A1C32601878D8
:1010E00006065ED4C04B1B78DD073FF528A9032810
:1010F00028BF00200BF068F9FFF721B9DC2D00F0C4
:10110000918125D8D92D00F04B8113D8D62D7FF4AD
:10111000E2AD0025B54FDFF800833B789D42BFF676
:101120000EA930460EF089FD15F010FD48F8250097
:101130000135F2E7DA2D00F04281DB2D7FF4CBADF3
:10114000AB4B4A22AB49186816F0AEFAFFF7F7B876
:10115000EF2D2FD014D8DD2D00F06B82DE2D7FF423
:10116000BAAD30460EF069FDA34D288230460EF030
:1011700064FD688230460EF060FDA882FFF7DFB89C
:10118000F22D00F0E280FA2D7FF4A5AD964B1B788E
:10119000DB073FF5A0AD0BF02DF90BF05FFAFFF781
:1011A000CEB800F07F00032828BF002014F04EFFC7
:1011B000FFF7C5B830460EF040FD904DA88130468F
:1011C0000EF03BFD6881FFF7BAB85A1C32601A4630
:1011D0008B4912F8020B887032605B784B70FFF716
:1011E000AEB85A1C32601D78132D3FF674AD002145
:1011F0000C279A1C32605A78DFF820E207FB01E0E6
:1012000090F808C0944500F0F78401312429F5D105
:1012100061E55A1C326019780E293FF65CAD9A1CC4
:1012200032605D78032D3FF656AD06224A4375487D
:1012300081184D71DD1C35609D7885541A1D326012
:10124000DA784A705A1D32601A798A709A1D3260B3
:101250005A79CA70DA1D32609B790B71FFF76FB84B
:10126000092F7FF638AD68495A1C0D6832601A465E
:1012700012F8020B8846287032605B78681DAB70EC
:101280000023022B0CBF4FF0FF0E4FF0640E3168AD
:1012900001334A1C32600A787245A8BF7246032B9C
:1012A00000F8012BEDD18B1C33604B783046642B5A
:1012B00028BF64232B72CB1C33608B78EB700B1D23
:1012C0003360CB782B710EF0B8FC0A2F68810CD0FC
:1012D0003368D8F80020591C316019780B2F5172EF
:1012E0001FBF991C31605B78537010F0ABF8FFF7AB
:1012F00026B80F2F7FF4EFAC5A1C32601D78072DF3
:101300003FF6E9AC0C2730460EF097FC6F43DFF850
:10131000108108EB0705A88030460EF08EFCE880AF
:1013200030460EF08AFC336828815A1C32601A4617
:1013300012F8021B3046A97232605B78EB720EF035
:1013400066FC48F80700FEF7FABF5A1C32601A78AC
:101350000F2A3FF6C0AC991C31605D782B48C2EB78
:10136000C20285548118DA1C32609A784A701A1DBC
:101370003260DA788A705A1D32601A79CA709A1D02
:1013800032605A790A71DA1D32609A794A7103F132
:1013900008023260DB798B710DF0ECF8FEF7CFBFFD
:1013A00030460EF04AFC1A4D288030460EF045FCBF
:1013B000688030460EF041FCA880FEF7C0BF194699
:1013C0005A1C326011F8020B124A107031605978C1
:1013D00030465170D91C31609B7893700EF02DFC13
:1013E0000B4BD880FEF7ABBF301B0020441700200A
:1013F0002C19002074AE0108981700202039002015
:10140000161200205C230020383900207D2E002099
:1014100030390020FC110020282B002010BB0108CF
:10142000F02E00205A1C32601A46C64912F8020BF0
:10143000087032605978C44A9170DA1C32609A7828
:10144000C24B9A70FEF77BBF5A1C32601B78C04DAE
:10145000DFF8F0823046D5F8009088F805300EF0BD
:10146000ECFBA9F820003046D5F800900EF0E5FB23
:10147000052FA9F8220023D930460EF0DEFBA8F88C
:101480000A0030460EF0D9FBA8F80C003046D5F81B
:1014900000900EF0D2FBA9F824003046D5F8009059
:1014A0000EF0CBFB0D2FA9F8260009D930460EF01F
:1014B000C4FBA8F80E0030460EF0BFFBA8F81000E1
:1014C0000BF052F813F00DFA28680DF05FF9FEF7F3
:1014D00036BF5A1C32601A469B4912F8020BC8707C
:1014E000326059789B4A1170DA1C32609A78974BB7
:1014F000DA70FEF724BF984B1B78D8073EF51FAF74
:101500000BF070FA0AF076FF0BF0A8F8FEF717BFA1
:10151000914B1B78D9073EF512AF4FF4C8728F4B31
:101520001A80FEF70CBF8C4B1B78DA073EF507AF2D
:101530008B4A137843F004031370FEF700BF894A07
:101540001278012A3EF6FBAE19465A1C326011F899
:10155000020B854A9070316059781170D91C316046
:101560009B785370FEF7EBBE11F0DAF8FEF7E7BE9A
:1015700000237E4D30462B600EF049FB2B6818434C
:101580002860FEF7DCBE5A1C32601A78784B1A705D
:10159000FEF7D5BE5A1C32601F78112F3FF69BAB69
:1015A0009A1C32605B78734D304605F817300EF0A8
:1015B00044FB40F6CA039842A8BF184640F2EE2307
:1015C0009842B8BF18461923A0F2EE2090FBF3F022
:1015D00005EB47056870FEF7B2BE674D05F14007A1
:1015E00030460EF02AFB3368A5F880005A1C3260A2
:1015F0001A4612F8021B043585F87E1032605B78BB
:1016000085F87F30AF42EBD1FEF799BE5A1C3260AD
:101610001D781F2D3FF65FAB052F7FF45CAB304686
:101620000EF0F5FA544B43F8250008F0FBF8FEF7EE
:1016300086BE5A1C32601A4612F8020B3260DA1C5F
:10164000597832609A7808F0C9F800287EF477AEAD
:10165000FFF741BB262D3FF47DA82A2D7EF489ADEE
:10166000434B1A782368591C21601A70FEF767BE35
:10167000302D3FF466A91BD82E2D7EF47AAD3E4D59
:1016800005F14006B5F8801020460EF0FFFA2368F9
:1016900095F88220591C21601A70236895F88320E0
:1016A0000435591CB54221601A70EBD1FEF747BED4
:1016B000322D3FF43FA9342D7EF45BAD2F4B03F167
:1016C0005A0122685879551C2560107022681878D4
:1016D000551C2560107022685878551C25601070C4
:1016E00022689878551C256010702268D878551C9F
:1016F00025601070226818790633551C99422560C0
:101700001070DED1FEF71BBE462D3FF46DA939D80F
:101710003B2D3FF486A808D83A2D7EF42AAD00214F
:1017200020460EF09FFAFEF70ABE3D2D3FF420A89A
:10173000402D7EF41EAD0822114920460EF088FA95
:10174000FEF7FDBD963A0020203900200A12002045
:101750002C19002002120020301B002048250020F8
:10176000C4160020901700208C410020A8220020E1
:1017700031190020A1380020B01900205C2300207E
:10178000341900204F2D3FF45BA90AD84B2D3FF4AC
:101790009BA84D2D7EF4EDAC0025B14FB14EFFF767
:1017A000C5B8502D3FF43AA95A2D7EF4E2ACAE4EA6
:1017B0002368F278002A3FF48AA95A1C2260082282
:1017C0001A7023685A1C226001221A70A74D2368E0
:1017D0002A79591C21601A702368AA78591C216043
:1017E0001A70298820460EF051FAE98920460EF039
:1017F0004DFA2368F279591C21601A702368EA783F
:10180000591C21601A70FEF79ABD702D3EF4E2AFAC
:1018100000F2E180672D3EF45BAF00F28A80602D1C
:101820003FF48CA94FD85E2D7EF4A3AC0021204656
:101830000EF02CFA002120460EF028FA0021204656
:101840000EF024FA23688A4D5A1C226000221A7076
:101850002B6893F82F102368581C206019702B6890
:1018600093F83A102368581C206019702B6893F87D
:101870003B102368581C2060197023682046591CAF
:1018800021601A702368591C21601A702368591C42
:1018900021601A702B68D98F0EF0F8F92B6820465A
:1018A000998F0EF0F3F92B6893F831202368591CB7
:1018B00021601A702B6893F832202368591C21602C
:1018C0001A70FEF73CBD652D3EF445AE662D7EF4E4
:1018D00050AC684E0025328AB2F5007F8CBF0427D9
:1018E00001277319596B204691FBF7F1043589B232
:1018F0000EF0CCF90C2DF4D101255F4E5F4F396A03
:1019000056F8250015F02EFA16F034F8013581B29C
:1019100020460EF0BBF9042DF1D10025584E36F8C3
:101920002510204601350EF0B1F9032DF7D1FEF751
:1019300006BD6C2D3EF4F2AE0AD8682D3EF4CEAE54
:10194000692D7EF416AC0025454F4E4EFEF7E2BEE3
:101950006D2D3EF4F6AE6F2D7EF40BAC4A4D2B6828
:101960001A782368591C21601A702B689A782368AA
:10197000591C21601A7000232A681A445179226880
:101980000133501C032B20601170F5D12B682046C9
:101990001A7A2368591C21601A702B68DA78236838
:1019A000591C21601A702B681A792368591C216010
:1019B0001A702B6859890EF069F92B685A7A2368D6
:1019C000591C21601A702B685A782368591C2160B1
:1019D0001A70FEF7B4BC7E2D3FF466A826D8782D89
:1019E00000F08B8005D8752D7EF4C3AB274BFEF736
:1019F00013BF7C2D3FF43AA87D2D7EF4BAAB244B67
:101A000022681978501C2060117022685978501C87
:101A1000206011709A7823682046591C21601A7042
:101A20001C4BD9880EF032F9FEF789BC962D3EF496
:101A300092AD31D87F2D3EF48FAF832D7EF499ABDC
:101A40000A4D2046298A0EF021F9698A20460EF0B7
:101A50001DF9A98A20460EF019F9FEF770BC00BFE7
:101A6000FC370020A1380020963A0020981700206B
:101A70002C190020F8160020FC3F0020A83A002076
:101A800008360020EC1E0020383900206CA0010828
:101A9000FC11002030390020F02D3EF4C8AEF12DAD
:101AA0007EF467AB724B03F1700122681878551C05
:101AB0002560107022685878551C256010702268C7
:101AC0009878551C256010702268D878551C2560C0
:101AD000107022681879551C25601070226858799A
:101AE000551C25601070226898790733551C99425F
:101AF00025601070D9D1FEF722BC5E4D05F160065D
:101B0000A98820460EF0C2F8E98820460EF0BEF8FB
:101B1000298920460EF0BAF82368AA7A591C216058
:101B20001A702368EA7A591C21601A7055F80C1B48
:101B300020460EF097F8B542E2D1FEF700BC4E4DBC
:101B40004E4F05F12806002395F90220D9579142FE
:101B500026D00C333C2BF9D10835AE42F3D1FEF739
:101B6000EEBB474D05F1500628780AF0BDFB23680F
:101B7000027A591C21601A7023686A78591C216006
:101B80001A702368AA78591C21601A702368EA78B1
:101B90000435591CAE4221601A70E5D1FEF7CFBB67
:101BA00023682046591C21601A7029880EF06EF8AF
:101BB0002368EA78591C21601A7023682A79591C15
:101BC00021601A702368AA79591C21601A70236851
:101BD0006A79591C21601A70BEE79A1C32605978E4
:101BE000284A1170D91C316099785170191D3160E3
:101BF000DB789370FFF76FB80178214A002002F874
:101C00002510D91C3160997802EB85025170191D9D
:101C10003160D9789170591D31601B79D3700FF004
:101C200087FB194B80F001001870FEF788BB89F81C
:101C3000023030460EF001F833682AF835001946B4
:101C40005A1C326011F8022B013789F803203160E9
:101C50005A7889F80420DA1C32609A7889F80620CC
:101C60001A1D3260DB7889F80530FFF71DB900BF17
:101C70007D2E0020F02E00200E4000203C40002051
:101C8000BC220020D0110020000000202DE9F04FE0
:101C90000B4B0C4D0C4AC5F8B834002310680B49A7
:101CA000A1B08842C5F8BC3416D1136062B6084BA7
:101CB00018680BF08BFB074B1B689847FEE700BFCB
:101CC00093F4000868060020F04F0020EFBEADDE60
:101CD00000F0FF1F04F0FF1F0A930B930C934FF4C7
:101CE000E013BB4C0D93236843F480332360A36956
:101CF00043F01003A361236803F400330B930A9BA2
:101D000001330A930B9B1BB90A9BB3F5A06FF2D169
:101D1000236813F4003300F0B08202230C93AD4B20
:101D2000AD491A6842F010021A601A6822F00302E4
:101D30001A601A6842F002021A606368636063689E
:101D40006360636843F480636360A44B1A68043B78
:101D500022F070425A60A24A1160616821F47C113D
:101D60006160596841F000415960D96821F400412F
:101D7000D9609B681F0449BF9A4B4FF4E01313606E
:101D80004FF480130D930C9B012B00F08E82022BDD
:101D900005D10D9B61680B4343F480336360236876
:101DA00043F08073236023689E01FCD5636823F0B1
:101DB00003036360636843F002036360636803F0D6
:101DC0000C03082BFAD16368874F03F00C03042B34
:101DD00000F06F82082B00F06E827F4B3B606368DF
:101DE000DFF84882C3F3031318F803203B68DFF8D9
:101DF0004092D3403B607D4B4FF0000AC9F8083059
:101E00007B4B0DF1800BC9F80C30A369794E43F080
:101E10000103A361636A636A304643F080736362BF
:101E2000A36943F01C03A3614FF6FF732BF82C3D0D
:101E300059468DF856A011F0FDFA59466E4811F03A
:101E4000F9FA59466D4811F0F5FA10238DF846302D
:101E500002238DF847304FF4007320A921F83C3D50
:101E60003046336111F0E6FA654A5846536843F04C
:101E7000007353600BF09CF8159B624A3046B3FB2D
:101E8000F2F34FF47A72C5F8C0343B684646B3FBB0
:101E9000F2F35D4A013B5360F02389F823300723B6
:101EA0004FF0010CC2F808A0DFF888E11360574A30
:101EB00008F10E01002331F8027F47FA03F818F009
:101EC000010F18BF0CFA03F803F101031EBF1060E5
:101ED000A2F804800832102BEFD100F58060704525
:101EE000E8D10DF025FD18B90AF07CFD0AF082FA60
:101EF0000AF0B4FB95F8C434454F43F0010385F86C
:101F0000C434444BDFF830919A78434B09F1060A08
:101F10001A70424B1B683B6095F8C93485F8C5348C
:101F2000002313F809004FEA830B03F1010800288E
:101F300000F0D281039310F0BBFE039B4AF823000C
:101F400018B1052380F80780837112215AF80B001D
:101F500010F0D4FE4346032BE3D10021084610F0D5
:101F60002FFF0021012010F02BFF0021022010F094
:101F700027FF0121022010F023FFA369002143F075
:101F80000103A3614022264817F0BFFF4FF0FF3343
:101F90000024244AC5F818356420C2F8033010F034
:101FA000DEFDA0220021204817F0AFFF144ADFF821
:101FB0008C805368DFF8889023F4406343F07063AB
:101FC00043F400635360002354F808003AE000BF74
:101FD000001002400020024000127A00041001406C
:101FE000DC030020001BB7001003002000000008E5
:101FF0000005FA0500080140000C014000100140F6
:102000000000014040420F0010E000E0842000206A
:10201000601B00205820002030190020A82200203A
:10202000400B0020800B0020A8240020A0A0010865
:1020300000ED00E0001401402E0B002038A501083F
:10204000B8A0010859F83310DA00884240F04781FF
:10205000B318187F103412F06BFBC02CB3D1B24C04
:102060000021A146B14ADFF8CCE200260B5D01F168
:102070000F0020440EEB030A10F8018FB8F1000F97
:1020800005D09AF80CC0C44508BF82F858C090F833
:102090000380B8F1000F05D01EF803C0C44508BF87
:1020A00082F859C00136032EE6D1B2F8580040B18B
:1020B00009EB010005EB83035065C3F8202502F509
:1020C00017721C313829D0D10524DFF860823C22F8
:1020D0000021974888F82C453D6817F016FF954B6E
:1020E000224693F80BC093F80A900023904CCDF849
:1020F0000C801846A0464FF0FF0ADFF890E205F08A
:1021000040061EF9011F1E29195540F0EE80002ED1
:1021100000F0F380B9F1000F00F0EF800C333C2B9E
:10212000EFD110B1039B83F82C25834B834C93F89C
:1021300000A0834E834B15F4805214BFA088B08A50
:1021400083F800A09946059214F004FD7E4ADFF85A
:1021500040821060308A069214F0F8FC7B4B1860C5
:10216000708A14F0F3FC7A4B1860608814F0EEFC6F
:10217000784B1860208814F0E9FC774B1860B8F8A9
:102180001A30C3F5FA60049314F0E4FC7349B8F80C
:102190001880049BB4F806B00860A8EB0300A0EB1D
:1021A0000B0014F0D7FC6E4B1860C8F5FA60A0EB7A
:1021B0000B0014F0CFFC6B4B069A18606A4B9046EC
:1021C0002B406A4A002B40F09E80694B03EBCA0A01
:1021D0009AF80130136040F2DC510023654A22F87E
:1021E00013100133082BFAD1B38A0493059B0BB16A
:1021F000A3880493B378042B05D14FF480500DF0DD
:102200008FFB00230493002599F800205A4CA2F17B
:102210001703022B257000F2BF804FF0000BDFF890
:102220007491594655F8090005EB090A14F07AFE35
:1022300000286AD03B68DA0400F1CF800023D8F888
:1022400000104E4A42F823100133082BFAD12378AC
:10225000C02200214A48069317F057FE3779B37819
:10226000003718BF0127042B00F2DC80DFE813F0F1
:102270008501DA008701DD007F01226842F001025A
:1022800022600A93236803F002030B930A9B013335
:102290000A930B9B1BB90A9BB3F5A06FF2D123687D
:1022A0009B0701D5012339E5FEE7636843F460131A
:1022B00074E5136892E563686168C3F38343C803F8
:1022C00003F1020302D42F4A534387E56168126881
:1022D000890348BF5208F7E74AF823003AE601337A
:1022E000042B7FF4AFAE0020B4E61F297FF416AFB5
:1022F0001EB1BCF1000F7FF411AF013A08F803A042
:10230000D2B201200AE7012364E71F4B05EB030E5D
:102310009AE80F008EE80F00237810350133802DE6
:1023200023707FF47EAF85E7D8A0010868060020FF
:102330003C4000201C2A00203119002030390020A8
:102340009817002040120020982C0020B017002081
:10235000CC110020681200205C12002074120020B2
:1023600064120020701200202000100000130020D2
:1023700070AB01087817002044170020282B00209C
:10238000502B002000093D007C1200200FA1010805
:1023900034190020A4210020B44B13F8321003EBB1
:1023A000C2030829217088BF0821D3F804C088BF60
:1023B0002170BCF1000F3FF43DAF0025DFF8109312
:1023C00023789D42BFF636AF2B0103EB090E634421
:1023D0000FCB01358EE80F00F2E72378012B7FF653
:1023E0002DAF4FF07C59A24D05EB031303F11007FD
:1023F0001035BD423FF422AF494655F80C0C14F09D
:10240000FDFB494645F80C0C55F8100C14F0F6FB92
:10241000494645F8100C55F8080C14F0EFFB45F848
:10242000080CE5E7934CA04602E0934CDFF8A48249
:10243000924A934B21461A60924A934B4046002F92
:1024400018BF1346914A0025136014F0CFFA0146D5
:102450004FF07A5014F086FC8D490590204614F018
:10246000CDFB8C4CDFF870A20790069BAB4240F38B
:10247000E58005EB0A035E79002130460AF0D0FBC7
:10248000834600287DD1844A7D4B1A607D4A7F4B6C
:102490001A60824C82482368002B40F01F81037829
:1024A00003F0EF02082A7F4A40F03A811178182B96
:1024B00041F01001117001D10CF05CF82368002B81
:1024C00040F03781784A794C1368079213F001067F
:1024D00040F076819B0440F1C08194F81826744B3B
:1024E00004F5A8651A7004F5C26816F80890002172
:1024F00048460AF095FB074698B300224FF0010AC0
:102500005FFA86FB05F80FBC45F8040C05F80E2CA5
:1025100005F8062C05F810AC484610F0C9FBD3446A
:102520005FFA8BFB18B180F806A080F807B04FF077
:10253000000B2A2110F0E2FB5E4A0021384610F021
:1025400013FA5D4B2A1D2B605C4B294638466B60A5
:10255000C5F808B010F05CFA5A467979386808F086
:10256000F7FF0136082E05F11C05BED175E10024E8
:102570000023A046012704935AE7454CF8E7504C46
:1025800051E7304610F094FB6B1C6061DBB210B178
:102590000322C37182711A2110F0B0FB002F51D0B9
:1025A000BAF8000014F0D6FA14F02AFD454B4FF6A5
:1025B000FF791E68B6FBF0F34B441B0CB6FBF3F639
:1025C0000FB1B6FBF0F99AF80230042B3ED1484621
:1025D00014F0BCFA2E4914F011FBA06009903046AB
:1025E00014F0B4FA414614F009FB099B08903649EF
:1025F000184614F003FB089A0146104614F0F4F94B
:102600009AF80330E0600193049B324600935946E8
:102610001FFA89F3204613F0B7FC002318221D4946
:10262000AB4218D1002383F00103237401231D441E
:10263000082D637404F118047FF417AF0122234BB3
:102640001A7026E7059815F00BF9ADE7304614F03F
:102650007DFA0799BFE702FB03104668606886426F
:1026600001D00133DCE70123DDE700BF70AB0108D7
:10267000801200206F120339ACC5A7378DB0000857
:102680003C3A00200DAE0008B9B00008C832002066
:102690006F12833A502B00200FAE00080013002069
:1026A00040120020C4160020601B00206806002095
:1026B000402A002040420F008DB5000883AC00087E
:1026C000282930381003002000007A443A3A0020CC
:1026D0007C120020ACC5A736981700200278324B38
:1026E000324913F8325003EBC2035E680D70002EBE
:1026F0003FF4D5AE00232E4FAB42BFF6D0AEC3EBB6
:10270000C3017218D2F800C001EB070E41F807C0F0
:1027100091880133AEF8041092798EF80620EBE729
:102720000E2B3FF4C3AE1178192B21F0100111705C
:10273000C1E600244FF0040A1E4E1F4DDFF87C90C6
:10274000A6F1030816F8017F002F3FF4BBAE384610
:1027500010F0AEFA013483466861E4B210B180F83B
:1027600006A0C471002138460AF05AFA07461A2119
:10277000584610F0C3FA002F3FF4A4AE0022B8F878
:102780000230019299FBF3F3B8F800209BB200925B
:1027900028460A4A394613F0F7FB0123082C6B74CC
:1027A00005F11805CED18DE6D0A901080C2E002028
:1027B0000D2E002029350020442A002040420F0021
:1027C0000025FF2294F82D75C54B294638461D700B
:1027D0005D609D60DD601D6483F8442083F84520C2
:1027E00083F8465083F8475083F848500AF018FAA7
:1027F000064690B30368BB496A18507C18B152680A
:10280000934200F03D841835C02DF5D10025C4F861
:102810003C6584F83055384610F04AFA10B102236E
:10282000C571837100252A2110F068FAAE4A002193
:10283000304610F099F8AD4BAD4AC4F84035AD4B79
:10284000111F3046C4F84435C4F8485510F0E0F87C
:102850002A467179306808F07BFE94F8C434B4F8E5
:102860001E7643F0040384F8C434A4F8207694F868
:102870001A06002F40F00F8410F01AFA94F81B2665
:10288000C4F82406003218BF012284F8282650B16B
:10289000242294F81C368271002BC7710CBF1221C0
:1028A000162110F02BFA002010F05EFA924B002057
:1028B000C4F8483610F0A0FD022010F09DFD4FF046
:1028C000000C8E4800F1200E50F8055CA5B310F9FD
:1028D000093CE21892F84C6692F84E7692F85086CF
:1028E00004EB0311821E12F8019FB14592F8029089
:1028F00008BF81F85866B94592F8049008BF81F87E
:102900005976C14508BF81F85A868242EBD104EB63
:10291000031393F858267AB193F8592662B193F8C5
:102920005A264AB14279C3F8545683F85B26827915
:1029300083F860C683F85C2610308645C4D1142025
:102940000CF0CCFD2C200CF0C9FD00200CF082FE18
:1029500001200CF07FFE6A4B03991E795D79771E8A
:102960007A4205F1FF3E7A41DEF1000343EB0E03AC
:1029700081F87836079B81F874261B68142203F4CB
:102980000047C3F3C03381F876365E48002117F064
:10299000BCFA012E01BF039B039A93F8753682F8A7
:1029A0007C361FB194F8773684F88B3694F87A36F3
:1029B0001BB194F87B3684F88636012D08BF94F855
:1029C0007936504D08BF84F8813600232E464FF0EB
:1029D000070B1F469946DFF8488108F1980A3078BE
:1029E000E8B110F065F918B180F806B080F80790EA
:1029F000002110F083F9002331781AF813005A00EF
:102A0000884240F0778308EB020393F899307370A3
:102A10000723337101237A1CB770F370D7B20BF11F
:102A2000010B5FFA8BFBBBF10B0F06F10506D6D14C
:102A3000002B00F0DE80344E4920736843F440439D
:102A4000736011F075FE314A314900234FF01C0EBE
:102A5000104688460EFB032CDCF804C08C4540F081
:102A60004F83DBB21C2101FB0303726919694FF02C
:102A700000090A437261062283F819901A762448E5
:102A80000AF01DFA15A80AF0EFF9224B022F159350
:102A900034BF4B4680231A934FF480731B934FF43B
:102AA00080631C9320231D934FF400531A4E15A9E5
:102AB000174818971E931696CDF85C90CDF8649041
:102AC000CDF87C900AF0DDF9012F94BF002201229D
:102AD000D8F80030114943F00103C8F8003021E074
:102AE0005C240020502B002040420F00A9AC0008BD
:102AF000AC0B0020DDAD00081C2A002021A101083C
:102B0000521B0020E40C002000100240140300209F
:102B1000080002404C240140F80C00200024014031
:102B2000A0A001084B684FF0070E23F4702323F494
:102B3000807343EA02234B608A68C54B134043F419
:102B4000602343F002038B60CA6A7B1E22F470028A
:102B5000DBB242EA0353CB621F270123EA784AB370
:102B600095F80180581CB8F1090FC0B295F804C05F
:102B700040F2CC82A8F10A02D1F80C9002EB42029A
:102B80000EFA02FA29EA0A090CFA02F242EA0902EA
:102B9000CA60062B00F2C78203F1FF3C4A6B0CEBC4
:102BA0008C0C07FA0CF322EA030308FA0CF21A431E
:102BB0004A6303460535AE42D0D1A64B9A6842F42B
:102BC00080729A609A6842F001029A609A6842F0B4
:102BD00008029A609A681607FCD49A6842F00402C8
:102BE0009A609C4B9A685507FCD49A6842F4A002FC
:102BF0009A60D4F89806002841F04481D4F89C36B5
:102C0000002B41F03F81D4F8A036002B41F03A81EF
:102C100010220021904817F078F913238F4D2320BC
:102C200085F84D300023EB610FF099FF8C4BE8697C
:102C3000AB6110B9142010F03BF8E86118B11C2307
:102C400083710023C371132110F058F8E86910F064
:102C50007CF84FF48071A8690CF04EFC80226B2147
:102C600080480CF0E3FC06267E4F96200FF077FF9D
:102C7000752138460CF0A9FC682800F07182013EED
:102C800016F0FF06F1D1002195F84B3085F84A1077
:102C9000032B41F0B280744B744A2B60744B904606
:102CA0006B60744BEB60744B2B62042385F84A30E5
:102CB000136843F001031360704B93F80390D971CC
:102CC0009B46B9F1000F03D0B9F1070F40F06082C5
:102CD00002239BF80200DFF8DCA185F84730431E91
:102CE00085F8483013F036FF514613F087FF14F093
:102CF00087F9594E85F846903060584810F01CF915
:102D00009BF800300BB185F84A305D4D11F0E9FDBC
:102D10005C4E44220021284617F0F7F897E803009C
:102D200005F1080305F1200783E8030096E80F008A
:102D300087E80F0001204FF6027736F8053C524E27
:102D4000A5F81B30F278E97E102A134628BF00232D
:102D500000FA03F23A4240F0518212F0FD0F00F007
:102D60004D82032940F04A82484B45482B60484B2E
:102D70006B600423AB76D8F8003043F00203C8F848
:102D800000304FF480732B8210F088F84FF47A7380
:102D90002B63B4F8A436002B40F03882B378002BB4
:102DA00040F03282012194F8C434084643F0020313
:102DB00084F8C43410F004F80021084610F000F83C
:102DC000002102200FF0FCFF0A24324D01200FF0F9
:102DD00060FF00200FF05DFF19200FF0C0FE2B6890
:102DE000D80302D401200FF0BFFF19200FF0B7FE67
:102DF00000200FF0B9FF013CE8D1214620460FF03A
:102E0000DFFF214601200FF0DBFF234B234E186824
:102E10000BF0AEFDB289002A40F00982204B15AFBD
:102E2000587A13F097FE1F4913F0E8FE1E4913F07D
:102E3000DDFD0FF089F91D4B18600BF0E9FD012352
:102E40001593079B1A68510236D4194B159333E03A
:102E5000FDF7F1FF00240140FC3F0020A83A0020CC
:102E600000300140C03A0020392F010860190020CD
:102E70009D310108B92E010890C1793D963A002094
:102E8000F8160020F83A0020203900209D2E010875
:102E9000C92E0108B42200202C190020263500205C
:102EA0000033002035FA8E3CDB0FC93F2033002071
:102EB000010000100000FA42D3005EBF159B43F0F2
:102EC00010031593B54B1968994611F0020F1EBFF8
:102ED000159B43F0C6031593D60542BF159B43F0DF
:102EE00000631593AE4B1978039301F0EF000828A7
:102EF00001D00E2903D1159B43F480531593159BE4
:102F0000D50354BF43F4005343F420431593159B5A
:102F1000D0044CBF43F0644343F0444315939606FA
:102F200042BF159B43F480731593550742BF159B11
:102F300043F400331593159B43F40020159050057E
:102F400005D5984A127912B143F4C0131593182984
:102F500008BF159B4FF0010604BF43F06073159343
:102F60000723169321463846E5B20FF05CFA70B19C
:102F7000284609F0B9F950B9620957F8223005F02E
:102F80001F0506FA05F523EA050547F82250013426
:102F9000242CE7D1844D97E8030005F22C7383E8D5
:102FA00003004FF41972002105F2347016F0ADFFE2
:102FB00005F0AAFC0022DFF834E27C4CCDF810E0EA
:102FC000C4F804E0DFF828E2794BF4461A809A70DE
:102FD0007849794B794E7A481960338BDFF814A21F
:102FE000A06085F8982919B2059005F69C18DAF8C2
:102FF00000002EF8121000F5967048F822000132F9
:10300000122AF4D16F4A9046106810F4805F08BF0E
:10301000B6F92610ACF806106B49DFF8D4C101F1FF
:10302000500E0A78AAB98A7891F803A0524510D2B6
:10303000002A00F00E81013A02EB820202EB8202CA
:1030400002F5617291F801A092B20AF1040A2CF81B
:103050001A2004318E45E4D1010740F17D81307A98
:103060000A2800F27281DFE810F003010301CF03A8
:103070000E046D048D048D04D10470010405030158
:103080001B8D524A9BB212680133B2FBF3F3504AD4
:103090001370FFF7BBBB0FF00BFE4021C4F82406F2
:1030A000C4F8400605461F2009F0BAFD0646CDB11A
:1030B000C0B12423AB7101231A21EB7128460FF014
:1030C0001DFE0021A4F8447601914249424A91FB39
:1030D000F7F192FBF7F389B200919BB231463F487A
:1030E00012F052FF0023D4F82C26138084F83D36CA
:1030F000FFF7DCBB01330A2B7FF47FAC002386E4AF
:103100000133072B7FF4A6AC0023ABE40A6908EB7C
:10311000480A0EFA0AF922EA09090CFA0AF242EA06
:1031200009020A6135E50C2B0DD8DA1FD1F830C041
:1031300002EB820207FA02F32CEA030308FA02F216
:103140001A430A6335E50D3BCA6A03EB830307FAAA
:1031500003FC22EA0C0208FA03F31343CB6228E5CE
:103160000C211F480CF031FA1428FFF48CAD1828FC
:1031700003D9543806283FF686AD032385F84B3033
:10318000432385F85C30174B2B65174B6B657AE54D
:1031900085F84710DFF860A00120A0E56019002045
:1031A00031190020D02D002068060020FC370020B7
:1031B000641B0020A0860100DC37002034190020A9
:1031C00069030108601B0020BC22002010030020BE
:1031D000D803002020A1070040420F00940C0020DB
:1031E000C03A0020FDF500082DF600086D03010827
:1031F000EC1E00204C3A002000007A44012B4FF0D6
:1032000000023FF6A1AD1346AB76CBE50027DFF811
:103210005880B4F8A40613F099FC2A6B014608EB19
:1032200007002C370FF0BAF8842FF2D1B6E5254607
:10323000DFF838800B4FB08913F088FCD8F80020F5
:10324000014678192C350FF0A9F8B5F5B07FF2D109
:10325000E4E50AF1010A0AEB8A0A0AEB8A0A0AF58E
:103260006172EFE628130020100D002014190020D1
:10327000BC4B40201C6012F065FD8346002864D0E2
:103280000023B94A0793137006920AF0F3F9317AD2
:1032900082460129069A0DD0079BC0F0A4820A2914
:1032A00016D1B24B1B6813F480631CBF80F001037E
:1032B000DBB213700322AE4B1A700722AD4B1A70AB
:1032C0000122AD4B1A700C23237042F6F823638061
:1032D000AA4BA54A6360AA4BA3609BF90200BAF10E
:1032E000000F40F08D821378002B0CBF01230323C5
:1032F0001278002A40F08682B27A002A0CBF00229F
:103300000822019200939F4A4FF4E133402105F0D7
:10331000ADF89D4B1860BAF1000F01D09B4B1860BF
:10332000737D2178013BDBB2994A994213709CBFAF
:103330000023137028B18C4B1B7813B1012385F83F
:10334000E439003018BF012030B908200CF0E8FA49
:10335000049B6360059BA36042F20102D8F8003031
:10336000134209D044F6206262809A0440F1A98396
:1033700008222270874A62604FF0000B864CD90306
:1033800084F800B040F1918106F04CFA01232370DB
:10339000824B40F22A3293F8F13059468048049328
:1033A00016F0B3FD049B002B00F0728159461846BD
:1033B00009F036FC7B4A0168044611608168924638
:1033C000002900F06581049B18460FF071FCC5F8D8
:1033D000E80918B1282380F807B083711B210FF08A
:1033E0008DFC0023704ADAF8001002F1180E5EF826
:1033F00033004FEAC30C814240F06A836244107F7D
:1034000011F096F9DAF80000684A03884FF0000BD3
:1034100023F001031B041B0C0380654BDFF8A4E1C0
:103420001B68ADF83EB0934281BF03F1B7726149AA
:1034300002F55852B2FBF1F292BF002202F1FF32C4
:1034400092B2511CB3FBF1F35B49ADF83AB0B3FB58
:10345000F1F303219BB2B3FBF1F14FEA410CAEF85B
:1034600000C0DFF864E18DF840B0AEF8001020A98C
:1034700021F8482DADF83C3011F0A5F96023ADF8E6
:1034800046B0ADF848B0ADF84AB0ADF84CB0ADF8C4
:1034900050B0ADF84EB0ADF852B0ADF84430E3796D
:1034A000DAF800005A0758BF012203F0020356BFA2
:1034B000ADF8462004224FF48072ADF84C304FF046
:1034C00000034CBFADF84820ADF85020ADF84A30AD
:1034D00011AA6179049309F0AFFA6179DAF8000072
:1034E00011F044F9DAF800100120B1F84420049BEF
:1034F0006FEA42426FEA524292B2A1F844200A882F
:10350000DFF8C8B092B242F080020A806279B1F866
:1035100020E000FA02F292B21FFA8EFE2EEA020EAC
:10352000A1F820E0B1F820E01FFA8EFE42EA0E0278
:103530004FF01C0E0A840A8892B202430A80227B52
:103540001E490EFB02121E49D2F810E0D1F814C039
:103550004EEA0C0CC1F814C04FF0280C537682F8D8
:1035600018C035E04438002049380020601B002096
:103570004338002048380020D7360020E5FE0008F8
:10358000710501089106010878380020F42D00200B
:1035900042380020654D0108CC1E0020B0190020E3
:1035A000981B0020C81E0020A0A00108FF6BDC02B1
:1035B00010030020006CDC0200350C001403002016
:1035C00000100240961B0020941B0020C41E002007
:1035D000D1F814C04EEA0C0EC1F814E0BC49536196
:1035E0009160527B8DF855008DF8570038468DF864
:1035F000563004938DF8542009F04CFEA068CBF8A7
:10360000000009F05CFCDBF80000026822F0010217
:103610001204120C026009F052FC384609F024FC36
:10362000DAF80020617934320A44159240F22A32E5
:10363000189280221A92A74A049B1692102217927F
:103640004FF400721B924FF400523946DBF8000031
:1036500019931C931E921F931D9309F012FC62791B
:10366000049B0C2ADAF800109CBF9B4B03EB42032F
:103670008A8998BFB3F8AC3092B21343DBF80020CC
:103680008B81136843F0020313600122934B1A707D
:103690000023FF211C4692481A181C520433802B29
:1036A0009170D170F8D106F02DF98E4B1B6858053A
:1036B00034D5042012F046FB8B4B0421186005F032
:1036C00079F98A4B1870082012F03CFB884B0821CE
:1036D000186005F06FF9874B2C221870002186487E
:1036E00016F013FC7C2385F8EC398E2385F8ED3930
:1036F000E02385F8EF397D23202085F8173A12F072
:1037000021FB7E4B2021186005F054F97C4B18708A
:1037100009F0BAFF09F02CFF09F06EFE794CB4F8FD
:1037200000A0BAF1000F40F02B8295F8180A00288B
:1037300000F026820FF0BCFAC5F81C0A18B11A2353
:1037400080F807A0837113210FF0D8FAD5F81C0A6E
:103750000FF0FBFA00BF02216B480BF0CDFE4FF0DB
:10376000000A9F2332208DF844308DF845A08DF853
:1037700046A08DF847A00FF0F2F98DF855A000BFD4
:10378000D5F81C0A0FF0DCFA042311AA39465E486A
:103790000BF0D1FED5F81C0A0FF0D7FA00BF9DF848
:1037A00056309DF855201B0243EA02439DF85720EE
:1037B0001343564A934200F0118300F38F81544A19
:1037C000934200F094810132934200F0CC81A2F543
:1037D0001A42033A934200F0FC8200232380638064
:1037E000A360E360CCE102214A4A117003214A4AF6
:1037F00011704A4A13700723237045F2F05366E5AF
:10380000032375E508227CE50A221B0193FBF2F3F2
:1038100000224349A3F5B06341F822300132122A55
:10382000FAD142F6F82363803E4B402063603E4B62
:103830002270A36012F086FA824600283FF485AD1C
:1038400009F018FF737AB17A00280CBF0122032215
:10385000002B0CBF0623072300290CBF00210821E1
:103860009AF902E082460B438DE80C002F4B304A58
:103870004021704604F0FAFDBAF1000F3FF461AD4B
:103880002C4B18605DE51023237042F6F82363800B
:10389000294B40206360294BA36012F053FA824603
:1038A00000283FF452AD09F0E5FEB27A00280CBFC3
:1038B00001230323002A0CBF002208229AF902E008
:1038C0000192009382464FF4E1331D4AD0E700BFD6
:1038D0000B2F0108981B0020A0A00108C21E002089
:1038E000A41A0020601B0020EC2D0020F82D0020E1
:1038F000E42D0020E82D002054100020CC2D0020C5
:10390000C92D00207C040020003800401620C20091
:1039100017BA20004338002048380020D73600204E
:10392000083700200DFF000829FF0008A0860100CD
:10393000DD060108F42D002049FE00085DFE0008A8
:10394000CD0401080823237042F6F8236380694BF5
:1039500040206360684BA36012F0F4F982460028AF
:103960003FF4F3AC09F086FE002200280CBF0123CF
:1039700003239AF902E00192009382464FF4E13367
:103980005E4A75E700234FF00C0E5D4A5D491370E7
:103990005D4A062884F800E00B7013702BD01B22C0
:1039A0005A4B4FF4E13B1A700522594B83F800E063
:1039B000584B1A7042F6F8236380574B40206360DF
:1039C000564BA36012F0BEF9824600283FF4BDAC0E
:1039D00009F050FEB27A00280CBF01230323002A0D
:1039E0000CBF002208229AF902E00192009382465D
:1039F0005B464B4A3CE72122444BDFF858B11A7032
:103A0000434B83F800E0434B1870D3E74FF0000AB4
:103A1000444B402083F800A00E23237044F620631B
:103A20006380414B6360414BA36012F08BF9002827
:103A30003FF48BAC03883E4A03F48253B17AB3F56A
:103A4000825F82F800A090F9020014BF01220322D5
:103A500069B9B3F5825F14BF534608238DE80C00A3
:103A60004FF4E133334A402104F000FD69E40823B8
:103A7000F4E70A221B0193FBF2F300222E49A3F57F
:103A8000B06341F822300132102AFAD142F6F8230D
:103A900063802A4B40206360294B2270A36012F0A0
:103AA00051F900283FF451ACB37A90F90200002B91
:103AB0000CBF0023082301930323224A0093224BC7
:103AC000D1E7D8077FF558AC0C2222701F4A52E488
:103AD0000133042B7FF48BAC002091E41C4A934209
:103AE00000F07E8138DC023A93427FF476AE802388
:103AF00070E100BFC1FD0008D9FD00088504010880
:103B000011380020303600201038002031360020D7
:103B10005536002012380020FFFC000815FD000873
:103B2000AD03010846410020714D01087D4D01089B
:103B30004D410020994E01086C370020A900010872
:103B4000D900010831070108A0680600594D010895
:103B50001920C20090D00300AE4A9342C7D0013270
:103B600093427FF43AAE4FF4807323806380A3883E
:103B700022881B02A3605343E360012385F8203AA7
:103B8000E468B4B14FF0000BE40AA3450CDA0BEB88
:103B9000040A4FEA6A0A102239464FEACA200EF098
:103BA000DDFD0F2800F31F810EF07CFD9A4BE4022F
:103BB0001C609A4B9A789A4B02B101221A70039BAF
:103BC00098481B78984F052B02BF4FF4C872974B4B
:103BD0001A800CF00BFE964A00211378A5F8221AE1
:103BE00043F0080313700323924A85F8213A1370B7
:103BF000914B924A198059803B791170012BA5F89D
:103C0000241A0AD130228E4816F07FF94CF2503235
:103C10004FF07E518B480EF0C1FB00218A4B85F896
:103C2000581A1960596099607B79012B09D11022CB
:103C3000864816F06AF94CF25032854985480EF0F4
:103C4000ADFB854B854A1B684FF0010AC8F8003070
:103C5000834B00211B6883489B1A18BF0123824AAB
:103C600085F898AA13703C2216F04FF900237F4C78
:103C70007F4A2046C5F89C3A136004F035FBD9F81A
:103C80000030D90709D57B4B51461B685046642B41
:103C900038BF6423636404F05FFBD9F800309A07EF
:103CA00009D50121022004F057FB734B1B6B642BD9
:103CB00038BF6423A367D9F800100320C1F3400183
:103CC00004F04AFB0121052004F046FB6B4B97F8FA
:103CD00004A01A8D6A4B072093FBF2F3642B38BFC4
:103CE00064231AF10001C4F8143118BF012104F053
:103CF00033FB97F80590082019F1000118BF012146
:103D000004F02AFB3B7A002B40F047817B7A002BA2
:103D100040F04381D8F80010C1F38041BAF1000FA0
:103D200003D1B9F1000F00D14946092004F014FB7A
:103D30000121042004F010FB95F8E419062004F09A
:103D40000BFB01210A2004F007FBD8F800100B2020
:103D5000C1F3802104F000FBD8F800104B0507D513
:103D6000337A083B012B9CBF4FF4FA63C4F84C3202
:103D70000C20C1F3004104F0EFFA4FF4804011F041
:103D8000E1FF68B10022032390F902004FF4804163
:103D9000009301924FF4E13304F068FBC5F8A00AE8
:103DA000D5F8A03A63B10121022385F8A41A85F859
:103DB000A51A85F8A61A0D2085F8A73A04F0CCFAC2
:103DC00095F8C43463F07F0385F8C43421B0BDE8AE
:103DD000F08F202323804FF48073C7E64023F9E758
:103DE0004FF40073F6E7002357F8232001320DD17A
:103DF0000133042BF8D15446C7E6022101200FF00D
:103E00001DF8012012F0A8F8FEF7CCBF0AF1010B53
:103E1000A246F0E71740EF009C4100208C410020B3
:103E200090170020503B0020521B00204825002006
:103E3000C41600204D1B0020681700207C200020A5
:103E400090100020941000206C170020C410002057
:103E5000CDCCCC3ED4100020A82200200FAE00080C
:103E60003C3A00201C2000203A3A00203800002074
:103E700018200020FC3F0020F81600200E400020F3
:103E800040420F000022464B00B21A7012F062FE50
:103E9000444912F0B3FE0746B4F99C0612F05AFEEC
:103EA000404912F0ABFE0646B4F9A00612F052FEED
:103EB0003C4912F0A3FE3C490546384612F096FDF7
:103EC0000EF042F9814638460EF03EF93649074673
:103ED000304612F08BFD0EF037F9804630460EF07A
:103EE00033F931490646284612F080FD0EF02CF9D0
:103EF000834628460EF028F949468246584612F075
:103F00007DFE49460390504612F078FE59460490D3
:103F1000384612F073FE51460590384612F06EFE98
:103F200041460690584612F069FE204D51462860E1
:103F300008F1004012F062FE05996860AE603046FC
:103F400012F05CFE049912F051FD0699E8603046CB
:103F500012F054FE0146039812F046FD41462861D6
:103F600007F1004012F04AFE03996861304612F0F2
:103F700045FE0146069812F037FD0499A8613046C7
:103F800012F03CFE059912F031FD4946E8614046C9
:103F900012F034FE2862FEF73BBE0121BEE600BFF0
:103FA000F403002035FA8E3CDB0FC93F7C3800203B
:103FB0002DE9F04F7A4F9DB03B780690012B07D149
:103FC0007849794A0968C969118078490988518016
:103FD000774C2278002A00F04D83072B40F0D580E3
:103FE0000EF06AFD0790734B1A68984612F4806FC2
:103FF00005D07148836813B100F1440198476F4BB5
:104000006F4D1A780593B2B16E4BB3F906206B8BE6
:104010009A4210DC6C4B1B78012B01D0192B02D17A
:104020006A4A927B3AB90E2B05D0082B1FBF00239A
:10403000674AE3609360A67C002E33D0654B1B88F3
:104040009B072FD0644B6549D3F82090484612F067
:104050007DFF002840F09C80484613F003FD616915
:1040600012F0CCFD13F086FCB0F5617FA8BF4FF4D1
:10407000617012F06FFD5A4912F0C0FD0EF064F845
:104080008146304612F066FD494612F0B7FD13F046
:1040900071FC00B212F05EFD4D4E0146F06812F068
:1040A000A5FCF060EB7F94F818900493B9F1000F31
:1040B0005ED04C4B0420D3F8EC6044F620639E4263
:1040C000A8BF1E46B6F57A7FB8BF4FF47A76B6B26F
:1040D00066830DF067F918B9D8F80030DD0047D5D0
:1040E0004FF47A73B6FBF3F6642393FBF6F6142EC3
:1040F000A8BF14263C4DD8F800303548E1692A683D
:1041000013F4805FD0F80CA014BFB2F83680B2F977
:10411000368001F10102E261504604EB410B18BF09
:104120004FEA5808089212F045FF089AABF82000B1
:10413000B242A4BF0022E261E26904EB4202B2F99A
:10414000200012F007FD0146504612F04DFC12F01F
:1041500031FF00B20028B8BF404240451ADD2B684D
:10416000188F12F0F7FC214912F048FD059B5860AA
:10417000134A937F002B00F05D81022B3AD0032B72
:1041800000F02B811A4B588838E0002307932AE768
:1041900000207EE74FF07E53059A5360E8E700BFAA
:1041A00030190020542400203C17002080200020DB
:1041B00040110020601B0020A83A002000000020D1
:1041C00034190020EC1E0020311900202635002073
:1041D000341B0020141F0020D83200208FC2753CF1
:1041E000D06D393A380000202C1900206F12833A24
:1041F000FC370020608B00F57A7080B2049D023598
:10420000EDB2B9F1000F00F0FD80002800F0FA8057
:104210008C4B00261B68DFF86C82B0FBF3F000B219
:10422000A4F8480012F096FC01464FF07E5012F0C0
:1042300099FD8146DFF810A208F1100BAE42C0F2E2
:10424000D4803B78092B11D17F4B804E186813F036
:1042500091FB7F4B3080D3F8EC004FF47A7390FBE6
:10426000F3F012F077FC12F0A5FE7080B4F948303C
:10427000002B40F3E1804FF000084646DFF808923B
:10428000DFF8C4B1A9F1100AA845C0F2C180237EAD
:104290000025002B18BF02266E4BDFF8F091D3F8F3
:1042A00000803B78089308F105030993B54240F379
:1042B000EF80089B684D092B07D1644EB5F8483054
:1042C0006868B38012F076FEF080644B93F821604A
:1042D000002E60D01E200DF065F800285BD0604BEA
:1042E0001B88580657D495F88430B34214D085F80B
:1042F0008460304612F02EFC5A4912F07FFC5A4975
:10430000064612F073FB0DF01FFF584B98603046C5
:104310000DF01AFFC5F88800059B6668D3F8089071
:104320003046494612F06AFCD4F80C80D4F8887004
:1043300082463946404612F061FC0146504612F072
:1043400053FB4B49824612F001FE08B9DFF820A169
:104350004849504612F004FE08B9DFF818A1494652
:104360004046C4F804A012F049FC39468046304665
:1043700012F044FC0146404612F038FB3C49064628
:1043800012F0E4FD00B93A4E3A49304612F0E8FD29
:1043900000B9384EE66000232B76374B1B78002B94
:1043A00040F05B81354DAA78002A00F05681344CEC
:1043B0002378013B0D2B00F23D81DFE813F00F0164
:1043C00022012C0121023B013B013B024F026C0503
:1043D00089059A05B905C405CD0592F82000C0EB02
:1043E000401300EB8300C00007E75BF826105AF883
:1043F000260012F0F9FA494612F000FC48F82600AF
:1044000001361BE7B4F84830013BA4F848302DE7EB
:10441000464659F828005AF8281012F0E7FA022EFA
:10442000B8BF022649F828004BF82800F6B208F178
:10443000010829E7A4F84830237E002BADD00026E0
:1044400025E700BF14190020341B00203C17002072
:104450003800002038390020401100203419002095
:10446000141F002035FA8E3CDB0FC93F00000020EE
:1044700000C0F94400C0F9C4942C00208C410020F5
:10448000901700208C1100209C1100200AD7233C9B
:10449000022D15BF98F8000098F8010098F802B0B6
:1044A00098F809B012F056FB494612F0A7FB4FF0FE
:1044B0008041074612F05EFD60B14FF08041384602
:1044C00012F092FAAA4912F099FB0146384612F00E
:1044D0008DFA0746AB000493A64BA74953F8250075
:1044E00012F08CFB20F00043A44A0493049B42F892
:1044F00025000C32824642F82530BBF1000F20D057
:10450000584612F027FB494612F078FB8346514685
:10451000504612F073FB049912F070FB594612F0EA
:104520006DFB59460A904FF07E5012F05DFA0A9AE0
:104530000146104612F05AFA0146504612F05EFB50
:1045400082468F49384612F059FB514612F056FB0D
:10455000099B074613F8010B099300B312F0FAFA0E
:10456000494612F04BFB049912F048FB85498246FC
:1045700012F000FD68BB0021504612F0DDFC50BB7C
:1045800051464FF07E5012F02FFA01464FF07E5008
:1045900012F0E8FB0146384612F030FB0746089B54
:1045A0000C2B05D1384612F005FD774B23F815008A
:1045B0007649384612F0CAFC00B9744F744938463F
:1045C00012F0CEFC00B9724F724BAA00D7500135E1
:1045D0006CE64946DAE74FF07E51D7E76E4B1B7821
:1045E000D90707D5802010F0F7FA08B103F026FFAD
:1045F00012F08AFD1F200CF0D5FED8B10C232370D9
:1046000018E00022654B1A60654B1A60654A126813
:104610005A600323F3E711F0CDF9614E614B1A683C
:1046200073686433934205D2402011F09DF900284D
:1046300000F0C28011F0DEF90646002800F09384F5
:1046400023780C3B022B08D901232370564B93F897
:10465000D92012B1002283F8D920544B1B78072BA4
:1046600005D10EF029FA079BC01A474B988000220B
:104670004D4B1A704D4F3B78072B40F0CE840EF017
:104680001BFA07904A4C636820469847A2460028C8
:1046900055D00026B4F8A85084F84960DFF814918A
:1046A000002D40F00185E26AB4F9243094F84A10F4
:1046B0009B1AA363226BB4F9263004F138009B1ACD
:1046C000E363626BB4F9283004F134089B1A236465
:1046D0000CF09CF84C46DFF8B0900AF5707658F86C
:1046E000040F12F037FADAF8201012F087FA3B784C
:1046F0008346082B03D113F03DF929F815005946DC
:10470000DAF8BC3330469847DAF84434014606F10B
:10471000880098473B788346032B03D113F02AF98E
:1047200029F81500DAF8AC305946D8F878039847DC
:104730000135032D44F8040F06F12C06CFD11B4C94
:104740002278072A05D10EF0B7F9079BC01A0E4B45
:104750001880154B93F8E1201D460592002A00F0C1
:104760007185013A83F8E1201DB0BDE8F08F00BFEC
:10477000D7A36841341B00206F12033BAC1100200B
:1047800000004843A4707D3F3C17002000C0F9445E
:1047900000C0F9C444110020301B002088410020D3
:1047A000081900204C3A0020401100203019002048
:1047B000A83A0020FC3F0020DFF864834027C2466F
:1047C000DFF86093336818F8030068B111F088F9D6
:1047D000D9F80030013F03F1FF33C9F800303368E6
:1047E00003F101033360EDD133681AF80330002B75
:1047F0007FF420AF33604FF0FF3373600423FEE695
:1048000011F0D8F8934A5021A2F10C03019325230B
:10481000029200934920A2F10A03163A04F04CFCDC
:1048200000287FF407AF4FF0FF328B4B18605A60BF
:104830000723E4E611F0BEF8052300210093874B1F
:1048400002910191A3F10802532004F035FC0028E5
:104850007FF4F0AE804B18600823D0E611F0AAF880
:104860007F4B804E186813F085F88046D6F88C0090
:1048700013F080F88146402011F076F83146002888
:104880007FF4D8AE744E784F33687878492B01F2B4
:104890008F85DFE813F04A0050005E006500690074
:1048A0006E00730078007D008400890095009F00F1
:1048B000A400AF00B400B900BE00C600CE00D60010
:1048C0004901510159016101690176017F018801A6
:1048D00091019A01A301AC01B501BE01C401CD0152
:1048E000D301D901DF01E501EB01F201F901000279
:1048F00006020C0213021A02200226022C023202C5
:1049000037023C02410246024B025102AD02BA029A
:10491000BF02C402C902CE02D302D902DE02E30200
:10492000E802ED02F202F702FB02504A50495148F8
:1049300011F0A9F909E0504B4C4A01934F4B5049F3
:1049400000935048504B11F09EF9336801333360A7
:1049500070E64E4B4E4A4F494F4811F094F9F4E738
:104960004E4A43494E48E3E76B782A784D494E4812
:10497000F3E74E4B4E491A8A4E48D9E74B4B4C4908
:104980005A8A4D48D4E74FF07E524C494C48CFE705
:104990001FFA89F31FFA88F24A494B48DDE74B4B6F
:1049A0004B491A8A4B48C3E74B4B1B68DA0404D5C2
:1049B00091F8902049484649BAE70C233360C4E790
:1049C000474948488B784A7809780091464911F060
:1049D0005AF9BAE7454B3E491A884548A8E7404B83
:1049E0005B79012BB1D1B1F99430B1F996204148EE
:1049F0003449B2E7404B2E491A68404898E7404B8B
:104A00002B499A783F4893E73F4B29491A783F480A
:104A10008EE70C2303FB00113D4891F898202449B0
:104A200086E70C2303FB00113A4891F89A202049AD
:104A30007EE70C2303FB0011374891F899201C49AD
:104A400076E70C2303FB0011344891F8A1201849A4
:104A50006EE700BFDEA10108081900208CA3010841
:104A6000B017002040110020582000205FBE010830
:104A700085CB01086BBE01083BBE010855BE01088D
:104A80007FBE01088DBE010879BE01084CBE010839
:104A900040BE01088ECD01089FBE01085C200020A9
:104AA000ADBE0108B8BE0108BEBE010898170020BF
:104AB0002AD90108C9BE0108D5BE010819C50108D7
:104AC000E1BE0108B8BF0108ECBE0108F8160020DD
:104AD0007DCD0108F8BE010894170020FFBE010833
:104AE000521B002013BF01080ABF0108AE170020A7
:104AF00023BF01082BBF0108FC3F002039BF01087C
:104B0000963A002042BF0108BC32002052BF010883
:104B100064BF01086CBF010874BF010880BF0108B1
:104B200068A10108884100200C2303FB001185487F
:104B300091F89B208449FBE60C2303FB001183487A
:104B400091F89C208049F3E60C2303FB0011804878
:104B500091F8A0207C49EBE60C2303FB00117D4873
:104B6000B1F8A2207849E3E60C2303FB001191F889
:104B70009E3091F89D2091F89F10774800917749D9
:104B800025E7774B774819684B780A788978009140
:104B900072491CE7724B744819680B79CA784979D5
:104BA00000916E4913E76E4B70481968CB798A798A
:104BB000097A009169490AE7694B6D4819688B7A4F
:104BC0004A7AC97A0091654901E7654B69481968D5
:104BD0004B7B0A7B897B00916049F8E6604B664815
:104BE00019680B7CCA7B497C00915C49EFE65C4B01
:104BF00062481968CB7C8A7C097D00915749E6E6BA
:104C0000574B5F4819688B7D4A7DC97D0091534998
:104C1000DDE6534B4C491B685A481A7E88E6504BD8
:104C2000594819680B7FCA7E497F00914B49CEE6EF
:104C30004B4B45491B6855489A7F79E6484B42499A
:104C40001B6853481A8C73E6454B3F491B68514813
:104C50005A8C6DE6424B3C491B684F489A8C67E67C
:104C60003F4B39491B684D48DA8C61E63C4B36496D
:104C70001B684B4893F828205AE6394B32491B6889
:104C8000484893F82F2053E6354B2F491B68464878
:104C900093F830204CE6324B2B491B684348DA8EA0
:104CA00046E62F4B28491B6841481A8F40E62C4B9B
:104CB00025491B683F4893F83A2039E6284B22499A
:104CC0001B683D4893F83B2032E6254B1E491B6884
:104CD0003A489A8F2CE6224B1B491B683848DA8FDA
:104CE00026E61F4B18491B6836485A8D20E61C4B98
:104CF00015491B6834489A8D1AE691F8BC20334850
:104D0000114915E691F8BD2031480F4910E6314BA5
:104D10000D49DA7830480BE62E4B0B491A792F48AB
:104D200006E62C4B08495A792D4801E6294A2D49B7
:104D3000D3892D48528910E6264A2A49138A2B48DE
:104D400092890AE68CBF01082AD9010894BF01089C
:104D50009DBF0108A6BF0108BEBF0108B5BF01087D
:104D60002C190020C4BF0108CCBF0108D5BF010821
:104D7000DCBF0108E3BF0108EABF0108F2BF010878
:104D8000FABF010803C00108FCBF01080AC00108FE
:104D90001CC0010829C0010834C0010843C0010833
:104DA00056C0010863C0010871C0010882C0010833
:104DB00099C00108ABC00108C5C00108DBC00108EB
:104DC000E9C00108F3C0010800C101086DD601085F
:104DD00011C10108963A00201EC1010827C101082F
:104DE00039C10108B8BF010849C1010857C101080C
:104DF0008C4B188811F0AEFE8B4911F0FFFE12F0BB
:104E0000D9F88A4902468A4892E5864B8749DA787A
:104E100088488DE591F8C2208748844988E591F853
:104E2000CD208648814983E591F8D62084487F4982
:104E30007EE5844B7D499A7F834879E5814B7B49A8
:104E400093F82020814873E57E4B78499A8C8048FE
:104E50006EE57C4B75491A7A7E4869E57E4B73494D
:104E60001A797E4864E57C4B70499A787C485FE506
:104E7000794B6E491A887B485AE5774B6B49DA893A
:104E8000794855E5BA786949784851E5784B6749DA
:104E90001A6878484CE51A200CF084FAA0B1764BD9
:104EA0001B888BB9754B14A91B680E201493069BA5
:104EB000159303F071FE4FF48052714B1A800A2350
:104EC0002370069803F0B6FE03F048FEFFF7B2BB6E
:104ED0006C4B1B78002BF4D01A200CF063FA0028DE
:104EE000EFD1694B93F8D930002BEAD10923237015
:104EF000EAE7664B1A68664B5B68C833934211D287
:104F0000AB78032B0BD1634E306803F082FA002399
:104F10003360614B1B78022B01D103F0F5FC0123B8
:104F2000FFF76DBB12F088FB0028E9D1FFF782BBC9
:104F3000012A01D10DF0F4FB0D231320237010F092
:104F400039FFFFF777BB012A04D10DF0CDFA002815
:104F50003FF470AB0E23F0E71F200CF023FA00287B
:104F60007FF468ABDBE7EB78002B3FF476AB0027F0
:104F70004FF0010AB946494B1B68DB044BBF484B55
:104F8000354BB3F804B0B3F814B0584611F0E2FD55
:104F9000444B014653F82700D04611F0C3FF00B13F
:104FA000C846013746EA0806082FF6B2EDD1374B5E
:104FB000354F1B68BEB103F59C530833C7F8DC308E
:104FC0002378012B7FF449AB97F8D930002B7FF47D
:104FD00044ABAB78032B19D012F096F8012387F875
:104FE000D930FFF73ABBD7F8DC209A42E8D82378CB
:104FF000012B3FF432AB97F8D930002B3FF42DABA7
:1050000004F012F987F8D960FFF727BB80200FF072
:10501000E3FD00287FF421ABDEE700230793FFF7D1
:1050200031BB00BF203900200000C8422AD9010846
:1050300069C1010874C1010881C101088FC101085B
:105040009CC1010834190020B2C10108C3C1010884
:10505000DDC10108F7C101089817002009C2010845
:105060001AC201082DC201083CC201084DC2010844
:10507000A822002058C201088C17002088170020A1
:10508000B016002064190020401100204C3A002086
:10509000081900209441002011190020601B0020F5
:1050A00030390020282B00205E4BD9F800205B7897
:1050B000059608934FF47A73B3FBF2F3C3EB4312F4
:1050C00003EB8203DB009BB204933B7804F12C07D3
:1050D0000993554BB3F90690049B5B080A93049B14
:1050E0009D4201BF00237B63E3673B604F4BF31896
:1050F000B3F924007B6B03447B6311F02BFDE26F5B
:1051000002F10108B8F1010FC4F87C8007D1002337
:10511000012D2067E06663675DD1002030E0D4F8A0
:105120006CA00C9251460B9011F05EFC83464046F9
:1051300011F010FD0146584611F014FE514611F0D1
:1051400055FC0B9B014682462067184611F04CFC2B
:10515000594611F053FD616F11F048FC012D834653
:10516000A067C4F86CA060670C9A34D1B8F1010F45
:10517000D3DD104611F0EEFC0146584611F0F2FD69
:1051800012F0B8FE099B8046032B05D112F0F2FB0A
:1051900001230FFA80F90593089BABB1184611F073
:1051A000D9FC414611F0C8FE70B1059B13B11E4BEE
:1051B000A3F806901E480BF019FB00221D4B5A6005
:1051C0009A60DA60FFF7BBBA0A9A7B6B1344049AC1
:1051D00093FBF2F33B600236062E07F1040704F15D
:1051E00014047FF47CAF059B13B10F4BA3F806901A
:1051F000012D0FD10022104B1B689A621A63DA62EC
:105200000E4B93F8E03013B10D4B1B8813B90120FE
:1052100010F0D0FD054AB2F8A830013BA2F8A83042
:10522000CBE700BF963A00203C170020A83A0020A8
:10523000503B0020FC3F002054240020401100205F
:10524000881B0020AD4B5B79002B00F03384AC4B06
:105250001B78013BDBB285F8E1302378072B40F067
:105260002C840DF029FC0B90A64B4FF07E501B6850
:105270000793D5F8E4300D93D5F8E83019460A9332
:1052800011F0B2FBA04B196811F0B8FC4FF07E5141
:105290000C9011F05BFE10B94FF07E530C939B4BBA
:1052A000002509939A4B9B4C089300230493049B7D
:1052B000DFF8B0929E0059F82370049A964B294665
:1052C00053F82280404611F02DFEE8B9049B09F105
:1052D000E80959F823903846494611F085FB824683
:1052E00020F00041404611F027FE58B129465046B3
:1052F00011F040FE002800F0E4834946404611F0DA
:1053000075FB0746854BF750854BB3F800A01AF0A4
:10531000030F3DD0049B022B3AD0079B93F8320039
:1053200011F018FC7F4BF15811F068FC079B814687
:1053300093F831B0CBF1000011F00CFC804601462F
:10534000484611F0F9FD40B9584611F0FFFB4946B7
:10535000804611F0FBFD00B9C846049A724B33F940
:105360001200089BB3F90030C01A11F0F3FB6F492B
:1053700011F044FC0146404611F036FB1AF0010FD3
:105380000E9000F0CF836A4B196811F037FC074686
:1053900094F8F830002B57D0049B022B54D0089B74
:1053A000DFF88481B3F90000049B38F91330C01A88
:1053B00011F0D0FB5E4B07465C49186811F01EFCEB
:1053C0000146384611F01AFC069AD4F8FC3007461C
:1053D000D31A584A1268934231DC4FF07E510A9832
:1053E00011F0AAFD80B3544B54491A68B1F90A0070
:1053F000B8F900301B1A002BB8BF5B42934223DA86
:10540000B8F90230B1F90C105B1A002BB8BF5B423F
:105410009A4219DD4A4BDFF82C91D3F80080D9F875
:105420000400414620F0004011F086FD60B1D9F83B
:105430000810404621F0004111F09CFD20B10020F1
:1054400084F8F8000DF090FC3E4B38463344D3F816
:1054500004A0DFF81491514611F0C6FA80463A4B89
:105460000D98F15811F0CAFB414611F0C7FB049B9F
:105470000146022B46F8090006D1344A344B106825
:105480001B689847C9F80800099B53F8049F0993C3
:10549000304B5968304B186811F0B0FB0C9911F083
:1054A000ADFB2E4BF15811F0A9FB414611F0A6FBC4
:1054B000494611F09BFA049B8346022B40F001847D
:1054C00094F80031012B02D0192B40F0FA834FF0F1
:1054D0000103234940460E9311F04CFD0E9B00B989
:1054E0000346DBB2002B41D02BF0004029F00041F5
:1054F00011F022FD00283CD038E000BF963A002091
:10550000BC3200202C190020A42F0020DC16002023
:105510002A39002040110020982F00202C12002052
:10552000141F0020AC11002018330020CDCCCC3D3E
:105530007C2F0020A82F0020AC2F00202039002035
:10554000B02F0020FC3F0020502F0020A832002068
:10555000A432002000000020942F00205C2F0020A7
:105560000000964244110020D4160020099BC3F885
:1055700000B0049B022B6DD0A24AA34B51461B687E
:10558000B0589847A14AA24B01461B68B0589847AB
:10559000079B814693F83A30632B00F29C839D4B26
:1055A0001B88002B40F097839B4BF1589B4B18684E
:1055B00011F024FB4FF07E51824611F0C7FC08B970
:1055C0004FF07E5A964B5046196811F017FB014672
:1055D000384611F013FB494611F006FA914B81460B
:1055E000F15811F001FA904B196811F0BBFB8D4B8B
:1055F000074646F80390079B93F84890B9F1000FCF
:105600001ED04FF07E510A9811F0AAFCC0B1874B12
:1056100027F00040196811F0ADFC88B1844B28F0E8
:105620000040196811F0A6FC50B10120069BB9F1A9
:10563000020F84F8F800C4F8FC3001D10DF094FB9F
:105640007C4B0D98F15811F0D9FA394611F0D6FA81
:10565000794B985194F80C312BB9784BF550099B44
:105660001D60754BF550049B01330493089B023376
:105670000893049B032B7FF41AAE714E3278072AED
:1056800005D10DF019FA0B9BC01A6E4B5880337878
:10569000012B40F022830DF00FFA6B49D4F8103142
:1056A000684A0968C31A93805B1A0690D380C4F8CD
:1056B0001001664B664E1B6893F82F80654B1B6884
:1056C00013F4805F644B00F05583644AB3F818907C
:1056D0001278F668D70758BF1A8B614B58BFA4F8E9
:1056E0001421DF88A9EB070B584611F033FA8246E4
:1056F0000146304611F02AFC002800F0F782D4F869
:105700001C31C4F81831574B1B68C4F82031D4F849
:105710002411D4F82C0111F025FB4FF07E510446E2
:1057200011F014FC08B94FF07E540021204611F00E
:1057300017FC00B900244C4DD5F81831C5F82C41A0
:105740000793D5F8203107981946089311F04CF9C2
:10575000464BC5F838011968384B0B90186811F0A2
:1057600045F9354B196811F041F941490D9011F097
:1057700045FA404B82461D6805F10046314611F05E
:10578000DBFB002840F00A832946504611F0DEFB7F
:1057900000B9AA46354B5968284B586811F026F9CC
:1057A000254B596811F022F931490E9011F026FA73
:1057B00007460146304611F0DDFB30B93946284630
:1057C0002E4611F0C3FB00B93E46284B99681B4B8F
:1057D000986811F00BF926490F9011F00FFA264B3B
:1057E00081461D6805F10047394611F0A5FB0028E8
:1057F00044D1294648464F4611F0A8FB00283DD128
:105800002F463BE0C02F0020BC2F0020243000207A
:1058100020300020141F0020B8110020782F002015
:10582000742F002044120020942F0020B82F002055
:10583000B42F0020682F0020EC160020D416002082
:10584000301900203C170020141900202C190020CA
:10585000341B0020601B002034190020301B002066
:1058600030390020B017002040110020E016002041
:105870006F12833AC0320020C4320020B8F1000F0A
:1058800025D0924B1A7912B3914A1578FDB1187848
:1058900011F05CF98046284611F05CF9014640465B
:1058A00011F0ACF98B4B0546188811F04FF9014601
:1058B000284611F057FA8849054611F047FB00B910
:1058C000854D4FF07E51284611F04AFB08B94FF044
:1058D0007E55824B4FF000095B78002B804B14BF44
:1058E00001204FF0FF3093F800B011F033F9394642
:1058F00011F084F900237B4F0C900A930993D9454A
:10590000C0F266820A99099811F06EF8764D4FF050
:105910007E51C5F8E800064611F02CFB002800F087
:10592000988231464FF07E5011F01CFA0024074651
:1059300014AEA34500F384820BF03AFD18B14FF08A
:105940007C53C5F82C31DFF8A0A10025DAF82C3102
:1059500009939AF8BC310A93644BDB781093644B3B
:10596000D3F80080404611F025FB8146614B1E684C
:1059700006F010031193604B06F480561C785F4BC1
:1059800004F00104B3F906705D4B5A8B12930AF5CB
:105990009E730C9213935D45C0F0808224B9594BDD
:1059A000594AA34500F3C2824F4BD3F8C021002AC5
:1059B00000F08E8493F80031192B09D801229A4007
:1059C000524B1340002B40F0B782100300F1F883D4
:1059D000484E4F4D336813F0200F30D0002008F0B0
:1059E000EDFD4C4C80462080012008F0E7FD074685
:1059F000608008200BF0D6FC08B33B4B95F90A10E9
:105A000093F8E431012B444B40F0E583484295F98B
:105A10001620B3F90210B3F900304143534332204A
:105A20006FF0310291FBF0F193FBF2F293FBF0F097
:105A30000A44A8EB02022280084438446080002314
:105A4000364AEC18B4F90410B2F90200B4F9064071
:105A5000884203DB84422146A8BF01460C33602BF9
:105A600022F8021FEDD12E4DAB89002B40F0C383ED
:105A70001D4F97F80031013B182B00F2F283DFE84D
:105A800013F0E203F003F0035404F003F003F00317
:105A90004104F003F003F003F003F0036004F003AB
:105AA000F003F003F003840454047104F003F003E2
:105AB0006004E2030123FFF7CEBB00230B93FFF743
:105AC000D3BB4146484610F08FFF1AE4521B00201A
:105AD0007C20002068170020713DAA3F311900206A
:105AE000441700207C12002040110020641B00207D
:105AF000982C0020601B0020301B0020EC1E002092
:105B00003419002048170020282B00203241300390
:105B1000F02E002078170020183300207617002080
:105B200026350020D4F87890D4F87C804946404649
:105B300011F002FA00287DD049464FF07E5010F057
:105B400053FF974B8146B3F90000B3F9023080EA66
:105B5000E07183EAE372A1EBE071A2EBE3729142A0
:105B60006ADD0028D8BF404210F0F4FF8D4911F0E3
:105B700045F88D4B80461B78002B62D08B4B294615
:105B8000D3F800B0584611F0F5F9002800F09780DE
:105B9000874B2946D3F800A0504611F0EBF90028B6
:105BA00000F08D804FF07E51484610F01DFF814976
:105BB00011F024F8594611F0D5F84FF07E5110F04D
:105BC00015FF41468146504610F00EFF514611F038
:105BD000C9F84FF07E51804611F0B8F908B94FF07E
:105BE0007E582946404611F0BBF900B9A8464946FF
:105BF000404611F003F881466F4B0E98196810F07B
:105C0000FDFF4FF07E518046484611F09FF908B9DC
:105C10004FF07E592946484611F0A2F900B9A9462D
:105C20004946404610F0EAFF0146384610F0DEFED5
:105C3000FFF7ADBB414680E7002BCCBF184658426A
:105C400092E75E4B5E49D3F800A0504611F074F91C
:105C5000002830D051464FF07E5010F0C5FE594913
:105C600010F0CCFF41468346574810F0BDFE014678
:105C7000584610F0C3FF514610F0B8FE4B4B196860
:105C800010F0BCFF80462946404611F05FF9B0B9DC
:105C90004FF07E51484610F0A7FE414681464548E8
:105CA00011F060F80146484610F0A8FF4FF07E5111
:105CB00010F09CFE9FE73D4BD3F80080E3E7A94638
:105CC0009AE74FF001034FF07E51D4F8E8000E93AD
:105CD00011F046F902E429467AE4072B03D10CF0CF
:105CE000EBFE0690E5E400230693E2E409EB0700EF
:105CF00010F030FF0146304611F032F900B3D4F80D
:105D00008C303046C4F81831D4F82831C4F820312A
:105D100011F076F9A4F81401484610F01BFF014673
:105D2000304610F061FE0546384610F013FF01467C
:105D3000284610F059FEC4F82C01D4F83011E8E4DC
:105D4000B4F814319B450ADBD4F81C31C4F82CA1FB
:105D5000C4F818311D4B1B68C4F82031D7E4D4F8BF
:105D60008C30C4F82C51C4F81831D4F82831C4F858
:105D70002031E2E7588B10F0EDFE0146F06810F09C
:105D800033FE124BC4F82C011B68D4F83411C4F84C
:105D90002031D4F88C30C4F81831BAE4B246F9E4B2
:105DA00018330020CDCCCC3D882F0020842F00203C
:105DB0008C2F00200000C842802F0020902F002050
:105DC000AE47813F610BB63B00003443B017002063
:105DD0007968504610F012FFB9688046304610F0DE
:105DE0000DFF0146404610F001FEF96880460C9810
:105DF00010F004FF0146404610F0F8FD4FF07E51D0
:105E00008046284611F0B6F820B14046294610F0E9
:105E1000F5FE80464146099811F08EF868B9414672
:105E20000A9811F093F808B9CDF8288014AB43F81C
:105E30002980103709F1010961E5CDF82480F5E7E3
:105E400056F82400394610F0D9FE46F824000134F3
:105E50006FE50BF0ADFA38B94FF07C51204611F0E8
:105E600089F800283FF46FAD4FF07C51304610F0B8
:105E7000C5FE05460146204611F05EF850B9294698
:105E80004FF07E5010F0B0FD2146054611F05EF84F
:105E900000B92546BB4BC3F82C5154E5139A2B018E
:105EA0009958099810F0AAFE14AB53F8251010F079
:105EB0009DFD0B9910F0A2FE089910F097FD0A9B2A
:105EC00082463BB10899079810F090FD514610F0BA
:105ED0008BFD8246109B5046FBB111F06BF8484594
:105EE000824606DB079811F065F85045A8BF50467A
:105EF00000E0484610F02EFE119B824643B13CB1B3
:105F000036B90BF055FA18B90C9B9F42B8BFC24680
:105F10009D4B43F825A001353DE511F04BF8824635
:105F2000089811F047F88245E4DBDBE752F82410CB
:105F300043F82410013434E5944B1B88D90540F113
:105F40008C80934C206811F035F8ADF850006068F3
:105F500011F030F8ADF85200A06811F02BF8ADF850
:105F600054004FF47A724FF461618A48B0F90230FC
:105F700003F5E163534393FBF1F3A3F5FA73ADF833
:105F80006830B0F9003003F5E1635A4392FBF1F257
:105F90007D4BA2F5FA7280491868ADF86A2010F0BE
:105FA00023FD11F007F87D4A129B11881B8BADF879
:105FB0005600C91AADF858105188C91AADF85A10D0
:105FC0009188C91AADF85C10D188C91AADF85E1075
:105FD0001189C91AADF860105189C91AADF862105B
:105FE0009189D289C91AD31AADF866300023ADF869
:105FF000641019466A4A22F813100133082BFAD1AB
:106000004FF00C096427674B674C1B78674DC3EB57
:10601000C3032344DFF8A481DFF884A10993099B1B
:10602000A3423DD100254FF00C096427604EDFF8F4
:106030008C8109FB0583B6F9024093F90A004443B9
:1060400094FBF7F4E8B2748008F0B8FA0135204404
:10605000082D26F8020FECD1BAE456490D9810F03D
:10606000CDFD10F0A7FF5349ADF850000E9810F089
:10607000C5FD10F09FFF4F49ADF852000F9810F08A
:10608000BDFD10F097FF00B2ADF85400002E3FF4B4
:1060900068AF494B1B8B9F42BFF663AF40425EE740
:1060A000A07928B11630C0B20BF07CF9002867D077
:1060B00094F800E094F9051009FB0E83DA889B88B8
:1060C00094F801C0D21A94F9043092B2534393FB6E
:1060D000F7F34FEA520BA3EB0B030891E1781BB2E5
:1060E00007934FEA4C0681BB1CA90E4436F8201CCE
:1060F0002980012309FB0EF158F8011003FA0CFC6A
:106100001CEA010FB5F9006094F9021008BF1846A7
:1061100001FB06F191FBF7F1079B18BF4FF0FF3031
:10612000994209DB089B5A4392FBF7F2A2EB0B035F
:106130001BB28B42A8BF0B463AF81E2000FB03237C
:106140002AF81E300235073469E71CAB1E44B5F946
:10615000000036F9206CB04208DA0144884203DCC2
:106160008E423046A8BF08462880C2E7C1DD411AEA
:10617000B14203DB8842A8BF084606462E80B8E736
:106180002880DFE74011002048170020141F00205E
:10619000341B0020183300200080BB44EC1E00207C
:1061A000781700200C2E00200D2E00200413002054
:1061B000761700203333333F34190020F02E0020AF
:1061C000814A824830F8131022F813100133082B4B
:1061D000F8D1FFF7FDBBB3F90220B3F900004A4341
:1061E000322192FBF1F24244228095F9162050436D
:1061F00090FBF1F021E4DFF8D0810024C346744F16
:10620000DFF8E89138F9140010F0A4FC01462C20C6
:1062100000FB04900BF024FE11F0ACFBB7F9043046
:1062200000B298424FEA440AB7F9062003DB8242E3
:106230001346A8BF03460134082C2BF80A3007F197
:106240000C07DFD114E4AB7B002B54D05E4BB3F9C9
:106250000A0010F07FFC0146002005F0C3F901237D
:10626000059333689A0603D497F80031052B16D1AD
:10627000554CB4F9000010F06DFC0146059805F08E
:10628000C1F9B4F9020010F065FC059B0146013329
:10629000D8B205F0B7F9059B0233DBB2059333683A
:1062A000DB0215D50024EE7B484FE5B27319DBB253
:1062B000112B0DD8331937F9130010F04BFC059B47
:1062C00001461D44E8B2013405F09CF90E2CECD1D6
:1062D000404B1B78002B68D13F4B1B78072B05D117
:1062E0000CF0EAFB069BC01A3C4BD88001223C4BC9
:1062F0001A70FEF739BA3B4B187810F00100A5D19F
:106300000021AAE7304CB4F9060010F023FC014646
:10631000002005F067F9B4F9080010F01BFC0146F5
:10632000012005F05FF902239AE7274CB4F9080031
:1063300010F010FC0146002005F054F9B4F90A00F1
:10634000EBE70224DFF8808038F9140010F002FC3B
:10635000A31E01460134D8B205F054F9082CF3D13C
:1063600006237DE7184C049B34F9130010F0F2FB70
:10637000049B0146033BD8B205F044F9049B01336A
:10638000072B0493EFD104236AE70024DFF8388059
:1063900038F9140010F0DEFB0146E0B2013405F0DC
:1063A00031F9082CF4D105945BE708F013FB93E76F
:1063B00011F042F900283EF43DA94FF480520A4BF7
:1063C0001A800A23FEF71BB978170020EC1E002064
:1063D000F02E00203A3A0020301900203C1700200F
:1063E00040110020301B0020B01600202813002090
:1063F0002DE9F04FA84B00F59C4808F12008C3F8A0
:106400000080A64B87B01C780746002C69D0A44AB0
:106410001268904201D9013C1C70A24C2368DE0432
:1064200005D500200AF0BEFF08B904F07BFE9E4AA5
:10643000537D0092002B00F07E819C4A013B32F993
:106440001300994BDB7D1BB1C0F53B60083000B2F7
:10645000A0F57A70B0F57A7FA8BF4FF47A7020EA81
:10646000E07010F077FB924910F0C8FB10F0C8FD07
:10647000904B18802368DFF878B213F4807F00F027
:10648000D6818D4BDFF84CA29F4205D99AF80220A5
:1064900012B901228AF802209AF80220002A00F09C
:1064A000C6819AF821709BF800501B200AF07AFFF1
:1064B000012F05F0010908BF0025804EDFF8348266
:1064C000019018BF05F002059AF82020052A00F275
:1064D000AA81DFE812F06E01CF01DA01FB010802A8
:1064E00023020AF041FA0646754DDFF8BC91DFF849
:1064F000F0A1A64246DC42F201024FF47A71694BE8
:10650000B7FBF1F91B68134001936E4B06D06E4A3E
:1065100012781A706D4A11786D4A11701B780093C9
:1065200023B16B4B1E7886F0010300930F230024E8
:10653000DFF8C4B1DFF874A185F824300AF014FA4A
:10654000844249DB95F82430624C0F2B0CBF0122AA
:106550000022614B594D1A7040F0D0801B200AF088
:1065600021FF002840F0CA802B68E268A3609B1AD4
:10657000C82B02D9012384F82130584A13780133FB
:1065800013704AE7072CE1B25548D8BF14F8091038
:10659000DAF804309847032C1ADCC8B1514B33F8B1
:1065A000242003EB8401831A4FF47A7058434B88FC
:1065B0009B1A90FBF3F040F2EE2300F57A709842BC
:1065C000B8BF184640F6CA039842A8BF184680B222
:1065D00025F8140001348CE7009A6300D2B135F934
:1065E0001400314A80B2D18C81424FEA840103D831
:1065F000B2F828E0864520D23B4A515889450BD253
:106600003AF80300019AEAB92AF8030001340BF1C1
:10661000060B93E70098E4E7E0B202930AF0BCF9B6
:10662000032C029BEEDC012101FA04FE95F82410F4
:1066300021EA0E0185F82410E4E72B4E09F5967245
:106640007250DFE7254903EB040E91F800C00321E7
:10665000BCFBF1F101EB4101ACEB0101C9B27144AA
:1066600005EB4101C88495F86E1029B9BCF1020F01
:10667000CAD9012185F86E10BBF80010BBF80200E2
:106680000844BBF804100844184900B2C85203215A
:1066900090FBF1F080B2B7E708380020CC3800203A
:1066A000C8380020601B002034190020EC1E002098
:1066B000AAF1823F4A1B0020404B4C004C3A00207C
:1066C000D8140020311B0020D8370020E40300201C
:1066D000E5030020641B0020C516002000100020E8
:1066E000FC370020DE380020041000204815002070
:1066F000301B002044330020FE1400200123924A66
:106700001370924A13702B68A268E3609B1A626848
:106710008F4D934284BF002384F8213000240AF077
:1067200023F98442BFF629AFE0B20AF035F925F823
:1067300014000134F3E7226815047FF59BAE854A07
:10674000D2F88810791A0029FFF694AE8249C2F86F
:106750008880487C814931F81000009980B2897D99
:1067600090FBF1F092F88C10013101F00F0182F8EA
:106770008C10114481F88D0018468D32815C0130F7
:106780000B4410281BB2F9D193FBF0F31BB2002B82
:106790000ADB642BA8BF6423009AD27D32B918B2F9
:1067A00010F0D8F96E495FE60023F5E7C3F1640302
:1067B000F5E7B9F1000F2DD00AF008FE012807D146
:1067C00064203168B8F8062000FB0212CAF81020D5
:1067D000019B63B198F804204AB108F019FD032227
:1067E0008AF820204FF47A72CAF81C206CE6012F38
:1067F00019D03268DAF81010914207D208F008FD7B
:1068000003228AF8202040F6B832EDE701228AF808
:10681000202059E6019B4FF4806043B30FF08EFBBC
:106820000022CAF8102015B128460FF0C3FA0AF06A
:10683000CDFD06460AF0BCFD4A4D002800F09A80C6
:106840009BF80030D80740F19580009B988C10F0A1
:1068500081F9454B0146D86810F082FB002800F012
:10686000458201223B4B83F89D20012395E00FF0E8
:1068700055FBD5E7012F01D10522C8E798F808207C
:10688000012ABBD008F0C4FC1EE6012F04BF05227C
:106890008AF82020B9F1000F0AD00325009B2C4A6A
:1068A000B3F91810118051809180B8F80210D1808E
:1068B0003268DAF81410914202D3B9F1000F3FD1D7
:1068C00047F23052CAF81C200322A0E702200FF042
:1068D00043FB04F027FC3168DAF81C200A44CAF8AC
:1068E0001820042293E7012F11D13268DAF818102A
:1068F000914298D21D4B187818B90AF053FD002820
:1069000091D11B490A8822F002020A80B4E731685B
:10691000DAF81C200A44CAF8182084E76420316899
:10692000B8F8062000FB0212CAF8102000224FF42B
:1069300080608AF820208AF803200FF0EFFAC3E580
:10694000012F3FF4C1AD6EE7E4030020E503002012
:10695000EC1E0020D8140020E40C0020F80C0020CD
:1069600014AE23414C120020341B002000000020F4
:10697000881B00200022B54B83F89D20002E7FF459
:1069800074AF0022B24B1A605A609A60B14B1B6818
:1069900093F83030002B7FF468AF2B709BF80030F9
:1069A000D90725D52368DA0622D5AB4A1278D7064F
:1069B0001ED4DD041CD40AF0FBFCC8B9A74BA34DC0
:1069C0001B78002B00F0AE81A54B9B78002E40F089
:1069D0009781002B00F0A881A24B1A68A24B1B687C
:1069E0009B1A002B80F2A08104F09CFB85F89E602E
:1069F0000022009B9D495D8B9F8B134631F912004D
:106A00009B08A842C4BF63F07F03DBB20132B842E7
:106A1000B8BF43F04003042AF0D18C4D95F89F2075
:106A20009A4240F0888195F8A020F92A02D80132D4
:106A300085F8A020894F85F89F3097F80080B8F13D
:106A4000000F09D140460AF0ADFC002800F0758126
:106A500085F8A18004F0F0FB95F8A030142B1AD132
:106A60003B785BB195F89F305F2B07D19BF80030E6
:106A700013F0010600F0858104F054FB9BF8003010
:106A800013F0010207D195F89F30572B40F07F811A
:106A9000774809F0ABFE23685E0728D595F8A43047
:106AA0009BB19BF80030D8070FD5704BB3F9062087
:106AB000009B5B8B9A4208DD00200AF073FC20B932
:106AC000322385F8A400A5F8A63011200AF06AFC4C
:106AD000002800F0BF8195F8A8302BB995F8A230B6
:106AE00013B93223A5F8A630012385F8A830002376
:106AF000604E04AF049306F150087B60314616F8EF
:106B0000010C0AF029FC30B116F8021C232902D826
:106B100038460BF07CFC0436B045EFD1564B97E875
:106B2000030083E80300554B1F78002F00F0BA8163
:106B300001200AF037FC524E524F40B92368DA0563
:106B400040F1B183504BDB78002B00F0AC8333680D
:106B50009B0740F1A8833D8815F0010540F0A8830C
:106B600001200FF0EBF902200AF01CFC002800F0D5
:106B7000A183002D00F09E8301200FF0CFF93B8808
:106B80009D0702D402200FF0D9F93988012011F0B5
:106B9000030118BF01210CF013F9336813F00A0F39
:106BA00017D006200AF0FEFB002800F087833B8800
:106BB000580602D440200FF0C1F907200AF0F2FB7A
:106BC00038B10A22314BB3F9043093FBF2F3304A67
:106BD00013800C200AF0E6FB002800F073834FF4CA
:106BE00080700FF0ABF92B4B1B78082B01D00E2BCC
:106BF00002D140200FF092F9236859050FD5264B9A
:106C00001B79002B40F063839BF80030DA0740F1DA
:106C100064833C200DF0E0FF002840F067830122F0
:106C20001E4B1F4D1A70114BB3F906B01D4B1B685C
:106C30005A89934580F260834FF07E532B60009B0E
:106C40004FF000081E8B184B30E000BFD814002016
:106C5000E01600202C190020C4160020000000209F
:106C6000161200204C3A002054250020EC1E002073
:106C7000503B0020BE220020B4160020942C00209F
:106C800060190020141F0020641B0020183300200E
:106C90005025002031190020D02D0020581100204F
:106CA0002412002038390020FC110020714D93F986
:106CB000042093F80190002A14BF01224FF0FF3204
:106CC0001B78029201936C4B33F918A0AAEB0600D3
:106CD000002840F32583B0F5FA7FC0F22783B8F18E
:106CE000020F4FF4FA7000F0FB8323E3002E7FF4D1
:106CF000BCAD624B93F89D30002B7FF4B6AD40E6FF
:106D00003BB14FF47A715E4A126801FB03235D4A7E
:106D1000136095F89E30002B3FF46AAE0FF034F804
:106D2000002305E0002EF4D110200FF043F80123DA
:106D300085F89E305CE600227AE6534B18609BF89B
:106D40000030D8077FF588AE504B1B78002B3FF4FE
:106D500083AE4F4BDB78002B7FF47EAE95F8A130ED
:106D60000133DBB2032B85F8A1307FF675AE494BBA
:106D70005B7813B104F0D6F96EE6002E7FF46CAEAA
:106D8000F8E70B200FF016F885F8A06076E621688A
:106D9000490717D55A2B15D195F8A2302BB10123ED
:106DA00085F8A22085F8A33075E695F8A43083F025
:106DB000010385F8A4301BB10C200EF0FBFF6AE63E
:106DC0000D20FAE75D2B00F069835B2B00F06D83EB
:106DD0005E2B40F06C83032061E300222A4B1A6093
:106DE00095F89F30972B04D14FF4C8722A4B1A8024
:106DF00051E6A72B05D1294A137843F004031370F9
:106E000049E60022BB2B049213D10223ADF81230C5
:106E1000234BBDF810105A890A445A81BDF812104C
:106E20009A890A449A8105F0D3FD002385F8A030A1
:106E300031E6B72B02D14FF6FE73E7E7BE2B03D145
:106E40000223ADF81030E3E7BD2B7FF424AE4FF6FC
:106E5000FE73F6E795F8A230002B3FF448AE9BF89E
:106E6000003013F0010302BF85F8A230012385F83A
:106E7000A3303CE6341B0020EC1E0020D814002078
:106E80004C3A00205425002058250020311B0020BA
:106E9000641B00201612002048250020C416002084
:106EA000203900204FF00C0A4FF00109BF4E06F1C7
:106EB0005A08314616F8010C0AF04EFAE0B1317961
:106EC000B3780AFB0150BA4A013B03EB4303134476
:106ED000D0F8B02096F803E093420DD0C0F8B0305F
:106EE00095F8DC3009FA01F123EA010180F8ACE001
:106EF000C0F8B47085F8DC100636B045D9D14FF033
:106F00000009AC4BDFF8BC821E68AB4BA8F1AC05A6
:106F10001B680193A94B1B780293D8F80430002B0F
:106F200069D01F78002F66D0D8F8082001998A1AF6
:106F3000002A0CDB01F5FA72C8F80820012295F846
:106F4000DC1002FA09F221EA020285F8DC20029A3A
:106F5000002A50D098F8002059780432D2B2002983
:106F600040F04E81964931F91210009A128B02F1CD
:106F7000C80081422ADD93F802A095F8DC2042FA8D
:106F800009F2D10737D4BAF1000FD4BF0120022093
:106F90000EF0ACFF7A1E162A40D8DFE812F034005B
:106FA0004C00560066007D0084009F00BA00D600A9
:106FB000E200EE003F006600730084009F00BA000C
:106FC0009300AE00CA00FA0015012301C83A9142AD
:106FD00003DA9978C1F1000ACFE7012395F8DC20A4
:106FE00003FA09F322EA030385F8DC30019B03F579
:106FF000FA73C8F8083009F10109B9F1040F08F172
:107000000C088AD194E5317801205144FA29A8BFAF
:10701000FA2121EAE17131700AF000FAD5F8E000B6
:1070200007F0E8FA012395F8DC2003FA09F313438B
:1070300085F8DC30DFE7B178022051446429A8BF2D
:10704000642121EAE171B170E6E731798A44BAF14D
:10705000640FA8BF4FF0640A2AEAEA7A86F804A00F
:107060000AF0F0F951460320D6E7B1790D205144DA
:107070006429A8BF642121EAE171B1710AF0CEF957
:107080000D2FCBD071790E2051446429A8BF642103
:1070900021EAE1717171BFE7F1790520514481F373
:1070A0000801F171B8E7D5F8E0200F20D1785144FC
:1070B000C829A8BFC82121EAE171D1700AF0AEF950
:1070C0000F2FABD0D5F8E020122011785144C829F9
:1070D000A8BFC82121EAE17111709DE7D5F8E02031
:1070E000102011795144C829A8BFC82121EAE171B3
:1070F00011710AF093F9102F90D0D5F8E0201320E9
:1071000051785144C829A8BFC82121EAE1715170C2
:1071100082E7D5F8E020112051795144C829A8BF51
:10712000C82121EAE17151710AF078F9112F3FF479
:1071300075AFD5F8E020142091785144C829A8BF34
:10714000C82121EAE171917066E7D5F8E0200920B5
:1071500091795144C829A8BFC82121EAE1719171F0
:107160005AE7D5F8E0200A20D1795144C829A8BFB0
:10717000C82121EAE171D1714EE7D5F8E0200B205A
:10718000117A5144C829A8BFC82121EAE1711172BE
:1071900042E7717815205144B1F5967FA8BF4FF4AE
:1071A000967121EAE171717036E700BF5D2300201E
:1071B000ADA30108383900204C3A0020311B0020D3
:1071C000EC1E002084150020D5F8E020162092F84F
:1071D0003B105144FE29A8BFFE2121EAE17182F84B
:1071E0003B1019E7D5F8E020172092F83A105144E7
:1071F0006429A8BF642121EAE17182F83A100BE703
:1072000001297FF40FAFBF4931F9121040F6330264
:107210009142A8BF11469A784FF49663B1F5617F09
:10722000B8BF4FF4617193FBF2F3A1F561710C2FBC
:1072300091FBF3F11ED0182F7FF4F4AEC9B2C82928
:107240000B46A8BFC823D5F8E020D8B292F817E0C3
:1072500070453FF4E7AEA3EB0E034FF0080E93FB2F
:10726000FEF30133DBB2D075384603930AF0D6F84B
:10727000039B11E0A44ACBB252789A423FF4D2AEBB
:10728000184603930EF0E2FE039B384619460AF0B7
:10729000C5F8039B0133DBB2002B3FF4C3AE1846A5
:1072A0000EF024FEBEE601200EF038FE01255AE461
:1072B000002558E402200EF031FE66E440200EF076
:1072C0002DFE7AE44FF480700EF028FE8BE414203B
:1072D0000AF068F800287FF49CAC06F0D5F906F0B7
:1072E00047F906F089F801F00FFB98E401F0A6F8E1
:1072F0003C200DF03DFC8FE4BBF5FA6F187ABFBF60
:10730000ABEB02035843C2F5FA6290FBF2F0C0F116
:1073100064000FF01FFC7D490FF070FC28608EE4C4
:10732000A6EB0A00B0F5FA7F80F2D280B8F1020F26
:1073300000F0D480019B834280F29680019BC01AAA
:107340000FF008FCB24545F82800C0F2D38008F1E0
:107350000108B8F1030F7FF4B6AC246814F480542C
:1073600000F08680BBF5FA6FA8BF4FF4FA6BBBF54F
:107370007A7FB8BF4FF47A7BABF57A7B4FF0640E1F
:107380009BFBFEF3624A581C32F9131032F91000CD
:10739000421A6FF0630000FB03B0504390FBFEF015
:1073A000084400B20FF0D6FB8046E860E4B11D202F
:1073B00009F0F8FFC0B1574BDB78ABB956494046EE
:1073C0000FF012FB0FF0F6FD4FF47A7300B20003DA
:1073D00090FBF3F3C6F5FA6000B2584340F30F3068
:1073E00030440FF0B7FBE8603B885B0637D54B4B6A
:1073F000B3F904000A2390FBF3F0494B1B88C01A31
:1074000000B20FF0A7FB47490FF0F8FB46490446CE
:107410000FF0ECFA0AF098FE804620460AF094FE3F
:107420002E680446414630460FF0E8FB6F688146FF
:10743000394620460FF0E2FB014648460FF0D4FAE9
:107440004146286038460FF0D9FB314607462046B2
:107450000FF0D4FB014638460FF0C8FA686003F01D
:107460007BFE07B0BDE8F08F002069E7002039E01F
:10747000009B5B8B9B450FDBBBF5FA6FA8BF4FF4FE
:10748000FA6B4FF47A70ABEB030B00FB0BF0C3F518
:10749000FA6BB0FBFBFB71E79B46F2E7012001387A
:1074A000C0B204F091FFFFF7F6BA0220F7E7562BBF
:1074B00001D105F08DFA3B78002B3FF491AC95F8A3
:1074C0009F306F2B7FF489AC03F0B6FEFFF7E3BA71
:1074D000B8F1020F4FF4FA707FF430AF8145C5DA8E
:1074E000A0EB0900029B58430FF034FBB245A860A3
:1074F000BFF633AF55F8282002F1004245F82820A6
:1075000025E700BFEC1E0020582000200AD7233CAE
:107510003C390020641B002000007A44183300200E
:107520005025002035FA8E3CDB0FC93F2DE9F04F86
:1075300085B0804606F0A8F806F01AF805F05CFF62
:10754000CA4B1B78002B40F02E83C94E336800963F
:1075500013F4806F00F02783C64BC74D1B78002BB8
:1075600000F03881C54C2A68E368D31A7C2B40F2BE
:1075700031812427237CDFF83CB30133DFF83893D3
:10758000E2602374ABF1300A384606F063F85BF82A
:10759000040F0FF0DFFA0190BAF810000FF0DAFADA
:1075A000019B014618460FF0DDFB49460FF026FB14
:1075B0000FF000FD013700B2FFB206F039F8272FB7
:1075C000E2D1302006F046F8002006F031F806F04F
:1075D0003AF8277C17F0030723D141F28833E26899
:1075E0009A420BD9102006F035F8384606F020F8FC
:1075F000212006F02FF8384606F01AF8142006F07D
:1076000029F89F4BB3F904000A2390FBF3F006F02E
:107610000FF81C2006F01EF8002006F009F806F00E
:1076200012F8237C5B0740F0AF80022006F012F8CE
:10763000944BDFF88892B3F944000A2390FBF3F0EF
:1076400005F0F6FF032006F005F88F4B1B7813F0CA
:10765000010F00F0628109F0B9FE8C4B8C4907469E
:10766000D8680FF0CBFA0FF0CBFC80B22FB9009B9B
:107670001B6813F0100F18BF002000B205F0D8FFF0
:1076800099F80430002B4DD0DFF834A29AF800B0FE
:10769000BBF1000F46D064277E4B06201A88019369
:1076A00007FB02B24FEA4B07B2FBF7F2678A3F01D2
:1076B000BFB247EA0227BFB2C2F30322174305F065
:1076C000C9FF38B205F0B4FF628A019B013292B261
:1076D00092FBFBF10BFB112B6F4A1F88537AA4F826
:1076E00012B0012B40F01F81392005F0B3FF38B2F2
:1076F00005F09EFF282005F0ADFF0A23674F38688C
:1077000090FBF3F000B205F093FF042005F0A2FF18
:10771000B9F80630002B00F02A8100F0A7FD00B276
:1077200005F086FF02A95E4805F058FF132005F01A
:1077300091FFBDF9080005F07BFF1B2005F08AFFD3
:10774000BDF90A0005F074FF232005F083FF4E20E9
:1077500005F06EFF02A9524805F040FF122005F027
:1077600079FFBDF9080005F063FF1A2005F072FFEC
:10777000BDF90A0005F05CFF222005F06BFF4520F3
:1077800005F056FF05F05FFF237C282B22D1002354
:10779000172023742C6805F05DFF4EF660203C270F
:1077A000B4FBF0F3B3FBF7F007FB1030000200B2BC
:1077B00005F03EFF182005F04DFF4FF47A70B4FB42
:1077C000F0F4B4FBF7F007FB104000B205F030FF17
:1077D00005F039FF334B1B78002B00F08880274CD5
:1077E000314A6369A8EB030393426DD900222F4B02
:1077F0009A701A71274A1288D1B2120A9977DA77E9
:1078000019755A752968A269891A234AD07A4FF4E2
:107810007A72424391420AD32A68A261244A1278BA
:10782000013A012A9FBF10229A7002221A710A207F
:107830001A4AC4F814801168926891FBF0F192FB27
:10784000F0F283F82020121283F82120F4229A7695
:107850000122DA76302283F82220752283F8232051
:1078600078221977091259772CE000BF942C002058
:10787000601B0020F02D00204C3A0020BC15002099
:1078800018330020A83A0020301B0020341B0020B1
:10789000CDCC4C3E68170020D02D00206C17002066
:1078A00080969800E92D00203F0D03005410002021
:1078B0004D1B00202817002000007A44521B002096
:1078C0007C20002083F8242094F81CA0BAF1000F3B
:1078D00000F06883636A53B1237F002B70D040F6B9
:1078E000B732E36AA8EB0303934200F29680B84BE9
:1078F000D5F800801B78002B00F05581B54C23682B
:10790000002B00F05081B44B1B78013B012B00F29F
:107910004A81B24FDFF8D492B2E00523B9F80600ED
:10792000B0FBF3F0A9E66E2315217B43527B93FB5A
:10793000F1F322B19AF800209BB293FBF2F34FF0DF
:10794000640B9FB23A2005F085FEB7FBFBFA0FFAF5
:107950008AF005F06DFE3B2005F07CFE0BFB1A70F3
:107960000A2780B2053090FBF7F000B2C0E6B86895
:1079700080F31000D3E63B7823B1C4F8208087F869
:1079800000A0A7E7236AA8EB0303B3F57A6FA1D39E
:107990000123D9F800003B700BF051F90746D9F8E4
:1079A00000000BF04CF97F0694D18E2892D1237FF2
:1079B000002B8FD18A4B63622D2384F8283089E70E
:1079C000012284F83030874B22771B689B781E3B5E
:1079D0009342854B1CD918680221043005F07CFDC8
:1079E00094F82820804F013AD2B284F8282094F8E5
:1079F000301094F83130CAB94A1C013384F8302071
:107A000084F8313038680BF023F9C4F82C806EE725
:107A1000022118680BF00DF9E2E794F82830002BEA
:107A2000DED16362237705F089FDD9E7606A01330F
:107A300010F801EB84F831300EEB010284F83020AD
:107A400060627146DEE720680BF0F9F883B27E2BA6
:107A50002A6806D1002389F8323089F833307B70E8
:107A60000EE07A7862B999F8321061BB1B2B20D1F5
:107A700020680BF0EAF8002846D1012389F833305A
:107A800020680BF0E2F801460028DCD1574C94F84E
:107A90003730002B79D0637884F83700302B74D1DD
:107AA000A3785F09012F3DD084F8380005F091FCE0
:107AB0006BE00D2B28D1012289F8003089F83220A3
:107AC000A9F83410DCE77D2B03D1012389F8363087
:107AD000D6E799F836E0BEF1000F04D080F0200020
:107AE000C3B289F836204A1CD2B2092A89F832205A
:107AF00009F801300AD1B9F83420C2F1FF029342EB
:107B000002D1012389F837300123A8E7082AB7D822
:107B1000B9F83400034403EB132303F0FF03A9F87F
:107B20003430ADE703F00F0013F0100321D094F8C8
:107B300003E0237904F14C02A4F84430E26383EAC1
:107B40000E03724484F88C30A4F84610226484F842
:107B50003870631D002194F88C20DFF898E0E76B03
:107B6000266CBE4222D171BB734547D184F88D008B
:107B70000BE094F8382042B194F88D20013202F0E5
:107B80000F02824222D084F83830194FDFF8689013
:107B900094F833303BB12B68A3EB0803012B5BD97E
:107BA000002384F8333005B0BDE8F08F13F8011BD3
:107BB00007F1010C734582EA0102C4F83CC0397038
:107BC0004FF00101CBD384F88C20CDE7E31CC1E753
:107BD000CA2D0020B02C0020DE2D00200C0000203B
:107BE00054100020E42D0020E02D0020BC150020C2
:107BF000C82D0020C4150020F8A301081A7894F8B5
:107C00008C309A424FF0000284F8382003D0B4F947
:107C1000441001204AE7B04FE36BDFF8C892AF4849
:107C20002364E06309F58073394610387B60C7F838
:107C300000903A817A81F8F76BFA01304B4604D113
:107C40003A68511C3960022111703A683B607A60D1
:107C50000122A34B1A7098E797F800A0BAF1000F21
:107C600060D09D4A9F4913688B4294F88E3038D17A
:107C7000581C84F88E00B2F90A0003F00F0343F099
:107C800010030028B8BF43F020038DF80830536874
:107C90005B1A117A8DF809304B4084F88F300DF162
:107CA0000A030025D2F804C094F88F100DF10E00DD
:107CB000834228D21668ACEB060EBEF1000F1ADC28
:107CC0000DB184F88F1094F88F105A1C197000238E
:107CD000824224D302A9322005F0CCFB4FF0000AE7
:107CE0001AE0591C03F00F038DF8083084F88E1049
:107CF0000DF10903D5E7751C1560357803F8015BB4
:107D000069400125D4E70DB184F88F108342DAD1A0
:107D100002A9322005F0AEFB87F800A040E702F888
:107D2000013BD5E794F8903039F8130018B984F87E
:107D300090004FF4036094F89030B0F5826F03F137
:107D4000010384F8903000F0B78059D8B0F5007F77
:107D500000F094800DD8B0F5807F03D0B0F5887F17
:107D60007FF416AF604B1B685E077FF511AF0021F3
:107D70007CE0B0F5047F64D0B0F5806F7FF408AF8D
:107D800094F8913042F210710133DBB2032B88BFBB
:107D9000012384F8913094F891305943534B1B8858
:107DA000002B40F087800131514B1B78D807514B95
:107DB00048BF04311B88DA0748BF0A319E0748BF15
:107DC0001431180648BF2831DA0548BF28315E074C
:107DD00048BF6431180748BFC8319A0548BF01F54C
:107DE000C8719E0648BF01F57A71D80648BF01F5F3
:107DF000FA615A0648BF01F57A614FF4806035E0B8
:107E0000B0F5E26F53D00ED8B0F5C06F41D0B0F5E9
:107E1000E06F7FF4BDAE384A516B64234B43118A47
:107E200093FBF1F122E0B0F5046F3AD0B0F5116F99
:107E300000F0A980B0F5E46F7FF4AAAE2E4AD16BB2
:107E4000EBE72E4B1B79002B3FF4A2AE2C4B19789D
:107E500000293FF49DAE2B4B2B4A5B7B63B113880B
:107E600093FBF1F30A214FF40470594305F01CFB16
:107E7000002384F833308BE61388F3E71F4B5B79DC
:107E8000002B3FF485AE214B19680A2391FBF3F1D7
:107E9000ECE71A4B5B79002B3FF47AAE1B4B9968E9
:107EA000E4E70A211A4BB3F904305943DEE7124ADA
:107EB000916BB2E7023177E70B4B1B6813F0200A96
:107EC0007FF466AE009B1B681B0623D5514605F068
:107ED000EBFA84F833A05BE6B82C002008160020EB
:107EE000C82D0020C82C002060190020881B00200D
:107EF000301B0020141F0020F8160020521B002009
:107F00007C200020D02D0020681700206C17002056
:107F1000183300202D4B1B7B002B3FF439AE94F817
:107F20009230032B2DD8DFE803F002181F26284AD1
:107F30001268107892F803E09179090401EB0E21A0
:107F4000014401EB03610133DBB2042B08BF0023C2
:107F50004FF4826084F8923088E71D4A12685078A6
:107F600092F804E0D179E8E7194A1268907892F81B
:107F700005E0117AE1E7174A1268507992F806E0B5
:107F8000F0E70021DDE7144B1B79002B3FF400AE36
:107F9000124B197800293FF4FBAD114B1A880A23C4
:107FA00053433DE7DFF84090D9F800000AF04DFE5A
:107FB000C0B201287FF68EAC02280A4F3FF4DBAC3A
:107FC00005F0ACFA01233B7084E400BFD02D002003
:107FD0002C19002038390020521B00207C20002062
:107FE000681700200C000020E02D0020024B1A88AA
:107FF0009B7802808370704720A40108064A1168AC
:1080000049B1642350684343B3FBF1F303490B8048
:10801000002313605360704750160020802000201A
:1080200070472DE9F843304B06461B782BB92F4A91
:10803000136053609360BDE8F8832D4B9F68986090
:108040002C4B5B79012B09D001D3042B04D90022DE
:10805000264B1A605A609A60BDE8F88340F6E449FE
:108060004FF47A74244BDFF8A480DA79234B244D43
:1080700033F81200B8F9023080B209FB00F2C3EB0A
:1080800012336343B8F9002093FBF2F3EB600EF078
:108090005DFD01461B4809F0E3FE0EF0B1FF80B222
:1080A00009FB00F9B8F90200B8F90030C0EB193942
:1080B00004FB09F494FBF3F4D5F80C80F01BAC60DE
:1080C00008FB00F00EF046FD0F490EF097FD6968C1
:1080D0000EF08CFC68600EF06DFF044B286083E8A6
:1080E00010019860BDE8F8837C2000206C17002008
:1080F00050160020521B0020E40C0020F80C002039
:10810000C4100020D41000202FE33E31D4110020F1
:108110002DE9F843224B234D1B79012B3BD1224BF8
:10812000224E9A78224B33F81240A4B220460EF029
:108130000DFD0146304609F093FE1E4B9F7893F8E3
:10814000009093F801800EF05BFF44F6FB7209EBA0
:10815000491983B209FB032309FB0424C8EB08383F
:10816000B3FBF8F3B4FBF8F4B3FBF7F3B4FBF7F4A9
:108170009BB2A4B226F8043C26F8024C2B806C80FB
:108180000D4B1B78022B04D10C4B6A881A802A886D
:108190005A80BDE8F88300232B806B80F0E700BF96
:1081A000521B002068170020E40C002094100020CF
:1081B000F80C0020D0110020301900203C170020BE
:1081C000F7B5264E3368002B44D0254B1B78022B85
:1081D00040D10024234D244F04F12000C0B209F007
:1081E000E1F8C8B32B7883BBE25D72B3306850B35B
:1081F00055218DF8001001218DF80220AA228DF85A
:10820000011019468DF804308DF803201DF8012067
:108210005340082213F0800F02F1FF324FEA43036C
:1082200018BF83F0310312F0FF02DBB2F2D101314B
:108230000429EBD18DF80330AA23052269468DF875
:1082400004300AF008FD01232B700134032C05F1E2
:108250000105C1D103B0F0BD2870F6E70811002078
:108260000F1100200C11002023A4010838B5194B70
:10827000187808B31849CC88FCB120460EF066FC8B
:10828000164B054698680EF065FC014628460EF030
:10829000ABFB13490EF0B2FC054620460EF05AFC2B
:1082A000014628460EF05EFD0EF084FE6428A8BF4D
:1082B000642020EAE070C0B238BD0A4B4D781B88BC
:1082C0000A7800FB15346423521B63435043B3FB0D
:1082D000F0F0EBE77C200020521B00206C17002000
:1082E0000000C84268170020194B2DE9F0411C68B6
:1082F00007460D2C984607DC0023164A9C4206DCF4
:108300000025144EA54208DD0020BDE8F08152F89A
:1083100023108F42F8D00133F0E756F82530681C5F
:108320007BB98000621B011F92003144304401344C
:1083300011F0D1FD46F82570C8F800400120BDE8D5
:10834000F0811A7D3B7D9A42EBD30546DAE700BF08
:10835000182000201C2000200F28F8B50FD00D2871
:108360000CD83422124B02FB003009B1C3684BB960
:108370000022104D10492C68A24206DBF8BD0F4BBD
:108380001868F2E7BDE8F840AEE751F822709300B4
:10839000B84203EB010609D1A21A04339200194432
:1083A0003046013C11F097FD2C60F8BD0132E3E747
:1083B00038000020182000201C2000205424002019
:1083C00008B50C4B197801290CD00AD302290DD01D
:1083D0000AF072FB084B00F5F42000F5907018606D
:1083E00008BD002100200AF0EBFCF1E700200AF0B4
:1083F00050FCEDE74A2500204C25002010B504462E
:1084000020460AF019FC00B110BD0A200AF0A7FBB3
:10841000F6E700230C2130B5074C01FB03425568F9
:10842000A84203D00133052BF7D130BD0023C3622E
:108430001381536030BD00BF3C400020F8B50546B5
:108440000024094EA359A719AB4207D12846FFF7CC
:10845000E0FFCC220021384611F057FDCC34B4F5B2
:10846000197FEFD1F8BD00BF9C0D00202DE9F04F22
:1084700006464FF000080C2093B002939DF87070F0
:108480009DF874906B4B0591039200FB08F2D11894
:10849000D256B24200F0F08008F10108B8F1050FA1
:1084A000F3D100207CE01E2E00F0BB801F2EF8D1FF
:1084B000CDF800903B46029A03990120B7E01C20BA
:1084C0000AF0F6FB054616210AF018FC28460AF0C9
:1084D00037FC594FC8200AF042FB28460AF035FC09
:1084E000BB69564843F00403BB614FF4C053ADF879
:1084F0001C3003238DF81E301C230DEB03018DF877
:108500001F3004F0EBFE4FF480234D4D4D4A4FF0E9
:10851000010953616B65082305F1540085F8593052
:1085200085F85A900CF096F9474B484A1C60FB6955
:10853000474943F40003FB610227464B13601F7257
:10854000454A464B1360464A1B6811609847454BA5
:10855000454A07A8DA608DF81C608DF81D708DF80B
:108560001E408DF81F9004F095FE2A238DF81C30D4
:108570009DF81F308DF81D908DF81E409BB107A807
:1085800004F088FE394B3A48EB600C23294A067107
:1085900003FB0828BDF81430C8F80400A8F8083018
:1085A00013B0BDE8F08F4FF48062324BC3F88420E3
:1085B000E8E70133072B40F09280002397E0013376
:1085C000072B40F0AF800023B4E0049B53B1691C3B
:1085D000C9B220B14FF00B0EC17180F806E01A212C
:1085E0000AF08CFBFA0740F1F1800135EDB2BBF1E6
:1085F000000F04D00C218BF807508BF806104A218D
:108600005846E1E04FF6DF72236D1A80DA6842F0D7
:108610002002DA6034E1226DD36843F08003D36036
:108620005DE13B462046029A0399CDF8009002F0A6
:108630007BFE5BE13C40002000100240000801404E
:108640005016002000040140D8004242443A002065
:10865000100000208C4000206C39002030040020E5
:108660006839002000ED00E00005FA0528A40108A3
:108670005C16002000E100E00C89002C7FF411AFB3
:10868000142E3FF41CAF3FF70EAF16B1022E7FF44D
:1086900008AF984BF5B253F82640002C00F0258126
:1086A000954BD4F854A02360029BA36004F15A03B5
:1086B000636104F5AD73A3614FF48073E3602361DC
:1086C000DAF8043023659AF816000CF031F8DAF87D
:1086D0000C10F1B1894800234FF01C0E83460EFBAD
:1086E000030CDCF8042091427FF463AFDBB21C2062
:1086F00000FB03B3824A1869D2F814E04EEA000086
:1087000050610C201876681C5876236D2163043361
:10871000E364DAF8081000293BD0784800234FF0D2
:108720001C0C86460CFB030BDBF8042091427FF403
:1087300046AFDBB21C2101FB03EE714BDEF81010DB
:108740005869084358610B208EF81800681C8EF891
:1087500019005A699AF8190011435961694B800947
:10876000CEF808309EF80D308DF81D008DF81C30C5
:1087700000238DF81E300123CEF8144007A88DF891
:108780001F3004F087FDDAF808306363236D04338B
:10879000A36494F858000AF08BFA834694F85900C1
:1087A0000AF086FA07F0020319F0080F04933FF469
:1087B0000CAF0135EDB210B10B23C571837119F007
:1087C000100F14BF1A211E210AF098FADAF80C30A3
:1087D00013B1DAF808308BB99AF8183007A88DF879
:1087E0001C309AF81A309B098DF81D3000238DF843
:1087F0001E3001238DF81F3004F04CFD01230025AD
:1088000084F84430039B2562E362029BE561A36028
:10881000A5626562677184F8069020460AF05CFDE7
:10882000FB072DD5236B002B3FF4ECAE07A804F01B
:108830001BFBE36C206B07934FF480531093802352
:108840000C93E36811950A9320230F9363690B95AA
:1088500008930D950E95099504F031FB07A9206B3F
:1088600004F00FFB226B216D136843F001031360CA
:108870008B8A9BB243F040038B8253689BB2236484
:10888000049B002B2BD0636B002B3FF4C4AE07A8D6
:1088900004F0EAFAA36C002507934FF48053109379
:1088A00080230C932369606B0A931023119509931D
:1088B0000B950D950E950F9504F001FB07A9606BC4
:1088C00004F0DFFA636B1A6842F002021A60226D4C
:1088D0005D605D60938A9BB243F080039382226D5A
:1088E00093899BB243F400539381204600287FF480
:1088F0004CAED6E5880B002050A4010814030020DC
:1089000000100240ED3101082DE9F74F01200DF074
:1089100019FA0024234D244E78B3022C2DD84FF0A1
:10892000CC0909FB04F855F8087005EB080A17B1E3
:108930000134E4B2F0E70323C27890F90200009317
:108940001A4B019753F8223001213A46FFF78EFD6A
:10895000834640B14A4639465046013411F0D5FAB3
:10896000E4B245F808B0002196F85C20104FD3B26D
:10897000042B05D909B186F85C3003B0BDE8F08F4F
:1089800002F1010E07EBC20037F832200133D207A3
:10899000DBB24FF0010102D586F85C30BCE77246CD
:1089A000E5E700BF9C0D00205016002090A40108B0
:1089B0000E40002038B1038813EA010003D08B4237
:1089C0000CBF01200220704730B5224C85B02388AF
:1089D0006568B3F5805F207D1F49204A637D1ED303
:1089E00091F820101278E56020746174A274E37429
:1089F00053200DF075F8E0680DF025F9207C0DF09E
:108A000022F9637C01A80193A37C0293E37C039386
:108A10000DF08AF800230120238005B030BD91F8C5
:108A200020101278019504F10C058DF808008DF8DE
:108A300009108DF80A202946082201A88DF80B306C
:108A400011F03AFA0028E8D001AB03CBE0602161D5
:108A5000CEE700BFB0160020641B0020311B0020B1
:108A60002DE9F74F384C0025D4F8188004F1240183
:108A7000464608F1300746F8040B04F1300B04F1C8
:108A80003C0A04F14809685801910EF093FA46F83F
:108A9000040B55F80B000EF08DFAB06055F80A0083
:108AA0000EF088FA294B7061EB1858680EF062FFDF
:108AB00009EB05035B6B043527F8020B0C2DBB801B
:108AC0000199E0D10025224F08F1280657F825002A
:108AD0000EF070FA0135042D26F8020BF6D10025B0
:108AE000B4F88C3094F89470A8F83C30B4F88E3018
:108AF000DFF86490A8F83E30B4F8903008F14406EE
:108B0000A8F84030B4F89230A8F84230BD4212DBE9
:108B1000B4F8BA30A8F86430D4F8C030A8F8663099
:108B20000C4B1B88A8F86830B4F8D230A8F85E3037
:108B300003B0BDE8F08F59F825000EF03BFA01357F
:108B400026F8020BE2E700BFB0160020FC3F002031
:108B5000341B00204A1B0020481700200D4B1A88A8
:108B600001321A80D3F8D8200132C3F8D820B3F8E4
:108B7000DC20013292B2202A03BF0022A3F8DC20BD
:108B8000B3F8DE20A3F8DC2004BF0132A3F8DE2016
:108B9000704700BFB016002038B5244B054693F847
:108BA000E0300C46093B012B3FD845200CF098FFE4
:108BB00028460CF095FF0E2D0ED003D83DB10D2D9B
:108BC0000FD038BD1E2D07D0FF2D29D038BD20680D
:108BD000BDE838400DF037B820680DF034F8606813
:108BE000F6E763782078A3B180F080000CF078FF7E
:108BF000A468E0B20CF074FFC4F307200CF070FF1F
:108C0000C4F307400CF06CFF200EBDE838400CF0B8
:108C100067BF0CF065FF6068BDE838400DF022B812
:108C200003480CF0F9FE0020EFE738BDB016002035
:108C300018C301082DE9F04F5F4C8BB0B4F8DC305D
:108C400005465E4F002B40F0BF803B78012B04D1DE
:108C50007B78202B01D1FFF7B7FE2846FFF700FFF6
:108C6000A56949202E460CF03BFFD4F8D8000CF043
:108C7000EAFF56F8040B0CF0E6FF30460BF0B4FFA9
:108C800005F110000BF0B0FF10264FF0010905F1BF
:108C90001C08D4F8E42009FA06F3134203D0D8F8EC
:108CA00000000CF0DFFF0136132E08F10408F0D1AC
:108CB000032105F128000CF0D9FFB4F8F830B5F91C
:108CC0002E00C01A0CF0BFFFD4F8E430DB0408D546
:108CD000B4F8FE00B5F86430C01AC0F30D000CF013
:108CE000B2FFD4F8E4309E0403D5B5F866000CF06A
:108CF000AAFFD4F8E430180403D5B5F868000CF0E6
:108D0000A2FF032105F130000CF0B0FFD4F8E430ED
:108D1000D90204D5032105F136000CF0A7FFD4F8E1
:108D2000E4309A0204D5042105F13C000CF09EFFCA
:108D30000126B5F944000DF00DFFD4F800110DF037
:108D400053FE0EF05DF90CF07EFF94F8949005F15F
:108D50004608B14527DCD4F8E4309B0505D5B5F9C4
:108D60005E00A0F2DC500CF07DFFA269E26122629D
:108D70001349144B521A921053430322013393FBAD
:108D8000F2F202EB42029B1A6C2202FB0313A36174
:108D9000012384F84832BB78012B01D109F09EFCF5
:108DA0000BB0BDE8F08F38F9020BB5F9443001364D
:108DB000C01A0CF057FFCCE7B01600208C41002001
:108DC000B417002013DA4B68D4F84C32D4F8502290
:108DD0009A4207D00AA941F8203D0020C4F8503239
:108DE000FFF7DAFEB3490422A1F5147011F064F81C
:108DF00058B1D4F854320AA9039363681E2041F88D
:108E0000203DC4F85432FFF7C7FE3978B4F8DC309F
:108E100078780B44013BB3FBF0F200FB123399422C
:108E2000B9D9FFF7D1FD2846FFF71AFE5020D4F834
:108E30001890D4F81C800CF053FE226AA3691068C5
:108E40001B68E2690344106809F10405A3EB4000C4
:108E50000CF008FF002308F1040050F8231055F827
:108E60002320521A02A941F823200133032BF4D105
:108E7000002508460BF0B8FE09F1100008F11001BA
:108E800051F8252050F825309B1A02AA42F82530C7
:108E90000135032DF4D110460CF046FE10260122B8
:108EA00009F11C0B08F11C0AD4F8E43002FA06F1AF
:108EB000194208D0DBF80000DAF800300192C01A3D
:108EC0000CF0D0FE019A0136132E0BF1040B0AF1BF
:108ED000040AE9D1002309F1280008F1280131F939
:108EE000026B30F9022B921B02AE46F823200133AD
:108EF000042BF4D1002602AB53F82530B600F6B2AD
:108F00002BB103F108020F2A54D846F0010615F1DF
:108F1000FF35F0D2002530460CF0E2FDAA460DF1F7
:108F2000080B06F00303022B56D0032B68D0012B4D
:108F300007D1BAF1000F45D19A46DBF800502D0158
:108F4000EDB20BF1040B06AB5B454FEA9606E8D198
:108F5000BAF1000F02D028460CF0C2FDD4F8E4307C
:108F600013F4805506D00125B9F86420B8F86410D0
:108F7000521A02929E040AD50AAA02EB8501B8F899
:108F80006600B9F866200135121A41F8202C180441
:108F90004AD50AAB03EB8502B8F86810B9F8683017
:108FA00001355B1A42F8203C012D68D102980CF083
:108FB00059FE3BE08033FF2B94BF46F0020646F09B
:108FC0000306A4E7DBF800004FF0000A00F00F00F2
:108FD00028430CF085FDB4E7BAF1000F04D19BF8EB
:108FE00000000CF07DFDACE7DBF80000C0F30310DF
:108FF00028430CF075FDDBF800502D01EDB2A0E721
:10900000BAF1000F04D19BF801000CF069FDE6E70E
:10901000DBF80000C0F3033028430CF061FDDBF8FF
:109020000000C0F30710E4E7002DBDD1032130207C
:1090300007F0BCFBD4F8E430D90203D50321362075
:1090400007F0B4FBD4F8E4309A0203D504213C20A5
:1090500007F0ACFB94F89410442007F0A7FBD4F879
:10906000E4309B0506D5B9F95E00B8F95E30C01A48
:109070000CF0F8FDE369A2692362E26178E6002062
:109080006B1E02AA52F823204000C0B20AB140F081
:10909000010013F1FF33F4D20CF022FD002602ABE5
:1090A00053F8260008B10CF0DDFD0136AE42F6DBC8
:1090B000BCE700BF041900202DE9F74FA3EB020B1A
:1090C00016460E9B0D9A002914BF062504259B1AEF
:1090D00001934F4B0446D3F85C22894601329846EF
:1090E00029D1D3F85822954240F28F80DFF834A17D
:1090F0005AF822000CF0BEFF0B300CF035FC07468E
:1091000018B1012003B0BDE8F08FD8F858124148DB
:109110005AF82120032994BF214649460CF0DEFD70
:109120003D4988F860720A68101AD8F85C22086015
:109130000132C8F85C22DFF8E090D8F85C420C9B62
:109140009C421BDB13D101200CF00EFC78B9324994
:109150000A200A68013A0A600CF0C2FCD8F85822CA
:109160000132C8F858224FF0FF32C8F85C22D8F814
:109170005802854294BF00200120C3E70D9B53B1E4
:10918000019B04FB03F20D9B995C01228A40D8F8F5
:10919000E4100A4228D004FB0BF4D8F858223719FF
:1091A00042BB30590CF066FF00F1050A50460CF046
:1091B000DBFB0028A5D1D9F8000098F86022A0EBCD
:1091C0000A00C9F80000C2B12C200CF089FCD8F8C4
:1091D0005822B2B930590CF01FFC97F904104B1CFF
:1091E00002D00E480CF07AFDD8F85C220132C8F8A3
:1091F0005C22A2E74FF0030AD8E7012288F8602238
:10920000E5E7174439790648ECE700207AE700BF24
:10921000B016002023C301088841002032C3010892
:109220002AD9010878A4010810B50C4C94F8E02064
:109230000B2A0BD8012340F60301934019400CD1AF
:1092400013F4C06F02D0FF20FFF7A6FC044B1B688D
:10925000C4F85C320B2384F8E03010BDB016002057
:109260004C3A002030B5144A58B113885B08012BE2
:1092700098BF48F2050313800B6803F5C333A0338E
:109280000B60138813F0010306D10C4C04F1F405B4
:1092900092F878118B4200DB30BD54F8231049045A
:1092A00041BF92F8EC1002EB8101D1F8840045F83F
:1092B00023000133ECE700BFAC190020B0190020F7
:1092C0002DE9F047264B274CB8B11A78F02A28DD53
:1092D0007F2293F901001A7094F87A21904201DA02
:1092E000002802DA9A7852429A709A7802445A70A8
:1092F0000A6802F582421A320A6000221146187882
:10930000194D94F8786193F9017093F902E0C0F176
:10931000FF08A0F17F0C05F1F409B24204D3BDE8C7
:10932000F0870F321A70E3E755F8223094009B045F
:1093300010D5CBB2DB1B83EAE37AAAEBE37ABAF16E
:10934000010F09DC53B1734514BF434663464C44D7
:10935000E37001310132E0E70823F8E70346F6E75E
:1093600034000020AC190020B0190020F0B5264AC6
:10937000A0B192F87C31DBB1013BDBB282F87C31E9
:109380002D23D2F880014343642093FBF0F31F4860
:10939000053390FBF3F308681844086000210C467D
:1093A0001B4D05F1F40692F87831994203DBF0BDCC
:1093B00092F87B31E0E755F821008F00C0F30323DA
:1093C000062B1AD192F88431DB0718D592F87C313C
:1093D00092F87BC103EB040E9EFBFCF30CFB13E342
:1093E000012BCCBF0023012333B1C0F3834002EB38
:1093F0008000D0F88400B85101340131D3E7E34351
:1094000003F00103F0E700BFAC19002040420F0059
:10941000B01900202DE9F0410F46464C48B394F8AE
:1094200085310E68002B4AD0D4F88C51D4F888319D
:1094300025F0004523F00048414628460DF090FDF8
:1094400000B9454628460DF0B5FDA0F119032D20C1
:10945000584340F2DB1390FBF3F0374B053093FB9E
:10946000F0F094F89831064483F001033E6084F8EC
:10947000983194F8983103B3D4F888512F4928468D
:109480000DF078FD08BB28462D490DF055FD00284C
:1094900014BF08250025D4F88C61284930460DF00A
:1094A00069FDA0B145F0010500222649264F01F1D2
:1094B000F40694F878319A4212DBBDE8F08106F5A3
:1094C000433606F5A0760E60D3E70425E3E71C4992
:1094D00030460DF031FD0028E6D045F00205E3E707
:1094E00051F822304FEA820ED80318D594F999C169
:1094F000C3F3031003F00F03634512DD94F99AC11F
:109500006345ACBF0223002394F99BC160450ADB8D
:1095100043F004031D421CBF3B684EF80630013285
:10952000C7E70123F0E794F99CC16045D8BF43F039
:109530000803EFE7AC19002040420F000000C841CB
:109540000000C8C1B0190020DCA4010800230A4AA9
:1095500070B5151D02F1F80692F87841A34200DBC0
:1095600070BD55F8234030EA040404BF0C6846F887
:1095700023400133F0E700BFAC190020154B60B168
:109580006422B3F89E01424340F2FF3092FBF0F2B6
:10959000322A04DD012283F8A0210F4A09E0142AAF
:1095A00093F8A02182F0010283F8A021CCBF0B4ADE
:1095B0000B4A086802440A6093F8A02142B993F864
:1095C000EB300849203301EB83014FF48060BDE7A5
:1095D000704700BFAC19002040420F0020A10700D7
:1095E00048E80100B0190020144B78B193F8A1218C
:1095F0004AB1012A93F8A2210AD082F0010283F82D
:10960000A2210F4A09E0012283F8A2210D4A04E0B9
:1096100082F0010283F8A2210B4A086802440A6022
:1096200093F8A22142B993F8EB300849203301EBBB
:1096300083014FF4407089E7704700BFAC190020E8
:1096400048E8010040420F0020A10700B0190020A7
:10965000304B88B393F8A321013202F00F0283F854
:10966000A32122BB83F8A42193F8AA212AB193F85D
:10967000A12112B1022283F8A421D3F8B421D2058A
:1096800008D593F8BB212AB193F8A42142F0040233
:1096900083F8A42193F88421D00708D4B3F8DC21FF
:1096A0002AB193F8A42142F0010283F8A4210A68A8
:1096B00002F5C332A0320A6093F8A4211AB393F8DA
:1096C000A3118B081A41D20722D5012B01F0010109
:1096D0000BD002D3022B12D070470F4BA3F118020C
:1096E00000290CBF1946114606E00C4B03F1080295
:1096F000002914BF194611464FF4003026E7084BE5
:1097000003F11802ECE793F8DE310BB10549F3E7FA
:10971000704700BFAC190020E8A40108D0A40108DC
:10972000E0A40108DCA4010838B504468022002129
:1097300010F0EBFB3822002104F1800010F0E5FB73
:10974000174A00231546E118D0580433382BC1F8C6
:109750008000F8D12422134904F1C0000DF0A4FFC9
:109760000B22114904F1E4000DF09EFF00230322B7
:109770000E4884F8EF3084F8F020190142189279ED
:1097800012F0100205D0294491F86C3084F8F130C1
:1097900038BD01330C2BF0D184F8F12038BD00BF67
:1097A000D0A4010808A501082CA5010838A50108C6
:1097B000022803D0431E584258417047054B1B797D
:1097C00013B1142007F0EEBD034B93F8840100F0B1
:1097D00001007047D02D0020AC1900200F2A10B5D1
:1097E0001CD805280AD8052918D806240C4B04FBD8
:1097F0000030014481F8C420012010BD062806D1A4
:109800000A290BD80648014481F8E820F4E7072824
:1098100004D119B9024B83F8F420EDE7002010BD04
:10982000AC1900200022F0B5344C11461046A64673
:1098300054F820305BB1C3F30325062D00F101007D
:1098400008BF01319D0448BF01322028F0D1002417
:109850000F252B4B2F4683F8791183F87A21214667
:10986000224683F87801844227D1B94239DD394450
:1098700048100130013983F89B014910AA4283F84E
:109880009C1133DD2A4451100131013A83F89A11B9
:10989000521083F89921062293F87911B1FBF2F066
:1098A00002FB101010F0FF0F04D00A46062A01DD5B
:1098B000D10720D583F87B21F0BD5EF82460013408
:1098C000C6F3031C614506F00F06B8BF6146674545
:1098D000A8BF6746B242B8BF3246B542A8BF3546B8
:1098E000C1E7072183F89B110621C7E7072283F808
:1098F0009A210622CDE75210D8E700BFB019002008
:10990000AC1900202DE9F04F884987B091F8DF317C
:1099100003F0FF04002B49D1B1F8E8212746039258
:10992000B1F8EA21A4460292A64622463C2091F8CC
:10993000E49191F8E55191F8E631A1F8E041A1F800
:10994000E241019401F1F80B059121B2202930D1B7
:109950007649BCF1000F01D0A1F8E0E10FB181F828
:10996000E491019808B181F8E5510AB181F8E63136
:10997000BCF1000F02D02023A1F8E231012381F8CD
:10998000DF3191F816358BB140F22A33D1F8182522
:10999000D1F81C15536000238B840B889BB243F0D5
:1099A00001030B80136843F00103136007B0BDE8A7
:1099B000F08F0BEB840C9CF803109CF802C0CCF1E8
:1099C000FF0C1FFA8CFCBCF1000F00F0AA803C26B3
:1099D0003BF82480CCF1FF0CB8FBF6FA01FB0CFC41
:1099E0004FEA2C2CBAF1050F00F29E80DFE80AF056
:1099F000033A4F617586A1EB0C0508FB05F5B5FB35
:109A0000F0F55FFA8CF31D44EDB201221746019286
:109A10004FF0170C4FEA012949EA05490EEB0C06F5
:109A200049EA03090496049EA6EB0C08012606FAEF
:109A30000CFA039E1AEA090FB246029E1FFA88F832
:109A400018BFB246059E1CF1FF3CB04488F8ECA15B
:109A5000E9D20EF1180E1FFA8EFE01344FF0010C00
:109A6000894672E7B8FBF0F200FB12881FFA88F80B
:109A70005FFA8CF3C8F13C08A1EB0C0C0CFB08FC62
:109A8000BCFBF0FC0D469C445FFA8CF1BDE7B8FBD3
:109A9000F0F300FB13835FFA8CF29BB2A1EB0C0C8A
:109AA00003FB0CF3B3FBF0F30D461344DBB211469A
:109AB000ABE7B8FBF0F500FB15881FFA88F5C5F198
:109AC0003C08A1EB0C0505FB08F5B5FBF0F55FFACA
:109AD0008CF21544EDB20B46E9E7A1EB0C035FFAFB
:109AE0008CF5B8FBF0FC00FB1C8C1FFA8CFC0CFB0B
:109AF00003FCBCFBF0FC0B46AC44C5E7B8FBF0F341
:109B000000FB13881FFA88F3C3F13C08A1EB0C0398
:109B100003FB08F3B3FBF0F35FFA8CF52B44DBB2E5
:109B200073E70B460D4670E7494671E7AC19002014
:109B30002DE9F04FB24C8BB094F820350646E3B1D6
:109B400094F8DF31CBB90F2007F02CFCAD4DB8B144
:109B500094F8F33013B194F8DE318BB9EB7863B13C
:109B60000023A949A94A096842F823100133202B90
:109B7000FAD1FFF7C7FE0023EB700BB0BDE8F08F02
:109B8000012200239146EA70A148A24DA24FDFF8BE
:109B900098E2019350F823104FEA830C711A01EBFD
:109BA0000508B84509D9019A09FA03F842EA0802FA
:109BB0007145019288BF4CF800600133072BE9D151
:109BC000019B002BD9D094F88431944F13F00103FA
:109BD000059317BFB4F94635059BA3F57A72642344
:109BE0001EBF53434FF47A7293FBF2F3C4F88031F3
:109BF00094F8F430B4F89E2104EB4303B3F9409594
:109C000094F8EB304FF00008203307EB8303029306
:109C100043F69823534340F2FF3293FBF2F303F2EF
:109C20004913089394F8E830C4F86495203307EB9F
:109C30008303039394F8E9300697203307EB8303FB
:109C40000493B4F86835079394F878319B0009932E
:109C5000099B434516D1002401276D4D704E019A92
:109C600007FA04F3134205EB840156F8243014BFBD
:109C70000120002001349847072CF0D10BB0BDE83B
:109C8000F04F3FE6029B1D889C78DE78634B58F8C6
:109C900003A0CAF30323042B00F29280DFE803F051
:109CA0003C6294A20300B646A446AB460898002244
:109CB000FF2113461AF4805F1DD040F2DB5AD145D4
:109CC0004FF4FA7A00F3B280A9F57A74A3EB0B0390
:109CD000A2EB0C02A1EB0E0163436243614393FBD1
:109CE000FAF392FBFAF291FBFAF15B44624471449D
:109CF0009BB2D2B2C9B24FF4B474034493FBF4F0F4
:109D000004FB1033414828F80030034643449A705E
:109D1000D97008F104089BE7CAF3834E0EF11104D1
:109D20000EF1200304F00F040EF10F0E20340EF09C
:109D30000F0E07EB84000EF1200E07EB830137F8BE
:109D40002450C678847807EB8E008A7837F82EB0D6
:109D500037F82330C97890F802C090F803E040F259
:109D60006710A7E700232F499A0031F82310E9B9BB
:109D7000254BCAF385511A44002392F82A2141FA4F
:109D800003F0C00719D506211D4801FB0202134448
:109D900093F8C430069A203302EB830132F8233063
:109DA0008A78C978B646A446AB46D8E707980142F8
:109DB000DED10133042BD6D102E00133062BDED1F4
:109DC000314622462B46EDE7059B2BB1049B049AB6
:109DD0001B8892780499E4E7039B039A1B88927886
:109DE0000399DEE7FEF742FA96235843642390FB7B
:109DF000F3F0B64600F24910A446AB4657E700BF61
:109E0000AC19002034000020D0A40108A41A0020BE
:109E1000D01E00203F4B4C003E4B4C00B0190020A0
:109E200008A60108F8A501089F860100A9F2DC5EDA
:109E3000ED1AA41A761A0EFB05F50EFB04F40EFBC0
:109E400006FE95FBFAF594FBFAF49EFBFAFE2B4412
:109E500022448E449BB2D2B25FFA8EF14BE700BF30
:109E60001FB5074B074A0293074B08490193084B5C
:109E700008480093084B06F031FF05B05DF804FB7D
:109E800055BE01083BBE01084CBE01085FBE01087B
:109E900040BE010851C3010879BE010838B50A4B1C
:109EA0000D4603EBC00494F8B820084853F822107C
:109EB00006F05DFE94F8BE302BB1691C0448BDE885
:109EC000384006F054BE38BD24A6010885CB0108F1
:109ED00029D901082DE9F04F00252F46AA465E4EEC
:109EE0008BB05E4B5E491A680023934223DB013539
:109EF0000E2D06F13406F4D1584991F84330BBB128
:109F00004FF47A73886DCA6DB0FBF3F35209096E92
:109F1000544806F0E3FE0A2297FBF2F39AFBF2F1B3
:109F200002FB13775048009702FB11A206F0D6FE01
:109F30000BB0BDE8F08F51F82300864222D00133E8
:109F4000D3E74346079A0121484806F010FE4C46E5
:109F50003AE038B10CF0FEFD014645480CF002FF36
:109F60000DF028F8044642462946424806F0FFFD17
:109F70004FF0000928E0584631E021463E4806F0FF
:109F8000ADFE5BE07368012D0793336BD6F800805C
:109F90000893B36AD6F82CB00993F069D9D138B1D7
:109FA0000CF0D8FD014632480CF0DCFE0DF002F852
:109FB000324B81461B78012B90FBF3F4C1D942460A
:109FC00001212C4806F0D3FDBBF1000FD3D041F2A4
:109FD00088314FF47A700BFB0411B1FBF0F0099B50
:109FE0005B091DBF41F288324FF47A7103FB0422F2
:109FF0001A4618BFB2FBF1F21849052D91F843102B
:10A000001CBF8244BF180029B7D04FF47A7E08994C
:10A01000B1FBFEF104910A2192FBF1FE01FB1E222D
:10A02000039290FBF1F201FB120100920191CDF835
:10A0300008E05A462146124806F050FE012D7FF4F2
:10A0400056AF0E4B1B78012B7FF651AF4A4607994E
:10A050000C4806F043FE4AE7380000201820002094
:10A060001C200020C1C30108E1C301087AC3010814
:10A07000002474496BC30108BDC30108BC32002031
:10A080008DC30108B1C30108364B2DE9F3411968AE
:10A090004FF47A733448B1FBF3F106F01FFE334BF3
:10A0A000334F1A78334B3449344C03EB8203D3F8E3
:10A0B000203197F864200988314806F00FFE314BB3
:10A0C000D4F8D8123048B1FBF3F106F050FD06F099
:10A0D000EEFD2E4A2E492F4806F000FE2E4A2F4B49
:10A0E0000021D31A2E48B7F8662006F0F7FD266D3A
:10A0F0002546002E33D030460CF02CFD0146294871
:10A100000CF030FE0CF056FF8046D5F8EC0038B16C
:10A110000CF020FD014623480CF024FE0CF04AFF11
:10A120000446E86938B10CF015FD01461D480CF0F5
:10A1300019FE0CF03FFFB7F8681043466429019000
:10A14000A8BF642100943246174806F0C7FD174B9C
:10A150001748198802B0BDE8F04106F0BFBDB0460F
:10A16000D3E700BF4C3A00200FC401084D1B00206C
:10A170001820002024A601086817002038000020BD
:10A1800029C4010840420F004FC4010800500020BC
:10A19000000800005FC401080000020800F8010880
:10A1A00083C4010800247449BDC40108881B002031
:10A1B00003C501082DE9F04F0746304C87B02378DE
:10A1C0002F4A608852F8238005F098FB2D4BD0F879
:10A1D00004A093F86A3082689BB1D3469246012668
:10A1E00007F040030593A379721E002B08BF0123DB
:10A1F000934208DC244B08349C42E0D107B0BDE810
:10A20000F08F9B46EBE7A38813441AF803501BF822
:10A210000330EA1AD2F1000949EB020993B900961A
:10A2200043461A4A4946384606F01AFEC5B9059B08
:10A2300033B900964346154A4946384606F026FE8D
:10A240000136D0E703F00F021B094033029201935D
:10A25000009643460E4A4946384606F001FEE5E7B9
:10A2600005F00F032D0940350293019500964346F2
:10A27000074A4946384606F009FEE1E7DCA6010830
:10A2800024A601081820002044A701081EC50108C3
:10A2900032C501082DE9F04F89B007460BF0EAFE00
:10A2A000044628B94120FFF785FF09B0BDE8F08FCB
:10A2B0000246914938460FF06BFE904D0646002845
:10A2C00049D18F4806F028FF8E4CDFF86C82DFF80A
:10A2D0006C9204F58477A2882168B2FA82F201F1C7
:10A2E0004041A379A1F58431890A413155F82330E1
:10A2F000C2F11F02404606F03AFCE17911B148462E
:10A3000006F035FC083406F0D2FCA742E3D106F093
:10A31000CEFC7D4806F000FF7C4CDFF82482DFF89D
:10A320002492DFF824A2237E0136324601214046E2
:10A3300055F8237006F01BFC627E39463AB1504650
:10A3400006F0CCFC072E04F11C04ECD1ADE7484626
:10A3500006F0C4FCF6E7384607AA6D490DF0D8F9B7
:10A3600005F1B80782460026B84617F8363022466F
:10A3700055F8231050464FEAC6090FF009FE30B1D8
:10A3800001360D2EF1D1634806F0C6FE8DE707AA0F
:10A390005F490DF0BDF904460DF05EF94D4495F8A6
:10A3A000BE200746EAB9002828DCC844B8F80200F5
:10A3B00005F0A4FAFBB20193019AB8F804302778AB
:10A3C0001344029343680393002F00F09280524994
:10A3D00020460FF0A2FDD8B9039B029A98544F482B
:10A3E000D2E7002805DD1346BB4209DA002A08BF80
:10A3F000012201214A4806F07EFC56E70123F3E7DB
:10A4000007AA434900200DF083F9013F0446CCE739
:10A41000A7F14105EDB2072D04D9A7F16105EDB211
:10A42000072D66D8601C0DF017F9C3B20F2B8246BA
:10A430005FD86C1C40EA0414E4B2204608F038FCF3
:10A44000002856D0002C49D04FF000082309403393
:10A450000493DFF8F89004F00F03059300272FE032
:10A46000B9F8020005F04AFAB9F8043042683B44F2
:10A47000D15CA14223D1464504D101998F421ED01F
:10A480000021D154059A0499264806F070FB5FFA22
:10A4900087FB5FFA88F3594618460093FFF7FEFCE6
:10A4A000464509D1204806F062FB00985946FFF75F
:10A4B000F5FC1E4806F05BFB1D4806F02DFE01373B
:10A4C00099F80630002B08BF01239F42C8DB08F132
:10A4D0000108B8F10D0F09F10809BFD15FFA8AF23E
:10A4E00005F14101134806F0F9FB039B029A9C54C5
:10A4F000DBE606F017FED8E648C5010824A60108E9
:10A500004DC50108842000205BC50108140300200C
:10A510006CCC010879C501082DC5010887C5010863
:10A5200081C501088DC50108B1C50108B4C5010880
:10A53000CCCB0108BEC5010850C5010829D90108C6
:10A5400060C5010884CB010872C50108DCA60108BA
:10A550002DE9F84304460BF08DFD054620B1012896
:10A560001ED123782A2B1BD1104806F0D5FD0024DC
:10A570004FF00D09DFF83C800D4F09FB048638468B
:10A58000316806F0F4FA291C18BF01213046013465
:10A5900006F082FB06F08BFBAA2CEED1BDE8F88317
:10A5A0002046BDE8F84304F051BE00BFCAC501080B
:10A5B00062D90108D8AF01082DE9F84F0024804680
:10A5C00025464FF00D0ADFF85090DFF850B00AFB37
:10A5D00004963768414638460FF028FD78B1394671
:10A5E000584606F0C4FA0021304606F055FB06F046
:10A5F0005EFB304606F086FB06F059FB0135013460
:10A60000AA2CE4D125B9BDE8F84F024806F084BD74
:10A61000BDE8F88FDDC50108D8AF010862D901088F
:10A620002DE9F04F0D468DB0C149044601F0F8FB0D
:10A630000646002840F02682BE49204601F0F0FB85
:10A640000646002840F02082BB49204601F0E8FB86
:10A650000646002840F01A822046B84901F0E0FB87
:10A660000028064612BF0824264601240DB144F0F6
:10A670001004B34DB34FBD42C0F00A820123B24D66
:10A6800085F86A3002F0AEF9B049304601F0C8FBF7
:10A6900008B144F0200414F0090F00F0DB81002021
:10A6A000FFF7DEFB04F01803182B04D1A74806F0CF
:10A6B00087FA06F0FCFA95F87831A54A002B0CBF12
:10A6C00001210021A34B204618BF1346A24A06F0E1
:10A6D000DDFB2046FFF76EFDDFF8E4829F4B98F824
:10A6E00000601B789E4FA6EB0309D9F1000646EBEC
:10A6F000090607EB83033146D3F82C31994A2046EB
:10A7000006F0AEFB98F80030314607EB8307D7F828
:10A710002C31944A204606F0B9FB0021D5F88C0173
:10A720004FF001060CF0FEFB00B9064606F00101F1
:10A730008D4A204606F0AAFB8C4A204602F1800191
:10A740008B4E03F03DFC8B4A8B49204603F0C6F844
:10A7500096F902104FF00009B1FA81F1874A4909D0
:10A76000204606F093FB32468549204601F076FBF1
:10A77000DFF850B2D5F88C72D5F89082814B53F83F
:10A780002960002E40F08B81B14668EA0703DFF8AC
:10A7900038B203937B4B53F82960002E40F0A08120
:10A7A000D5F89432DFF824920393039AD5F89C32BB
:10A7B000DFF81CA25340DB4305930127059A07FAF3
:10A7C00006F31A42039A14BFB8464FF0000813402C
:10A7D00004934FF00C036C4A414603FB0623D3F865
:10A7E00008B014BF4A4652465B46204606F038FB86
:10A7F000049A5B46002A14BF52464A464146204608
:10A800003E4406F043FB132ED7D100235F4EDFF802
:10A81000C4E1DFF8C4C19A5D13F80E100CA810440F
:10A8200000F8181C13F80C000DF13008804408F8EB
:10A830000C1C2FB1A2EB0008D8F1000747EB08076A
:10A840000133082BE7D1002609AB514A394620468F
:10A850008DF8206006F004FB06AB4D4A39462046D1
:10A8600006F014FB4B4A4C49204606F021FB4B4AAC
:10A870004B49204603F014FA4A4A4B49204603F05C
:10A880007BF9464A4649204603F0BEF8474A20462F
:10A8900002F1500106F080FB454A204602F15A01C0
:10A8A00003F0CCFC434A4449204603F0F3FA4FF04E
:10A8B0000108DFF828A1DFF828B1730003931AF824
:10A8C00016201BF816309A4240F0318118F80A70B1
:10A8D00018F80B10781A47424741022ADFF8809097
:10A8E00040F0278119211BF808204B444A4393F874
:10A8F000143302F2EE2201920093304A3346394675
:10A90000204606F0ADFA192218F80A3039465343AA
:10A9100003F2EE230193730013F80A30274A994497
:10A9200099F8143320460093334606F0AFFA59E005
:10A9300001C60108CAD00108BEBF010808C6010847
:10A9400070E00108F4E30108182000200CC601089B
:10A9500090210020EAC5010815C601083119002020
:10A9600024A601081DC6010826C60108A42100204E
:10A970007D2E0020F02E00203835002035C601083D
:10A9800098350020C0A701083CA8010868190020DC
:10A9900059C601080E400020A8400020B019002030
:10A9A000241F0020301A0020A41F0020BC220020F9
:10A9B0005C230020DE380020CE38002060C601086D
:10A9C0009419002042C601084EC60108ECC50108D2
:10A9D000F6C50108FABA010834190020EE38002043
:10A9E000A13800200136122E08F102087FF465AF6D
:10A9F0002146002006F0C4F9210740F1B28021462B
:10AA0000002095F8746101F0F7F92146012001F06A
:10AA1000F3F92146022001F0EFF9304601F0D4FCB1
:10AA2000594800F013FE2146002095F8756101F0A9
:10AA3000CFF92146012001F0CBF92146022001F097
:10AA4000C7F930460BF002FB4F4800F0DFFD4F48DE
:10AA500006F0B6F8A20704D5214695F8740101F076
:10AA6000CBF9630704D5214695F8750101F0B0F9DB
:10AA7000474C484B9C427FD3002385F86A300DB089
:10AA8000BDE8F08F0124F1E50224EFE50424EDE5B3
:10AA90006A886968A8680CF007FE1435EBE533781E
:10AAA000DBB14FF0010A68EA07030AFA09FA13EA70
:10AAB0000A0F14BF0121002133465A46204606F0F2
:10AAC000CFF967EA080313EA0A0F5A46334614BF60
:10AAD00001210021204606F0D9F909F101094DE6CE
:10AAE00033780BB34FF0010A0AFA09FA18EA0A0F91
:10AAF0000BD067EA080313EA0A0F5A46334614BF1D
:10AB000001210021204606F0ABF917EA0A0F0BD00D
:10AB1000039B5A4613EA0A0F18BF0121334608BFA8
:10AB20000021204606F0B2F909F1010932E60027BA
:10AB3000D3E64B4493F8143339460093164A334610
:10AB4000204606F08DF9154B72009B5C39469944FE
:10AB500099F81433104A00932046334606F096F9CC
:10AB600040E7214695F8740101F046F9214695F831
:10AB7000750101F02DF96DE76288A16860680CF03D
:10AB800093FD143475E700BF14DB01087DC601088E
:10AB900070E00108F4E3010870C60108EE380020F7
:10ABA000426A806A131A584258417047417170478F
:10ABB00043799B070AD5436A8269D154436A016984
:10ABC0000133B3FBF1F201FB123343627047437967
:10ABD00013F0020308D00369426A806A013B101A2D
:10ABE0001840C0B2181A704718467047437913F0DE
:10ABF00001031FBFC369026AC0689B1A1ABF00F134
:10AC0000FF3018401846704710B54379014613F0DD
:10AC100001030ED0FFF7EAFF60B10B6A4A69CC6806
:10AC2000D05C0133B3FBF4F204FB1233C0B20B620D
:10AC300010BD184610BD90F8433230B53BB9012421
:10AC400090F8411290F84232DAB2914200D830BD09
:10AC5000B0F84A5204FA03F22A43A0F84A22013318
:10AC6000F2E7836B19685A79012393400A8C9BB2EF
:10AC700092B222EA03020A840A8C92B213430B8432
:10AC8000704710F80A3C0133DBB20A2B00F80A3C8B
:10AC900007D9002310F8131C024A22F8113000F8DB
:10ACA0000A3C7047E037002070B51424454B1A78F1
:10ACB0000132B2FBF4F004FB102298681A705A6C4F
:10ACC0008142DC680A4404D293F84C0008B102F5D2
:10ACD00080323D480678B2FBF6F2944223D293F8D4
:10ACE0004C501DB14FF4803595FBF6F5101B451BFC
:10ACF0001D61DA6040F68C2200209960196983F8A2
:10AD00004C00914241D9187993F94920904230D1B1
:10AD1000021F082A2DD893F84A20182A0BD801328E
:10AD200083F84A2009E04FF4803090FBF6F0001BD6
:10AD300010441861DDE783F8480093F948209042F9
:10AD40000FD193F84B1061B10021204C204D91425E
:10AD500011DB00241E490B2A13DD1E490A7801323B
:10AD60000A70012283F84B20002283F849001A71EF
:10AD700070BD0022D4E754F8046F25F8116001314A
:10AD8000E5E721F812400132E5E793F84B20C2B124
:10AD900040F2DA52A1F2EF20904207D81A790B2A3A
:10ADA00004D803EB820041610132E0E7002283F81E
:10ADB0004B20114613460848C2180433302B11614A
:10ADC000FAD170BD58240020D80300206824002048
:10ADD000E0370020D93700205C24002010B514246F
:10ADE000094B1A780132B2FBF4F004FB10221A70FE
:10ADF0005A6C01320A445A644FF6FF72914204BF02
:10AE0000012283F84C2010BD582400207047704761
:10AE100038B5A0F517746379A579DB0744D594F8A4
:10AE200040321BB3A06B0268938DC3F34E0393842F
:10AE300094F85132012B07D094F8453223B1B4F87D
:10AE40004C320133A4F84C32E94301F0010109F01E
:10AE50002FFD012384F84332002384F8413284F823
:10AE6000423284F84032A4F84A3238BD94F8433272
:10AE70002046012B04BF94F8413284F84232FFF798
:10AE8000DAFE94F843324BB90123E94384F84332A4
:10AE90001940A06BBDE8384009F00ABD002305F059
:10AEA000010184F84332F4E738BD10B583790446D4
:10AEB000DB07006B4CBF2A214A2107F01FFF01234B
:10AEC00084F8443284F840320023204684F841322A
:10AED000BDE81040C5E6084B10B41A681346B3FB32
:10AEE000F1F4B4F5803F03D3012BFAD95B08F6E700
:10AEF000A1B210BC07F038BD100300208160806B48
:10AF0000E9E78379406BDB0744BFB1FA81F1490976
:10AF100009B107F01ABF07F013BF10B5A0F51574FB
:10AF200063799A0714D594F84522002A59D1A36A67
:10AF3000616A994221D194F844324BB9A3791B0735
:10AF400006D5606B062107F0D9FE2046FFF7ADFF5E
:10AF50006379D90740F1998094F84032002B40F092
:10AF6000948094F841320133DBB2092B84F84132EA
:10AF70004DD12046BDE810405DE6591CA069A16294
:10AF8000C35C2069DBB25B0043F40073A4F8483271
:10AF90000A2381424FF0010184F8463294F844328A
:10AFA00028BFA26284F84512002BD1D0A3791807DC
:10AFB000CED5A06B02684079138C81409BB223EA06
:10AFC00001031384138C206B9BB21384062107F0BA
:10AFD00095FE0023122184F84432606B07F08EFE48
:10AFE000B6E794F946327BB1B4F8481220464B08D4
:10AFF000A4F8483201F00101FFF783FF94F84632CC
:10B00000013B84F84632A3E784F84532A0E70A2BD7
:10B010003BD194F843322BB9B4F84A3243F00103E0
:10B02000A4F84A32B4F84A02820501D4C3071AD4FC
:10B03000B4F84E320133A4F84E320122002384F8D2
:10B04000402294F8432284F84132012A1DD1A1798B
:10B05000A06B84F8433201F0010109F029FC20467D
:10B06000BDE81040FDE5E36AC0F347000BB1984727
:10B07000E3E7E3696269D054E369E1680133B3FB54
:10B08000F1F201FB1233E361D7E710BD182370B56D
:10B090000E465843074A14181558A16830460BF05D
:10B0A000ADFDE1680BF0A2FC0CF064FC80B22880DE
:10B0B00070BD00BF502B00202DE9F0471825502609
:10B0C0004FF028084FF00009144C154F05FB0045C0
:10B0D000A54201D1BDE8F087237CCBB1D4F804A010
:10B0E000504607F079FCEFF3128386F31288BAF822
:10B0F000242008FB007092B201324267BAF8142093
:10B10000DBB292B242F00102AAF8142083F3118854
:10B1100054F8183BA3F80090DAE700BF502B00204A
:10B120005824002008B50A4A1378D9070FD523F010
:10B1300001031370074B9B780BB1FEF775F80020E5
:10B1400007F012FEBDE8084004200AF033BE08BD37
:10B15000301B00208C41002038B5304B1B78D907BC
:10B1600005D5BDE838400121002007F029BE1B208D
:10B1700006F018F92A4C002836D004200AF0ECFE1C
:10B1800006F024F9002834D008200AF0E5FE254B0B
:10B190001B781A0732D410200AF0DEFE224B1B88DF
:10B1A000642B30D920200AF0D7FE204DB5F8F030BE
:10B1B0001BB11F4B1B689B0703D41E4BB3F8A83071
:10B1C00033B340200AF0C8FE238803B1022385F878
:10B1D000F23007F071FCD5F8F430C01A00281CDBFF
:10B1E000BDE83840FDF7ECB8238823F00403238042
:10B1F000C6E7238823F008032380C8E7238823F0C9
:10B2000010032380CAE7238823F020032380CCE7A0
:10B21000238823F040032380D6E738BD301B00206D
:10B22000881B0020C4160020802000205824002005
:10B2300060190020A83A002070B5314C23783BB14A
:10B24000304D2B7823B9304805F0D0FA01232B700C
:10B25000FFF782FF2D4B1A8802BB2D4A137813F09B
:10B2600001014BD10A2043F003031370294A2A4BF2
:10B27000B2F90420C3F8001192FBF0F2A3F8F82011
:10B28000264A1068A2784FF47A7404FB0202052063
:10B29000C3F8FC20BDE870400AF08CBD194B1B7848
:10B2A0001BB11F4BB3F8A83043BB92FAA2F3002A9C
:10B2B000B3FA83F308BF4FF0FF33174A0133D2F8D4
:10B2C00000118B421AD0C2F80031DBB29B00402B38
:10B2D000A8BF4023002214260A200525114954182E
:10B2E000565404326070A5709A4202EB010404F8CF
:10B2F000010CF4D3FF230F208B54CBE770BD00BFAC
:10B300001612002020120020503B0020881B002035
:10B31000301B002018330020582400204C3A002015
:10B32000A83A0020102400202DE9F04F4FF41874A3
:10B3300089B098469DF84830814E039300F10A0386
:10B34000334493F8D0B593F8C435059144430021B4
:10B35000054658460292019301F062FC00210790D5
:10B36000019801F05DFC8146584607F0A1FC06906B
:10B37000019807F09DFC039B06F5827713F0080304
:10B38000049307EB040A069A079B00F09B80B9F12F
:10B39000000F03D1002009B0BDE8F08F3319C3F8C6
:10B3A0003C91C3F83801C3F8340105F10B03DBB25B
:10B3B00010B10B22C37182714FF418794FF0000B5A
:10B3C0004FF4807209FB05695E4BC9F81021C9F87A
:10B3D0000431029BC9F81421C9F80C319DF80C30D6
:10B3E000029989F80A31059BD9F83C01C9F8303136
:10B3F00004F140033B44C9F8183104F5A0733B4401
:10B40000C9F81C3189F80981C9F824B1C9F820B1FB
:10B41000C9F82CB1C9F828B189F85453A9F850B328
:10B42000A9F852B389F848B389F849B3FFF753FD37
:10B43000039BD9F83C0103F0010109F039FA424AB3
:10B4400004F51773C9F86023404A04F5157418F021
:10B45000020F3B44C9F858232744C9F85CB362D0B3
:10B46000D9F8400100285ED0D9F83C11026809687B
:10B470008A4258D00122029989F855230193FFF797
:10B480002AFD3A465946D9F8400107F0C1FA019B16
:10B490005A461946D9F83C0107F0BAFA049B63B939
:10B4A0004FF4187303FB05651221D5F8380107F036
:10B4B00025FC01215046FFF724FD5046FFF7F5FC1F
:10B4C000504668E718F0010E12D0BBF1000F3FF4B0
:10B4D00061AF002B3FF45EAF3119C1F83C3105F18B
:10B4E0000B03C1F83421DBB212B10C21D37191717D
:10B4F00018F0020F3FF460AF019B002B3FF44AAFFE
:10B500004FF4187303FB0563C3F83801BEF1000F55
:10B5100006D1B9F1000F3FF43DAFC3F83C9144E7C9
:10B52000C3F8409141E74FF41870002200FB05601A
:10B53000194680F855233A46D0F83C01ACE700BFE5
:10B5400058240020A8A9010811AE00081BAF00086C
:10B550001FB50123ADF808300023ADF80C30ADF86D
:10B560000A30094BADF8041093F8E83501A9012B16
:10B5700008BF0323ADF8062008BFADF80C3001F07A
:10B5800072FD05B05DF804FB5824002038B510F8B2
:10B590000E2C044650F8043C52B9012220F80C1C31
:10B5A00000F80E2C597918680222BDE83840CFE720
:10B5B000002530F80C2C20F80A1C891A89B220F8D2
:10B5C000081C074A10F80F0C22F8101004F80E5C43
:10B5D0002A4659791868FFF7BBFF04F8065C38BDA6
:10B5E000E03700201823064A10B503FB0020D0F8EE
:10B5F000EC4524B108460CF0BDF980B2208010BDA6
:10B6000058240020072800D8ECE7704738B50446D6
:10B610000B4D204605F051FA30B10A4B0A485978D3
:10B62000BDE8384005F05ABB20460CF015F802285A
:10B6300004D8C0B20AF00AFD2C46EAE738BD00BFC4
:10B6400014DB010858200020E1CA010870B5044647
:10B650000A4E0B4D204605F030FA30B1074B094831
:10B660001978BDE8704005F039BB20460BF0F4FFB7
:10B67000022802D830702C46ECE770BD582000201C
:10B6800014DB0108E5CA01082DE9F743074605F078
:10B6900014FA044620B105F045FD03B0BDE8F0837F
:10B6A000384601AA2E490CF033F82E4FDFF8CC8033
:10B6B000DFF8CC9070B9022CEDD1A6F57A73B3F512
:10B6C0007A7F2DD94FF4FA624FF47A71264805F04B
:10B6D00012FBE2E744B1012C1ED001AA2049002050
:10B6E00001340CF015F8E5E70BF0B6FF051E0DDB95
:10B6F0003B789D4204DA2946484604F0D1FAECE74B
:10B70000FF2D03D1404604F0CBFAE6E7397817481D
:10B71000013904F0C5FAC0E70BF09EFF0646DCE7EE
:10B72000FF2D0AD104460F4B114F1D78AC4210DBA0
:10B730003146104805F0D2FAAFE730460BF006FA72
:10B740000B4B324643F8250029460B4805F0C6FA54
:10B75000A3E730460BF0FAF947F824000134E5E797
:10B760006CCC010844170020C5CD010818CB010896
:10B77000282B00204ECB010841CB010803CB010848
:10B78000F0CA01082DE9F0470546204FDFF8848014
:10B79000DFF87C90DFF894A028460AF06BFC0646A0
:10B7A00050B91B4B1B4A1B781B48013B52F8231016
:10B7B000BDE8F04705F092BA0246394628460EF039
:10B7C000E7FB40B1002458F82410A1B91348BDE8A4
:10B7D000F04705F0A1BC124805F0F2F9114C124DEA
:10B7E00054F8041F19B1284605F0C1F9F8E7BDE87F
:10B7F000F04705F05CBA324628460EF0C9FB01342A
:10B800000028E0D189F800405546C5E748C5010841
:10B810003119002054A701085DCB0108DDC50108DE
:10B8200067CB010850A7010884CB010814DB01088D
:10B830002DE9F74F82460AF01DFC474D04462F685C
:10B84000E8B9464805F093F90125454EDFF8348103
:10B8500005FA04F33B4206D00C2303FB0463404685
:10B86000996805F084F90134132CF1D117B93D48DA
:10B8700005F0A6F903B0BDE8F04F05F018BA02468E
:10B88000394950460EF084FBDFF8D490064668B97B
:10B89000364805F095F9364D09EB060399682846B8
:10B8A0000C3605F064F9FC2EF6D1E3E79AF8003087
:10B8B0004FF000082D2B0CBF4FF0010B4FF0000B89
:10B8C0004FF00C0304BF0AF1010A04F1FF3403FB3B
:10B8D0000892966850462246314601930EF058FB76
:10B8E000019B70BBBBF1000F19D0B8F1130F0BD146
:10B8F000204B2B60204805F063F931461C4803B00B
:10B90000BDE8F04F05F0EAB9B8F1140F01D16B684A
:10B91000EFE7012303FA08F31F432F60EAE7B8F1CA
:10B92000130F03D1C5F800B01448E4E7B8F1140FC1
:10B930001DBF012303FA08F39F436F6018BF2F60F8
:10B94000F2E708F10108B8F1150FC0D10C4803B0B7
:10B95000BDE8F04F05F0E0BBB422002072CB010837
:10B960003CA801087CCB010848C5010867CB010849
:10B9700084CB0108FFFF070088CB010891CB0108A9
:10B98000DDC5010883CB010870B5134C054613488B
:10B9900005F016F9206A03F0F9FE606AFCF72EFD47
:10B9A0000F4B1820197800231E4628348B420BDBDE
:10B9B00040F2DC5007F0C8F80A4B0B4A15B10B48AF
:10B9C0000B490860DA6070BD00FB03F2125902B146
:10B9D00016800133EAE700BF282B002099CB01082D
:10B9E0004417002000ED00E00400FA05EFBEADDED4
:10B9F000F04F002010B50C4C206A03F0C7FE002366
:10BA0000D4F8702184F8E830C4F8683184F86C31D7
:10BA100044F823200133082BFAD10020FFF7B4FFAC
:10BA20000023236210BD00BF282B002008B500F0C2
:10BA3000D9FF00F0DFFCBDE808400020A4E708B50E
:10BA400000F0D8FCBDE8084000209DE701209BE7FE
:10BA50002DE9FF4107460AF00DFB08284AD10025D1
:10BA600001AE7C5D0BF000FE2044437803F003033D
:10BA7000022B08BF203CAC550135082DF1D1002523
:10BA8000DFF87C808DF80C507C5D0BF0EDFD2044E0
:10BA90004378404603F00303022B08BF203C745553
:10BAA000E4B221460EF066FA28B10135214670193C
:10BAB0000EF060FA20B105F035FB04B0BDE8F0816E
:10BAC000082DE1D10D49304604F034FF00230B4C22
:10BAD0000B481A5D04A90A44195C0133082B02F8CB
:10BAE0000C1CF6D1002301A906488DF80C3005F096
:10BAF000F5F8E2E70028E9D0DDE700BF34190020BF
:10BB0000FABA010859C601082DE9F84F05460AF0AE
:10BB1000B1FA364F0446D7F80090B0B9344805F072
:10BB20004FF80126334D344F55F8241049B106FA29
:10BB300004F313EA090F02D0384605F018F801346F
:10BB4000F2E7BDE8F84F05F0B2B802462B492846A7
:10BB50000EF01EFA78B92A4805F032F8294C2A4D21
:10BB600054F8041F0029ECD00B78002BF8D028469D
:10BB700004F0FDFFF4E72B7800262D2B0CBF4FF0CF
:10BB8000010A4FF0000ADFF86CB004BF013504F180
:10BB9000FF345BF82680B8F1000F04D11B48BDE8E4
:10BBA000F84F05F0B9BA2246414628460EF0F0F9A2
:10BBB000D0B90120B040020601D51548EFE7830552
:10BBC000FBD4BAF1000F0AD003F0AAFE114804F02A
:10BBD000F7FF4146BDE8F84F0B4805F07FB840EA53
:10BBE000090038600C48F2E70136D2E7A8220020AD
:10BBF000A5CB0108C0A70108AFCB010848C50108C3
:10BC000067CB0108BCA7010884CB0108DDC501088A
:10BC1000B3CB010888CB010891CB010870B505466C
:10BC20000AF028FA044690B1112200210F480EF0C4
:10BC30006CF922460E4928460EF0D1F938B1102C85
:10BC40002246294628BF102208480EF0DAF9BDE83E
:10BC50007040084B012013F8042F002A044A06BF45
:10BC6000012113460021044A05F010B95C20002090
:10BC7000EAC501085820002015C6010808B50D487E
:10BC800005F04AFA0C4B186A03F080FD06F048FDF7
:10BC900006F02AFC48B113200AF08CF805F007F8EA
:10BCA000BDE80840054805F037BA642006F057FFA4
:10BCB000EEE700BFBFCB0108282B0020C8CB01084E
:10BCC0002DE9FF410A480488856846888788D0F8AE
:10BCD0000C8006F0E9FB8DE88001029033462A468D
:10BCE0002146044804F0FAFF04B0BDE8F08100BF2B
:10BCF0007C040020CECB0108F0B585B0054604F0E9
:10BD0000DCFE002838D104462B78002B3CD1062CD1
:10BD100042D1BDF904309AB2072A3DD840F2DC5432
:10BD2000BDF90610A1F2EE2292B2A24234D8BDF9BA
:10BD30000820A2F2EE2080B2A0422DD8BDF90A0060
:10BD4000814229DC824227DB914225DCBDF90C507F
:10BD500005F16404A4B2C82C1ED8BDF90E40112C04
:10BD60001ADC0C27194E07FB03639980DA801881CF
:10BD70009D72DC7205B0F0BD00220120134905B0B0
:10BD8000BDE8F04001F0AABD2D2B03D0A3F1300295
:10BD9000092A16D8052C04DD05B0BDE8F04005F0F1
:10BDA000C1B928460BF058FC04AB661C03EB4404F5
:10BDB00024F80C0C15F8013F303B092BFAD9344616
:10BDC000A2E7202BE8D101352646F8E7F02E002027
:10BDD000022810B50C460CD80AF038F90548FFF7D0
:10BDE00015FC04F064FF2146BDE81040082004F073
:10BDF000C7BF10BD14DB0108022810B50C460CD8D3
:10BE000000F0E2FA0548FFF721FC04F050FF21465C
:10BE1000BDE81040042004F0B3BF10BD14DB0108DE
:10BE200070B5044608460E460AF024F9314602462B
:10BE300020460EF0ADF808B1002070BD0BF014FCE8
:10BE4000054630460AF016F9235C1D446A7812074D
:10BE500001D4002BF0D10130204470BD2DE9F04F0A
:10BE6000824691460E46154600278FB0337896F9E4
:10BE70000280089373780993F3780A9396F9043053
:10BE80000B9396F905300C93B3790D93B8F1000F2D
:10BE900004D10FB0BDE8F04F04F009BFB9F1000FB5
:10BEA0004CD02B78089C6A789C4295F90210E8786F
:10BEB00095F904E095F905C095F806B03CD1099CC8
:10BEC000944239D1884537D10A9C844234D10B9CA5
:10BED000744531D10C9C64452ED10D9C5C4514BF3A
:10BEE000002401240390029101920093CDF818B030
:10BEF000CDF814C0CDF810E03B46114A214650461B
:10BF000004F0AEFF0D9BCDF8088006930C9B0C4A05
:10BF100005930B9B214604930A9B50460393099B70
:10BF200007360193089B073500933B46013704F021
:10BF3000ADFF102F9AD1ACE70024D3E74C46E1E7E0
:10BF400029CC01082DE9F0478AB005460AF092F89D
:10BF5000024630B995490120FFF780FF0AB0BDE8DD
:10BF6000F0870522924928460EF012F8044660B97F
:10BF7000702201468D480DF0C8FF204622468D4BA9
:10BF8000C2500C306028FBD1E8E704228A492846D9
:10BF90000DF0FEFF0446002841D1284604F095FD2F
:10BFA00006460028DAD00AF065F80746DFF8308246
:10BFB00058F824501DB9814805F0AEF8CEE73A464E
:10BFC000294630460DF0E4FF01340028F0D1774BCC
:10BFD0000246194603F170069A719A705A7003F876
:10BFE000072BB342F8D1764B13F8347003EBC4043B
:10BFF000B84205DB2946734804F070FE724886E0BB
:10C000006368C0EBC0021344D3F800E08E1841F817
:10C0100002E09A880130B2809B79B371E8E7072289
:10C020006A4928460DF0B4FF0446002875D1202146
:10C0300028460DF09FFF06460AF01CF8054680BB17
:10C04000634804F094FD2C46624D21462846013495
:10C0500004F08DFD0E2CF8D104F029FE0024DFF849
:10C060008491544FDFF880810C262146484604F025
:10C070007EFD002506FB0476DFF870A101233268FF
:10C08000AB40134214BF414651465348013504F0BA
:10C090006EFD0E2DF2D1013404F009FE082CE3D11F
:10C0A0005CE7304601AA4D490BF032FB4B4E02AD26
:10C0B00000283DD0022C15D1029A072A2AD80399CC
:10C0C0000D2927D80378722B17D06E2B22D10C2381
:10C0D00053430122374802FA01F1C25822EA010211
:10C0E000C25013E00BF0B8FA01AA45F8240031461B
:10C0F00000200BF00DFB0134DAE70C230120534341
:10C100002C4C00FA01F1E0580843E0502F48FFF7AB
:10C1100019FF23E705F006F8F8E7284601AA2F499A
:10C120000BF0F6FA00242D4E02AD78B1082C02D1A6
:10C1300004F0F8FF12E70BF08FFA01AA45F824008B
:10C14000314600200BF0E4FA0134EEE7082CEFD181
:10C15000029B0F2BECD8DDF80CC0BCF1070FE7D821
:10C16000049F0D2FE4D8059E06F16402C82ADFD88B
:10C17000069DFF2DDCD807986428D9D80899642932
:10C18000D6D88842D4DA099C032CD1D8DFF81CE039
:10C19000C3EBC3020EEB02030EF802C05F709E7089
:10C1A000DD70187159719C7128E700BF7D2E002049
:10C1B00046CC0108F02E00204CCC0108DDC501085A
:10C1C000D0A9010851CC010814DB01085BCC01089F
:10C1D00086CB010863CC010868CC01086CCC01084F
:10C1E00054A701082AD901083DCD01086FC00108F4
:10C1F00003680A7A591C01601A70704738B5054601
:10C20000064C206800B938BD4368EB1A002BFADBF6
:10C210008368236003689847F3E700BF2438002051
:10C2200000231A4630B5084C037219198D79AD07F1
:10C2300042BF097981540132B02B03D0072A03F1A0
:10C240001003F2DD30BD00BF38A50108002210B593
:10C25000064C04EB02118B7913F0010302D00B7929
:10C26000037010BD01320C2AF3D1F9E738A501089B
:10C270000123102203704270037121228370202356
:10C280004271C370704738B54D680446284609F0BE
:10C29000F1FE29460246204603F0DAFC23685A1CC8
:10C2A00022603B221A7038BD08B50B4B1820197854
:10C2B00000231D46094C8B4207DB40F2DC5006F0A0
:10C2C00043FC074A074BDA60FEE700FB03F2125912
:10C2D00002B115800133EEE744170020502B0020F7
:10C2E0000400FA0500ED00E030B500220C250749F6
:10C2F00005FB02F46318645C844201D1184630BD2A
:10C300000132242AF4D1002030BD00BF10BB010847
:10C310002DE9F84F00248046914625464E01DFF86E
:10C3200034A006F12007214650465FFA84FB06F050
:10C330007AF850B1AE4207D8AF4205D95846FFF758
:10C34000D3FF01464046C84701350134242CEAD1C9
:10C35000BDE8F88F940D002080B50121022006F081
:10C360002FFD144B1B7803F00503052B12D1124B44
:10C37000002418680AF01EFE104B114F1D7806B2FB
:10C38000AC4210DB0F4B1B780BB102F023FB3220C9
:10C3900006F0E5FB0021012006F012FD0021084611
:10C3A00006F00EFDFEE730460AF0D4FB47F8240005
:10C3B0000134E5E72C0B0020982C002044170020C6
:10C3C000481700203A3A0020022828BF0220064BD6
:10C3D000064A18704A2303FB0023054A0130C0B205
:10C3E000136009F083BD00BF5820002036340020C0
:10C3F0002C1900202DE9F04F8DB004F013FB03261B
:10C40000DFF85C914F4FA7EB0907182200210DEBD5
:10C4100002000DF07AFD4C4B4C4ACDF8189007976E
:10C420005A6002F188325A6001228DF82C203422A1
:10C43000DA60474B04A918689A889B790490ADF894
:10C44000142006A807228DF8163003F019FA0722E7
:10C4500004A94FF6FF7005F05DFE4FF0000A80461C
:10C460003C4CDFF800B15C4536D300250CAC24F819
:10C470002C5D0222214606A803F002FA0222214680
:10C48000404605F047FE40BAC0430222ADF808001E
:10C4900002A906A803F0F4F9099860B108ABC0F14D
:10C4A0000402294618440DF030FD089906A803F04F
:10C4B00079F909950A909DF82C300A9A23B12249FE
:10C4C0000B6943F080030B61013E2DD0002A9CD103
:10C4D00003F02EFA50B330E0658806A8C5F30B05CB
:10C4E000AA1DADF8082022888DF80DA0C2F30B011B
:10C4F000120BADF80A108DF80C2002A9062203F0E9
:10C50000BFF9062202A9404605F004FE8046616894
:10C510002A4606A803F0B4F9616840462A4605F0A9
:10C52000F9FD143480469EE7002AD1D00A21052067
:10C5300006F084FC084A094BDA6004F05BFA0DB09F
:10C54000BDE8F08F0000020800200240230167458B
:10C550003CAB010870E001080400FA0500ED00E0C2
:10C5600000F80108F4E301082DE9F843344B354D98
:10C570005A899989914228BF0022198A28BF5A8175
:10C58000DA89914224BF0022DA81DA78002A50D079
:10C59000072A4ED001222A709A7000222A4CDA71A2
:10C5A000D9799A78002946D0102A38BF1022274C12
:10C5B0009A7098780AF0CEFA21460AF01FFB81465D
:10C5C00095F80080224C40460AF0C4FA49460AF029
:10C5D00015FBA6780146022E97BF1E4B1B4F03EB9F
:10C5E00086039F6838460AF0C5FC80B14946384644
:10C5F0000AF0B8FB0AF0DEFC1028A8BF10200128C2
:10C60000B8BF0120C0B2404528BF404628702379FA
:10C610006BB1013E032E0AD839464FF07E500AF026
:10C62000A1FB0BF0A7F92388984238BF2080BDE812
:10C63000F883094CB4E7032A38BF03229A70B8E79D
:10C64000963A0020BC3200206F12833A6F120338F2
:10C65000981700203CAB01086F1203392DE9F8430D
:10C6600004F0E0F9AD4CAE4FDFF84883BC422DD268
:10C67000AC4D00E015462E88002E00F09D81AA19D1
:10C68000424580F09981052E40F296812388698881
:10C69000C3F30B039942EDD16B799B07EAD1616833
:10C6A000204695F8049003F004F92388B9EB133F72
:10C6B0000AD16388B21FC3F30B039A42A8BF1A467C
:10C6C000A91D60680AF0F0FF1434CFE7964B5A7842
:10C6D000022A84BF00225A705A78022A05D80C20F8
:10C6E000924900FB021292490A601A78914E022A7E
:10C6F00084BF00221A701878022806D84A228E4B6E
:10C7000002FB0030306002F033F98C4A1178A1F15D
:10C710001703022B12D98A4BC80013F8314024B1F9
:10C720001C1864680CB91724147003445B782BB18F
:10C73000844B13F831300BB918231370824B9A785D
:10C74000042A40F0D2809A8AB2F57A7F02D24FF45E
:10C750007A729A827D4C7E4A23681A4012B943F05D
:10C76000010323602368DD0702D57A4803F0D8F877
:10C770002368580402D5784803F0D2F823681907D3
:10C7800002D5764803F0CCF823689A0103D546F227
:10C79000090003F0C5F823689B040FD5704803F027
:10C7A000BFF84FF4004003F0BBF86E4B40205A79BD
:10C7B000012A04BF00225A7103F0B2F83368002541
:10C7C0009A8CD98C684F914224BF00229A84FFF73B
:10C7D000CBFE2C46B9464FF0FF08EA5B530803F046
:10C7E0007733900800F03330D31A1B1AD00800F0CA
:10C7F00011301B1A03EB231303F00F3393FBF8F0F4
:10C8000012F00101C0EB002018BF0134A3EB0003BC
:10C8100018BFE4B2012B0DDD022B40F0D28011B124
:10C8200012F42F7F06D109EB050000F023FF00284A
:10C8300000F0C7800835282DCFD1013C022C00F232
:10C84000C08004F0FFFD3022002148480DF05DFB60
:10C85000002004F06DFD464B80F001003468187034
:10C86000444B454A1C60454B0024197864234B43D4
:10C87000C83353609460D460146154619461D4618E
:10C8800082F8204082F821403D493E4A3E4D0A60F0
:10C890003E4E32F8042C286B3280002830D13C4DBB
:10C8A0003C4B28881E880AF055F93B490AF0A6F946
:10C8B0003A4C606068880AF04DF937490AF09EF9F1
:10C8C0006B79374A23722B7920606372354B30467F
:10C8D0001A600AF03FF9014633480AF043FA334B35
:10C8E0001860BDE8F84304F085B8002A7FF432AF41
:10C8F0001A88B2F5F07F84BF4FF4F0721A8029E7EE
:10C900002B4F30880AF022F92A6B014638192C3453
:10C9100005F044FD842CF4D1C1E700BF70E00108AC
:10C92000F4E3010807F8010858200020D81100207E
:10C93000383900202C19002036340020311900200D
:10C9400070AB0108D0A9010898170020A822002088
:10C950000960000208600002092000020160000274
:10C9600009400002521B00200E40002084150020C8
:10C9700000000020B8150020641B00204433002074
:10C98000003A002024390020F81600200C0D002069
:10C990009C2C00205011002017B7D1380033002004
:10C9A0003661023D2C330020C0C9FB4854110020E1
:10C9B000100D0020000002086168204602F079FF97
:10C9C00082E6024809F09CF93BE700BF0E400020D8
:10C9D00008B5FFF70FFDFFF741FEBDE80840012055
:10C9E00009F084BA38B50D4C0D4DAC420FD300257B
:10C9F0000C4C0D4B0D482570186001F0B9FF0C4B25
:10CA00000C4A65701A60BDE83840FCF70BBF6168DE
:10CA1000204602F04EFF1434E7E700BF70E0010843
:10CA2000F4E30108582000202C190020363400209F
:10CA300038390020D811002070B50C2948D8DFE81B
:10CA400001F0074747474847474784474747BE00E5
:10CA5000038C158823F001031B041B0C0384038C37
:10CA60008488018B23F0020321F073010904090C6F
:10CA70002943568815891B0435431B0C2B43674DEE
:10CA8000A4B2A8429BB20FD005F50065A8420BD016
:10CA900005F54065A84207D005F58065A84203D09A
:10CAA00005F58065A8420ED1558923F008032B4374
:10CAB000958823F004032B43D689958924F4407488
:10CAC00035432C43A4B2D2888480018382860384B8
:10CAD00070BD038C148823F010031B041B0C03840B
:10CAE000038C8588018B23F0200321F4E64109049F
:10CAF000090C41EA0421568814891B0434431B0C99
:10CB000043EA0413454CADB2A04289B29BB203D0B4
:10CB100004F50064A04213D1548923F0800343EA52
:10CB200004134FF6BF741C409388D68944EA03135C
:10CB3000948925F44065344345EA84059BB2ADB23F
:10CB4000D288858001830287C1E7038C148823F48F
:10CB500080731B041B0C0384038C8588818B23F456
:10CB6000007321F073010904090C214356881489CC
:10CB70001B0434431B0C43EA0423284CADB2A042EF
:10CB80009BB203D004F50064A04213D1548923F46E
:10CB9000006343EA04234FF6FF341C409388D68990
:10CBA00044EA0323948925F44055344345EA0415A7
:10CBB0009BB2ADB2D28885808183828787E7038C60
:10CBC000158823F480531B041B0C0384038C848876
:10CBD000818B23F4005321F4E6410904090C41EA56
:10CBE0000521568815891B0435431B0C43EA053380
:10CBF0000A4DA4B2A84289B29BB203D005F50065E4
:10CC0000A84205D1958924F4804444EA8514A4B24D
:10CC1000D28884808183A0F8402058E7002C01400E
:10CC200030B598B10A4B00221C461D79854207D1C8
:10CC30009D79294202D004EB021030BD0029FAD0C0
:10CC400001320C2A03F11003EFD1002030BD00BFE8
:10CC500038A501080149024805F021BE2025002021
:10CC6000000800400149024805F019BEF8240020E0
:10CC70000004004002494FF0804005F010BE00BFA4
:10CC8000D02400200149024805F009BEA824002054
:10CC9000002C0140FFF7F6BF10B5204B18B9022257
:10CCA0001B681A8210BD00201D491C68088023786B
:10CCB0000A4613F07F0313D1637A990644BF022119
:10CCC000117013F0400F137814BF43F0010323F0E9
:10CCD00001031370134B1B681B699847104810BD64
:10CCE000012B18D0022B17D1617901F00F039B00A3
:10CCF00003F1804303F5B84311F0800F1B6805D0A2
:10CD000003F03003102BE5D10123E2E703F4405395
:10CD1000B3F5805FF7E7084610BD00BF443A002036
:10CD2000AC2C00206839002010B5064C18B901223F
:10CD300023681A8210BD044B1B689B6898472068C3
:10CD40000C3010BD443A00206839002010B5064C64
:10CD500018B9012223681A8210BD044B1B681B6896
:10CD6000984720680A3010BD443A002068390020F6
:10CD7000084BDA68D10709D4DA68520708D4DB68AF
:10CD800013F0100F14BF03200420704701207047D8
:10CD90000220704700200240A0F17D03012B70B5F6
:10CDA00004460D460A4E11D87D21706805F050FFEB
:10CDB00084F02001706805F04BFF35B128882044CD
:10CDC00000EB102000F0FF00288070BD0146F1E765
:10CDD000AC2C00205E2810B50146094C09D15D211C
:10CDE000A06805F035FF3E21A068BDE8104005F0C1
:10CDF0002FBF5D29A068F8D105F02AFF3D21F3E798
:10CE0000AC2C00200E4B0F4A1B683E299BB223F02E
:10CE1000070303EBC00002444FEA42020AD94B0960
:10CE2000C80604BF03F1FF339BB29B0243F40043E7
:10CE3000136070474B08C90748BF01339B02F7E7EF
:10CE4000505C004006300020054B1B689BB223F06D
:10CE5000070303EBC000034B03445B0019607047FA
:10CE6000505C004002300020002303604360836078
:10CE7000C360036143618361C36103624362836290
:10CE800070478B6810B50C6A026823430C6922F462
:10CE9000FF4223434C6922F0700223438C692343F1
:10CEA000CC6923434C6A23438C6A234313430360B6
:10CEB000CB6843600B6883604B68C36010BD036838
:10CEC00023F001031B041B0C036000230360436079
:10CED0008360C360284B984204D1284A536843F0CA
:10CEE0000F0326E0264B984204D1244A536843F0AE
:10CEF000F0031EE0234B984204D1204A536843F4C8
:10CF0000706316E0204B984204D11C4A536843F4E6
:10CF100070430EE01D4B984204D1184A536843F405
:10CF2000702306E01A4B984205D1144A536843F423
:10CF3000700353607047174B984204D10F4A5368EF
:10CF400043F07063F5E7144B984201D1134AC5E7EB
:10CF5000134B984201D1114AC8E7124B984201D1B4
:10CF60000E4ACBE7104B984201D10C4ACEE70F4B4B
:10CF70009842DFD1094AD1E7080002400000024090
:10CF80001C000240300002404400024058000240B1
:10CF90006C0002408000024008040240000402408D
:10CFA0001C04024030040240440402405804024081
:10CFB0001F4A10B5536803F00C03042B21D0082B33
:10CFC00022D01C4B036053681B49C3F30313CC5C92
:10CFD0000368E34043605468C4F302240C5D23FA01
:10CFE00004F484605468C4F3C2240C5DE340C3605D
:10CFF0005268C2F3813211440A7CB3FBF2F303613D
:10D0000010BD0E4B1B68DDE753685168C3F38343C3
:10D01000C90303F1020302D409494B43D2E7516823
:10D0200011F4003F0549096818BF4908F5E700BF3A
:10D030000010024000127A0050AB0108DC0300200F
:10D0400000093D0010B50446FFF792FE012806D105
:10D050000CB9052010BDFFF78BFE013CF6E7002C54
:10D0600008BF052010BD0B88F0B54E88B1F804E06C
:10D070000F89CC88002B3CD1038C23F001031B04C7
:10D080001B0C0384018B824B89B221F0F301058CC8
:10D090004EEA010141EA07119842ADB289B212D0BD
:10D0A00003F5006398420ED0B0F1804F0BD0A3F58A
:10D0B0009833984207D003F58063984203D003F574
:10D0C0008063984212D125F0020546EA050343F039
:10D0D000010301830384038B23F00C031B041B0C4B
:10D0E0000383038B9BB21C430483F0BD25F00A0528
:10D0F000EBE7042B44D1038C4FEA0E2E23F01003F0
:10D100001B041B0C0384038B4EEA073723F4407384
:10D110001B051B0D1F435E4B018C984289B2BFB2A9
:10D1200012D003F5006398420ED0B0F1804F0BD0BF
:10D13000A3F59833984207D003F58063984203D053
:10D1400003F58063984214D121F0200141F01003CF
:10D1500043EA06139BB207830384038B23F44063E3
:10D160001B041B0C0383038B9BB243EA0424A4B26D
:10D17000BAE721F0A00146EA010343F01003EAE711
:10D18000082B038C3FD123F480731B041B0C0384F6
:10D19000818B3F4B89B221F0F301028C4EEA0101F1
:10D1A00041EA0711984292B289B212D003F50063A6
:10D1B00098420ED0B0F1804F0BD0A3F5983398422F
:10D1C00007D003F58063984203D003F5806398424B
:10D1D00013D122F4007343F4807343EA06239BB215
:10D1E00081830384838B23F00C031B041B0C838338
:10D1F000838B9BB21C438483F0BD22F420633343B2
:10D2000043F48073ECE740F6FF4223F480531B04A1
:10D210001B0C0384818B038C0A40390341EA0E21E5
:10D2200011431B4A9BB290421FFA81FE12D002F5B5
:10D23000006290420ED0B0F1804F0BD0A2F5983230
:10D24000904207D002F58062904203D002F58062DE
:10D25000904215D123F4005343F4805343EA06333C
:10D260009BB2A0F81CE00384838B23F440631B046F
:10D270001B0C8383838B9BB243EA0424A4B2BAE7DA
:10D2800023F400735B045B0C334343F48053E8E7FF
:10D29000002C01400F4BDA684378D243C2F30222DC
:10D2A000C2F104018B400F2121FA02F281780A4079
:10D2B0001343094902781B018818DBB280F8003358
:10D2C0000123500902F01F0203FA02F241F8202064
:10D2D000704700BF00ED00E000E100E02DE9F04103
:10D2E000CB780E88DA0648BF8A7803F00F0548BF6E
:10D2F000154316F0FF0F1AD000214FF0010E4FF02A
:10D300000F0C02680EFA01F737EA06040BD18C0005
:10D310000CFA04F822EA080205FA04F4282B42EA7F
:10D32000040225D1476101310829EBD10260FF2EAB
:10D330001CD900214FF0010E4FF00F0C426801F193
:10D3400008040EFA04F434EA06070BD18F000CFA35
:10D3500007F822EA080205FA07F7282B42EA070233
:10D360000AD1446101310829E9D14260BDE8F08168
:10D37000482B08BF0761D6E7482B08BF0461F1E7D7
:10D380000F4B1A6842F001021A6059680D4A0A40B0
:10D390005A601A6822F0847222F480321A601A6885
:10D3A00022F480221A605A6822F4FE025A604FF476
:10D3B0001F029A604FF00062034B9A60704700BFF3
:10D3C000001002400000FFF800ED00E080F3088844
:10D3D00070474FF6F672074BDA8203F11C02DA60EF
:10D3E0000122998203F11D011877196183F81C212C
:10D3F000704700BFAC2C002037B51C4C94F81D01C1
:10D40000FCF7D6F994F81E310546834223D020B3A9
:10D41000D4F82021FAB194F82A3192F90200002BB5
:10D4200014BF0823002394F829212021002A08BFD3
:10D4300043F0010301930323002200934FF461435F
:10D44000FBF714F8606030B1012384F8323184F8BE
:10D450001E31074B1B6803B030BD6068FAF7D9FF77
:10D46000656084F8325184F81E51F4E7AC2C00203A
:10D470004C3A0020002373B502AD25F8023D0C465E
:10D480002946FFF789FCA61D14F8010B2946FFF772
:10D4900083FCB442F8D19DF806000021C043C0B21D
:10D4A000FFF77AFC02B070BD07B50B0A8DF80000DB
:10D4B0008DF802108DF80330000A0B0C090E8DF860
:10D4C00001008DF80510102069468DF80430FFF733
:10D4D000D1FF03B05DF804FB73B50F4C0646D4F8DA
:10D4E00034010D46FAF795FF94F8293194F82A2172
:10D4F000003318BF01230AB143F00803019396F9E2
:10D50000000000954FF4964300220821FAF7AEFF81
:10D51000C4F8340102B070BDAC2C002010B5064C2C
:10D52000D4F8340105F091FB00B910BDD4F83401F2
:10D5300005F085FBF4E700BFAC2C002008B50B4BD1
:10D54000D3F8382192781E3A012A08D9D3F8340149
:10D5500001210430FFF7C0FFBDE80840DEE70121EC
:10D56000D3F8340105F065FBF6E700BFAC2C0020D2
:10D5700037B5194C94F83C01FCF71AF994F83D3191
:10D58000054683421CD0E8B1D4F83831C3B194F8D1
:10D590002A2193F90200002A0CBF0022082203234B
:10D5A0000192009300224FF496430821FAF75EFFA0
:10D5B000C4F8340120B1FFF7C1FF012384F83D31E5
:10D5C00003B030BDD4F83401FAF723FFC4F8345166
:10D5D00084F83D51F4E700BFAC2C00200028114A2C
:10D5E000B8BF404290FBF2F330B50F4C04FB03058B
:10D5F0003C2068430D4D90FBF2F295F82B5175B924
:10D6000003EB830303EB830302EB83030B804FF4F1
:10D610007A7304FB020292FBF3F24A8030BDC3EB43
:10D620000313F1E780969800806967FFAC2C002017
:10D6300010B50446C0B2FFF7CDFBC4F30720BDE828
:10D640001040FFF7C7BB024B5E21986805F000BB96
:10D65000AC2C002038B50546054C5E21A06805F0CD
:10D66000F7FA2946A068BDE8384005F0F1BA00BFD6
:10D67000AC2C0020038813F0400004D013F4057F85
:10D6800014BF0120002070471F4A73B5D2F84061D3
:10D6900014467EB13046FFF7EDFF58B192F84431A1
:10D6A00033B9D2F848311BB19360012382F8443179
:10D6B00002B070BD94F84C01FCF77AF894F844314C
:10D6C00005468342F4D0C0B1002EF1D094F8293140
:10D6D00096F90200B3FA83F35B0901930223002257
:10D6E000009304214FF41653FAF7C0FEA0600028FF
:10D6F000DED0012384F84431DAE7A068FAF789FE26
:10D70000A56084F84451D3E7AC2C00202DE9F04FFC
:10D7100085B0044603F0D1F9064620B103F002FDBE
:10D7200005B0BDE8F08F204603AA5E4909F0F0FF7E
:10D7300034460546B0464FF0FF37DFF89491DFF8E6
:10D7400094A1DFF894B1BDB90C263946564802F0D1
:10D75000A7FA564B78B206FB05F2D118D256824290
:10D7600000F086800135052DF5D1B8F1000F33D1D9
:10D770004F4802F095FAD3E7012E0ED0022E11D0B9
:10D780001EB9284609F068FF074603AA454900204C
:10D7900009F0BEFF01360546D5E7284609F05CFFD3
:10D7A0008046F2E7494628460CF040FC20B9414942
:10D7B00028460CF03BFC08B144F0010451462846D1
:10D7C0000CF034FC28B9594628460CF02FFC0028F0
:10D7D000DBD044F00204D8E7002C08BF0324002269
:10D7E000E4B20192009443461146FAF73FFE054623
:10D7F00008B93148BDE74146304802F051FA304897
:10D8000002F04EFA2F4B1C682046FAF7F7FD284627
:10D81000FAF7F4FD0021084605F0D2FA00210120B4
:10D8200005F0CEFA204605F010FA70B10121002073
:10D8300005F0C6FA204605F002FA0146284605F032
:10D8400007FA0021084605F0BBFA284605F0FDF965
:10D850000028E7D00121002005F0B2FA284605F0A3
:10D86000EEF90146204605F0F3F900210846D7E716
:10D870004D68002D3FF479AF134802F011FA54B10E
:10D8800069798C4207D02246104802F009FAE1B2C9
:10D89000284605F0CEF9EB6A002BB0D00023EB62EE
:10D8A000ADE700BF6CCC010874CC01083C400020FF
:10D8B0007DCC010855C7010895CC0108ACCC010806
:10D8C000EFCC01084C2B0020C1CC0108D1CC0108C1
:10D8D0006ECC010871CC010862CA01082DE9F04F35
:10D8E0008046894616460D4614464FF0000ADFF87A
:10D8F00010B189B0002E6FD06A6863689A4269D10E
:10D90000AF68A368FB1A5F425F4194F90B305A4637
:10D91000049394F90A3039460393B4F90830404629
:10D920000293B4F906300193B4F9043000935346DE
:10D9300003F096FA95F90B305A46049395F90A309C
:10D9400039460393B5F9083040460293B5F90630DD
:10D950000C340193B5F904300C35009353460AF1A9
:10D96000010A03F093FABAF1080FC3D10024254647
:10D97000DFF890A096B300270123325903FA07FB82
:10D9800059F8043053403BEA030314BF012300233A
:10D9900012EA0B0F079306D000972B4652460799C1
:10D9A000404603F05DFA59F804301BEA030F06D035
:10D9B00000972B4652460799404603F067FA013715
:10D9C0000E2FD9D10135082D04F10C04D2D109B0A4
:10D9D000BDE8F08F002798E73746ABE737460123CD
:10D9E00059F80420BB40134206D000972B465246FC
:10D9F0000121404603F04AFA01370E2FEFD1E1E74B
:10DA000012CD01082ACD01082DE9F04F05468846C0
:10DA100014460027DFF8E0A085B0062300267B43EC
:10DA20000393039B334408EB030292F8C0B0002C2D
:10DA30005ED0234493F8C0305246ABEB0300D0F1E4
:10DA4000000949EB0009019300963B4649462846E8
:10DA500003F006FA8DE840083B4652464946284600
:10DA6000013603F013FA062EDBD10137062FD4D18D
:10DA70000026DFF884B008F1E40A1AF8019B002CB4
:10DA800038D0A31993F8E4305A46A9EB03014F426A
:10DA90004F410193009606233946284603F0E0F9EA
:10DAA0008DE840020623144A39462846013603F021
:10DAB000EDF90B2EE1D198F8F0606CB194F8F030EC
:10DAC0002846F21A019300235442544100930A4A13
:10DAD0000723214603F0C4F9002301960093064A68
:10DAE00007232146284603F0D1F905B0BDE8F08FA1
:10DAF000A146AFE72746D3E73FCD01087FB50546EE
:10DB000002F0DBFF044630B1002218490120FFF784
:10DB10007BFF04B070BD28466A46154909F0F8FD40
:10DB2000134E01AD78B1032C02D103F0FBFAF0E7FC
:10DB300009F092FD6A4645F824003146002009F0BC
:10DB4000E7FD0134EEE7032CEFD101AC70CC324697
:10DB50002946E0B2FBF742FE0028E6D033462A46CB
:10DB60002146044803F0BAF8D3E700BFB0190020FB
:10DB70006CCC01083FCD01082DE9FF478146904656
:10DB80000E4615460027DFF864A0B8F1000F2AD032
:10DB90002B8832889A4224D174886A88A21A544207
:10DBA0005441EA7821460292AA78484601920093AD
:10DBB00052463B4603F054F9F37852460293B37849
:10DBC0002146019336F8043B484600933B46013713
:10DBD00003F05CF9102F05F10405D6D104B0BDE8BF
:10DBE000F0870024DDE74446E6E700BF53CD010897
:10DBF0002DE9F041064602F060FF044628B1BDE879
:10DC0000F041002222490120B6E7304609F024FD08
:10DC10000F2805462EDC304602F057FF0646DFF897
:10DC20007C801C4F2035304609F016FD38F8143042
:10DC3000984226DC012C11D0022C13D027F82500A5
:10DC400030462C210CF096F9064678B101230136B6
:10DC50000134B3B1032CE6D1BDE8F08107EB8503B5
:10DC60009870EDE707EB8503D870E9E7A21E5342F1
:10DC70005341EDE72146BDE8F0410F22064803F08D
:10DC80003AB8002347F82530BDE8F04103F04ABA1E
:10DC9000301A0020B019002081C5010864AB0108CA
:10DCA0002DE9F04F07468A46164600248FB0DFF86C
:10DCB00060800DF124095AF82430494602A80293E5
:10DCC00006F09FFF16B356F82430029D0393EB1A1B
:10DCD0005D420DF1100B5D41594603A806F091FF1E
:10DCE000CDF800B0234642462946384603F0B8F83E
:10DCF0002346CDF80090424629463846013403F0C9
:10DD0000C5F8202CD7D10FB0BDE8F08F3546EFE72E
:10DD100065CD01082DE9F04F87B0054602F0CDFE34
:10DD2000044638B1002255490120FFF7B9FF07B07A
:10DD3000BDE8F08F284609F08FFC1F28074600F346
:10DD40009780284602F0C1FEA0460646A246A1469C
:10DD50002546A346494B009443F827400193484B7E
:10DD6000E1B2E05C00230DF10C0CB64616F8012B75
:10DD70001AB190420FD00A2B09D106AE33440026C7
:10DD8000904203F80C6C08D003F0CCF9CFE703F80D
:10DD90000C200133E9E70246EFE701390EF10106F5
:10DDA000032932D8DFE801F04E1F025B4FF0010E6D
:10DDB000DFF8DCC00DF10B0010F8011F49B30023A0
:10DDC000304AD25C8A4203D00133072BF8D1534644
:10DDD000002212F80CA08A453DD10EFA02F248EA60
:10DDE00002089A46E8E74FF0010C0DF10B0111F81B
:10DDF000012F72B10023244813F800E0964526D184
:10DE00000CFA03F349EA0309F1E703A809F024FC3B
:10DE100083460134052CA2D1009B05F00F0545EA8D
:10DE2000834545EA895949EA0A2A4FEA0B134AEA27
:10DE30000838019ADBB248EA030342F82730FBF7BF
:10DE4000F1FC74E703A809F007FC0546E1E701339C
:10DE5000062BD0D1CBE70132062ABAD1C1E703A8FD
:10DE600009F0FAFB03460F28C8BF00230093D0E750
:10DE70001F222146054802F03EFF58E7B019002056
:10DE80006AAB01086BBD010865BD010881C50108C9
:10DE900072BD01082DE9F34781460F4690460226E0
:10DEA0000024DFF860A0B8F1000F28D037F8242054
:10DEB00038F824309A4238F806201ED1BD5BA91AE2
:10DEC0004D424D4101920093524623462946484611
:10DED00002F0C6FFBB5B5246019337F82430294657
:10DEE000009348462346013402F0D0FF042C06F18B
:10DEF0000406D8D102B0BDE8F0870025E2E7454628
:10DF0000E8E700BF6FCD0108F8B5054602F0D5FD82
:10DF1000064628B1BDE8F840002226490120B9E7AD
:10DF2000254928460BF0F9FF68B94FF47A714FF490
:10DF3000FA62204B19805A809980DA8019815A81BF
:10DF40009981DA81F8BD284609F086FB032804464A
:10DF500028D8284602F0B9FD064658B109F07CFBE6
:10DF600001270546304602F0B0FD30B9BDE8F84063
:10DF700003F0D8B805460746F4E709F06DFB002F1B
:10DF8000F4D040F2DC53A5F2EE229A42EED8A0F291
:10DF9000EE229A42EAD8074B23F8245003EB84037D
:10DFA0005880F8BD3146BDE8F8400322034802F02E
:10DFB000A2BE00BFDE38002046CC0108CBD101084C
:10DFC0002DE9F04F0E461546002797B008900992AC
:10DFD000D6F800800021404608F0A4FF044600283F
:10DFE00069D173680493B3680593F3680693099B3A
:10DFF000002B3DD0D5F800B0EB6859464046D5F827
:10E0000004A0D5F80890079308F08CFF80B1514622
:10E01000049808F087FF58B14946059808F082FF38
:10E0200030B10799069808F07DFF041C18BF012441
:10E0300013A9584601F056FD10A98346504601F039
:10E0400051FD0DA98246484601F04CFD0AA98146C2
:10E05000079801F047FDCDF808900390CDF804A093
:10E06000CDF800B03B46154A2146089802F0F8FE6C
:10E0700013A9404601F036FD10A90446049801F0AA
:10E0800031FD0DA98046059801F02CFD0AA98146B5
:10E09000069801F027FD3B4603908DE81003074AE0
:10E0A00000210898013702F0F1FE082F06F1100652
:10E0B00005F110058CD117B0BDE8F08F80CD0108B7
:10E0C0002DE9F84F07460026534D384602F0F5FC7F
:10E0D000804628B10022BDE8F84F4F4901206FE784
:10E0E00005224E4938460BF053FF38B900224A4BFF
:10E0F000C25010308028FBD1BDE8F88F0422484977
:10E1000038460BF045FF04463846002C3FD102F05C
:10E11000DCFC814600287CD007F0ACFFDFF818A1BA
:10E120005FFA80FB5AF82480B8F1000F04D13D4813
:10E13000BDE8F84F02F0F0BF5A46414648460BF0A2
:10E1400027FF013407460028ECD1374B2E6003EB44
:10E15000C404D4F810E02E612E622E632E642E6566
:10E160002E662E67BEF1000F03D094F80CC06745F1
:10E1700005DB41462D4802F0B1FD2D4FA5E73B01DF
:10E18000EC1873440FCB013784E80F00EFE709F078
:10E1900063FA0728054635D8384602F096FC06464D
:10E1A00028B301F003FC01241B4A2B01D050304658
:10E1B00002F08BFC064630B101F0F8FB164B01343F
:10E1C00003EB05135860304602F07FFC064630B181
:10E1D00001F0ECFB104B013403EB05139860304663
:10E1E00002F073FC28B9BDE8F84F02F09BBF04466B
:10E1F000DDE701F0DBFB084B032C03EB0515E860C2
:10E20000F1D167E74146BDE8F84F0722094802F01F
:10E2100072BDBDE8F88F00BFA421002046CC0108E4
:10E220004CCC0108DDC5010864AB010851CC0108E4
:10E2300014DB010881C5010854A701082DE9F04F3E
:10E24000814690460C46154600261927DFF8B0A0F7
:10E2500087B0B8F1000F51D023782A7893422B79F8
:10E260004AD160786978884246D1A078A9788842F6
:10E2700042D1E078E97888423ED1217999423BD178
:10E2800061796879081A414241410593EB78484623
:10E290000493AB788B467B4303F5617303936B78F0
:10E2A00001927B4303F5617302936B7952460093AD
:10E2B000334602F0D5FD237952460593E37859465B
:10E2C0000493A37848467B4303F561730393637813
:10E2D00006357B4303F5617302932378063401937B
:10E2E00014F8013C00933346013602F0CFFD0F2EA7
:10E2F000AFD107B0BDE8F08F0021C6E7C346DAE72B
:10E3000094CD0108F7B5074602F0D7FB044630B1BB
:10E31000002236490120FFF791FF03B0F0BD3846D7
:10E3200009F09AF90E28054659DC06264643781C62
:10E330008DF8074002F0C9FB2C4C074650B109F09C
:10E340008BF9032806D8A31958719DF807300133BB
:10E350008DF80730384602F0B8FB074658B109F08F
:10E360007BF90D2807D806236B43E0549DF807304E
:10E3700001338DF80730711C0DF107022144384636
:10E3800002F0AFFB02F0A1FB074660B109F064F9AF
:10E39000182808D8062303FB0543D8709DF80730DA
:10E3A00001338DF80730384602F08FFB60B109F079
:10E3B00053F90D2808D8062303FB05459DF80730BF
:10E3C000287101338DF807309DF80730062BA4D053
:10E3D0000023A219A351938002F0A4FE9DE70E2210
:10E3E0002146034802F087FC97E700BF5C2300202A
:10E3F00081C50108034610B500F16004064A0C33DC
:10E4000003CA43F80C0C106843F8081C43F8040CCA
:10E41000A342F3D110BD00BF68AE010840F2DC5347
:10E420000380322343800123042283730023C273B9
:10E430001A4630B5084C838119198D792D0741BFD3
:10E440000D7981180D710132B02B03D0072A03F129
:10E450001003F1DD30BD00BF38A5010838B5034613
:10E46000064D00F1DE0418464A22294609F01CF93F
:10E4700003464A33A342F6D138BD00BF74AE01084B
:10E4800040F22E4303824FF4F07303800123837024
:10E490004FF4FA6343824FF47A7383824FF4E1734B
:10E4A000C38100231A4630B5074C19198D796D07C1
:10E4B00041BF0D7981184D710132B02B03D0072A6D
:10E4C00003F11003F1DD30BD38A5010838B5002493
:10E4D000054D55F83400013402F072FB02F0E7FB01
:10E4E000232CF6D138BD00BFC0AE01080121FCF7D6
:10E4F00097B80021FCF794B810B5054C206804F0DB
:10E50000A4FB0028FAD02068BDE8104004F097BBB7
:10E51000303A0020082341F2210280EA012010F461
:10E52000004F4FEA400018BF5040013B80B2F6D187
:10E53000704738B50546064B064C0146186804F08E
:10E5400087FB20882946FFF7E5FF208038BD00BF04
:10E55000303A0020383A002038B5FFF7CDFF044D9F
:10E56000044601462888FFF7D5FF2880204638BD9D
:10E57000343A002070B5104D00242846214600F89A
:10E58000014B70220BF0C1FC284671352146A5F1E4
:10E5900070046B1893F902206AB11E680A190E51B3
:10E5A0009E889B79073193710378702903F10103E9
:10E5B00096800370EDD170BD0C2E00200C220A4B0A
:10E5C00002FB003292F8EF20FF2A07D007490978B2
:10E5D000914203D9064B33F9120070470C2202FB1B
:10E5E0000030B0F9EC0070470C2E0020FC37002002
:10E5F000EC1E00202DE9F74F0546074600265A4C31
:10E60000DFF880B1DFF8809104F5A27A04F5A878EC
:10E6100004F5AE723878019208F09CFA594608F079
:10E62000EDFA4AF82600787808F094FA494608F09E
:10E63000E5FA48F82600B87808F08CFA4B4908F05B
:10E64000DDFA019A033742F826000136032EE1D1A4
:10E6500095F83B0008F07EFA454908F0CFFAC4F877
:10E66000680195F83A0008F075FA0146414808F04B
:10E6700079FBC4F86C01687D08F06CFA3E4908F03B
:10E68000BDFAC4F87001A87D08F064FA3A4908F0B0
:10E69000B5FAC4F87401E87D08F058FA95F83430FA
:10E6A00095F8336084F87C31C4F87801C6F1AF0086
:10E6B00008F050FA314908F0A1FAC4F88001C6F117
:10E6C000640008F047FA2E4908F098FA6427C4F865
:10E6D0008401E88FD4F88861784308F03BFA31462A
:10E6E00008F08CFAC4F89001C4F88C01A88F784324
:10E6F00008F030FA314608F081FAC4F8940195F830
:10E70000280008F023FA1E4908F078FA01464FF075
:10E710007E5008F069F901464FF07E5008F022FB68
:10E720004FF47A73C4F89801B5F8442095F847007F
:10E730005343C4F89C310A2395F846205343C4F848
:10E74000A03108F003FAC4F8A401B5F8420008F0BB
:10E75000FDF9C4F8A801B5F8400008F0F7F9C4F8CD
:10E76000AC0103B0BDE8F08F0C2E002097AC0A3A44
:10E770000402013C0000C842CDCCCC3D6666E63FB9
:10E780000AD7233CD730033D033F7A3E2DE9F74FAC
:10E790006B4C0546D4F888114FF07C5008F0E2FA33
:10E7A00008F02EFCAB8C0746984230D3184608F090
:10E7B000CDF90021804608F0B5FB58BB614B4046BF
:10E7C000C4F8B03108F01CFCEE8C80B2314603F086
:10E7D000F1FD4FF0010B82465B4EDFF8909103464E
:10E7E000D9F8002041463046CDF800B0C4F8B461F5
:10E7F00003F030FD06F12C00CDF800B05346D9F8F7
:10E8000000204146C4F8B80103F024FD05E0EB8C7C
:10E810009842CCD84D4BC4F8B031288C08B187420F
:10E820000CD24A4BC4F81432688C08B1874269D2C2
:10E83000464BC4F8983403B0BDE8F08FAB7F012B92
:10E8400043D01AD3022BECD1414EDFF82081414B4B
:10E85000B8F80020C1B23046C4F81432C4F81862C7
:10E8600003F0DAFC06F58070B8F8002095F8201067
:10E87000C4F81C0203F0D0FCD6E7374BC0B2C4F892
:10E88000143208F067F90146344808F06BFAD4F8FE
:10E89000886180460146304608F0A8F801463046B7
:10E8A00008F060FA2E4BC4F82882C4F818321033EE
:10E8B000C4F82C62C4F82402C4F81C32C4F83882AC
:10E8C000C4F83C62C4F83402AEE71E4B254EC4F8CF
:10E8D0001432C4F8186208F039F9DFF89080014664
:10E8E000D8F8002030462C3603F058FDC4F81C62DE
:10E8F000288C08F02BF9D8F800200146304603F0A8
:10E900004DFD91E7144BC0B2C4F89834164BD4F8BF
:10E910008851C4F89C3408F01DF901460F4808F0EE
:10E9200021FAC4F8AC540146C4F8A804284608F0FB
:10E930005DF80146284608F015FAC4F8A4047AE701
:10E940000C2E0020611E0108C82F00203F1F010867
:10E95000A4300020FD1D0108211F010883F9223E7B
:10E960002C3000204C300020AC3200201419002044
:10E9700038B5134A134C054694F8B0341068584320
:10E98000114B186008F0E2F8104908F037F9C4F8A4
:10E9900088012846FFF7FAFE2846FFF72BFE688D10
:10E9A00008F0D8F80A4908F029F9C4F8B404A88D89
:10E9B00008F0D0F8064908F021F9C4F8B80438BDC9
:10E9C000FC3F00200C2E002014190020BD37863596
:10E9D0006F12833A2DE9F0410024094D094E0A4F88
:10E9E0002878844205DBBDE8F041084BD3F8BC34FD
:10E9F000184756F82410E0B23B6898470134EFE717
:10EA000044170020481700203C3A00200C2E00201C
:10EA10002DE9F74F4C4B4D4CD3F80090D4F8C0542F
:10EA20004946284608F0EAF8D4F8C47480464946B6
:10EA3000384608F0E3F8D4F8C864009049463046F8
:10EA400008F0DCF839468246284608F0D7F8314607
:10EA50008346284608F0D2F831468146384608F009
:10EA6000CDF839460190384608F0C8F8014607F05D
:10EA7000BDFF31460746304608F0C0F8014607F0B2
:10EA8000B5FF06460146384607F0B0FF01464FF095
:10EA90007E5007F0A9FF5146C4F8CC04584607F051
:10EAA000A3FF014607F0A2FF4946C4F8D00400982E
:10EAB00007F09CFF014607F099FF5946C4F8D404BB
:10EAC000504607F093FF014607F090FF2946C4F82F
:10EAD000D804284608F092F8014607F087FF00F1B5
:10EAE00000453146284607F07FFF4FF07E5107F082
:10EAF0007DFF4146C4F8DC04019807F075FF01462C
:10EB000007F074FF0099C4F8E004484607F06CFF72
:10EB1000014607F06BFF0199C4F8E404404607F092
:10EB200065FF014607F062FF3946C4F8E80428464D
:10EB300007F05AFF4FF07E5107F058FFC4F8EC047D
:10EB400003B0BDE8F08F00BFE00300200C2E0020D2
:10EB50002DE9F04FB44B87B01B6813F0020FB34B95
:10EB600000F0448393F84020002A00F03F83D3F85C
:10EB700034909F6B09FB09F5AD4C07FB0755D4F8A2
:10EB8000F024DE6B821A039206FB06526425C4F859
:10EB9000F00403985543B3F810A007F0D7FFA54938
:10EBA00008F02CF8DFF8ACB20090A349DBF80400C1
:10EBB00008F024F8A0498046DBF8080008F01EF8A9
:10EBC0000AFB0AFA95FBFAF501909B49DBF80C0069
:10EBD00008F014F8523D262D02904FF0000500F287
:10EBE000F282484607F0B6FF8146384607F0B2FF8A
:10EBF0000746304607F0AEFF39460646384607F06E
:10EC0000FDFF31468246304607F0F8FF0146504688
:10EC100007F0ECFE49468246484607F0EFFF014602
:10EC2000504607F0E3FE8549824608F0A3F9002824
:10EC300000F0C982504609F05DF901464FF07E5060
:10EC400008F090F883460146484607F0D7FF59463A
:10EC50008246384607F0D2FF59468146304607F0D3
:10EC6000CDFFD4F8EC34064619464846049307F025
:10EC7000C5FFD4F8E8B407465946304607F0BEFF52
:10EC80000146384607F0B0FED4F8E4440746214672
:10EC9000304607F0B3FF049B06461946504607F07E
:10ECA000ADFF0146304607F09FFE594606465046E6
:10ECB00007F0A4FF21468246484607F09FFF014621
:10ECC000504607F091FE8146594C0021D4F8F4A437
:10ECD000504608F04FF9002800F079820199084663
:10ECE00007F08CFF02990546084607F087FF0146AA
:10ECF000284607F07BFE41460546404607F07EFF6A
:10ED00000146284607F072FE4D4908F015F910B388
:10ED10005146009807F072FF05460146384607F055
:10ED20006DFFD4F8001507F061FE2946C4F8000510
:10ED3000304607F063FFD4F8041507F057FE294664
:10ED4000C4F80405484607F059FFD4F8081507F041
:10ED50004DFEC4F808053B4BD4F8F8041B78DA07DD
:10ED600000F13C82384B1A6844F61F639A4200F265
:10ED70003582364907F042FFD4F800150546404673
:10ED800007F034FE29468046384607F037FF014633
:10ED9000404607F02BFED4F804158046019807F092
:10EDA00025FE29460746304607F028FF014638462B
:10EDB00007F01CFED4F808150746029807F016FE67
:10EDC00029460646484607F019FF0146304607F037
:10EDD0000DFE4FF07C518146009807F00FFF414631
:10EDE000064607F00BFF39460546304607F006FF9A
:10EDF00049468046304607F001FFD4F8C094144BD2
:10EE00008246294609F10040D3F800B0059307F087
:10EE1000F5FED4F8C46401903146404607F0EEFE9A
:10EE2000019A014618E000BF60190020F816002082
:10EE30000C2E0020BD37863535FA8E3C0AD7233C90
:10EE4000E68AF93D301B00204C3A002000002041AA
:10EE5000E0030020FC3F0020104607F0C5FDD4F879
:10EE6000C87401903946504607F0C8FE019A014621
:10EE7000104607F0B9FD594607F0B8FD5946019014
:10EE8000284607F0BBFE31460290504607F0B6FE1A
:10EE9000029A0146104607F0A9FD494607F0A6FD73
:10EEA00039460290404607F0A9FE029A01461046F4
:10EEB00007F09AFD59460490404607F09FFE3946F8
:10EEC0000290284607F09AFE0146029807F08EFD50
:10EED000314607F08BFD49460290504607F08EFE02
:10EEE0000146029807F080FD59460290504607F00F
:10EEF00085FE49468246404607F080FE0146504660
:10EF000007F074FD394607F071FD31460746284683
:10EF100007F074FE0146384607F066FD0199064683
:10EF2000084607F06BFE049A05461146104607F0A6
:10EF300065FE0146284607F059FD02990546084638
:10EF400007F05CFE0146284607F050FD31460546B5
:10EF5000304607F053FE0146284607F047FD08F00B
:10EF6000C9FF01464FF07E5007F0FCFE0546014602
:10EF7000019807F043FE049A059B29461860104645
:10EF800007F03CFE2946C4F8C004029807F036FE9C
:10EF90002946C4F8C404304607F030FEC4F8C8045B
:10EFA000FFF736FDD4F8E834D4F8EC941846494617
:10EFB000019308F0A7FD904907F020FE08F0DAFC65
:10EFC000D4F8E4A4A4F80C050AF1004008F04AFDC6
:10EFD00001468A4807F008FD874907F00FFE08F050
:10EFE000C9FCD4F8D834D4F8CCB4A4F80E055946EA
:10EFF0001846029308F086FD7F4900F1004007F0B3
:10F00000FDFD08F0B7FC03B2002BA8BFA4F8103533
:10F010007B4BBCBF00F56160A4F81005D3F8141554
:10F02000484607F0A7FF774B1A78002800F0D980F0
:10F0300042F00802744D1A70686B07F08BFD0746AA
:10F04000A86B07F087FD8046E86B07F083FD6C4CEA
:10F050000646D4F8D014404607F0D0FD5946049037
:10F06000384607F0CBFD049B0146184607F0BEFC6E
:10F07000D4F8D4148346304607F0C0FD0146584604
:10F0800007F0B4FC51468346384607F0B7FD0199B6
:10F090008246404607F0B2FD0146504607F0A6FC06
:10F0A00049468246304607F0A9FD0146504607F022
:10F0B0009DFCD4F8DC148146404607F09FFD029980
:10F0C0008046384607F09AFD0146404607F08EFC20
:10F0D000D4F8E0140746304607F090FD0146384664
:10F0E00007F084FC94F8FC3400F10046012B7BD13E
:10F0F000464B1B78DB070ED44023D4F8180590FB51
:10F10000F3F3C01A07F026FD494607F06FFC07F03D
:10F1100051FFC4F818054023D4F8180590FBF3F00C
:10F1200007F018FD0146484607F05EFCD4F82015AC
:10F130000746009807F05AFC0146009807F012FEB7
:10F14000D4F81C5580462946384607F04DFC014648
:10F15000404607F053FD294607F048FC0546C4F831
:10F160001C05584608F006FC94F8FE74394602F077
:10F17000DCFFD4F824351844C4F82405304608F0E0
:10F18000F9FB394602F0D1FFD4F828351844C4F809
:10F190002805284608F0EEFB94F8FF1402F0C5FF9E
:10F1A000D4F82C35039A1844D4F83035C4F82C051B
:10F1B0001344C4F83035D4F834350133C4F8343549
:10F1C00007B0BDE8F08F2E462F46A9467CE5C4F86F
:10F1D0000055C4F80455C4F80855BCE54FF07E51FD
:10F1E000C8E522F0080225E7288A99E700225A6339
:10F1F0009A63DA63E4E700BF4C3D0F44DB0FC93F7D
:10F200000C2E0020C4160020F8160020301B002011
:10F21000012310B50A4C4FF48060E370022384F898
:10F22000203006F08BFE6421064B1A68064B93F8DB
:10F23000393501FB0323636123880133238010BD2B
:10F24000641B00204C3A00200C2E00202DE9F04FCA
:10F250003D21C7B081460AF08DFE002800F0DE8017
:10F26000034613F8012C591E202A50D0A3EB0903A2
:10F27000013005462A780130202AFAD04FF00008E4
:10F28000DBB2684E01930D2303FB08FB06EB0B0773
:10F29000D7F87041204606F0EDFE21460246029066
:10F2A00048460AF075FE0446002840F0AD80019BF8
:10F2B0001A46029B934240F0A78097F874315A4E49
:10F2C00003F03003102B5E4423D0202B4FD08BBB98
:10F2D000284608F0C1F9B7F9753101B28B4229DC33
:10F2E000B7F977318B4225DB304601F031FC0D2335
:10F2F0004C4A4E4803FB0828D8F8701101F037FC3F
:10F300000021304601F0C8FC47B0BDE8F08F0B4645
:10F31000A7E78346814697F87571424B03EBC70711
:10F3200097F818AA544502D2BBF1000F09D0B9F1E1
:10F33000000FDCD13E4801F0EFFE304601F0E2FC68
:10F34000E2E7D7F8143A294653F824000AF0E5FD1D
:10F3500000280CBF4FF0010B4FF0000B05D121B27C
:10F36000304601F0F5FB4FF001090134DAE7814640
:10F3700097F875B10DF1180A0BF1FF330293A3450D
:10F38000D5DD2F4600E017463B783D46202B07F1A0
:10F390000102F8D02C2138460AF0ECFD019008B3A8
:10F3A000029BA342C3DD054615F8013C6A1E202BD3
:10F3B00016D0ED1BEDB2032DB9D805AB2A46394660
:10F3C000184603930AF01DFE0022039B18465A5567
:10F3D00008F042F9019D0AF8040001350134CEE736
:10F3E0001546E1E7029B9C42A1D1384608F034F96A
:10F3F0000AF80400304601F09EFB5A46514608F0D8
:10F4000053F94FF00109E9E708F10108B8F1AA0F33
:10F410007FF439AF074801F07FFE75E74846FBF7F8
:10F42000CBF871E768AE0108D8AF0108B2CD01088A
:10F43000BDCD0108DDC501081523037016238370B7
:10F44000172303712D2343702E23C3702F23437181
:10F4500070470B4B984206D0A3F5784398420DD0E5
:10F460004FF0FF3070470022064B03EB02135A891E
:10F47000013292B25A81588980B270470122F3E773
:10F4800000300140BC0C002003685A1C0260197057
:10F490007047024B186803F0DBBB00BFB039002097
:10F4A0002DE9F04101270B4DDFF82C802C686A69AB
:10F4B00014400CB9BDE8F081B4FA84F3C3F11F0322
:10F4C00058F8230007FA03F60368984724EA06046D
:10F4D0006E61EEE700040140400B002008B503F028
:10F4E000E7FB40B12C2282710022C2714A21BDE8A3
:10F4F000084003F003BC08BD41F4807191FAA1F209
:10F500000029B2FA82F208BF4FF0FF320388013AB5
:10F5100023F040031B041B0C038003889BB223F0E1
:10F52000380343EAC2039BB2038003889BB243F0D3
:10F53000400303807047F8B584894FF6FF764FF497
:10F540007A740BB90120F8BD92B1157801320789A0
:10F55000BF070FD54FF47A74ADB285810589ED07E9
:10F5600012D58589ADB209B10D700131013BE8E7D3
:10F57000FF25ECE7013CA4B2B442E8D1FFF769FFF4
:10F58000003018BF0120F8BD013CA4B2B442E5D15F
:10F59000F4E708B540F2E9330289920708D540F252
:10F5A000E93389B281810289D20709D5808905E0D2
:10F5B000013B9BB2002BEFD1FFF74BFFC0B208BD60
:10F5C000013B9BB2002BEED1F6E737B504460D4662
:10F5D000406803F0B5FB45F080012068FFF7D9FFD4
:10F5E000012300220DF107012068FFF7A4FF6068E6
:10F5F00003F0ABFB9DF8070003B030BDF8B504463F
:10F600000F4616461D46406803F09AFB47F08001FE
:10F610002068FFF7BEFF3346002229462068FFF727
:10F620008AFF606803F091FB0120F8BD70B50446C5
:10F630000E461546406803F083FB31462068FFF70D
:10F64000A8FF29462068FFF7A4FF606803F07DFB50
:10F65000012070BDF8B5484C0601A7190546387A57
:10F6600005F066F801233A7A02F01F015209022AD6
:10F6700003FA01F357D0032A5AD0A319187903F0DB
:10F6800017FB0135EDB2074610B11223C571837126
:10F69000A319587903F00CFB10B11323C5718371C2
:10F6A000A319987903F004FB10B11423C571837179
:10F6B0001B213846A51903F021FB687903F0F8FAFD
:10F6C000072103F01BFBA87903F0F2FA1B2103F0DA
:10F6D00015FBA359294A93422FD102F56042D16804
:10F6E00041F48051D160D16821F48051D16034441B
:10F6F000227B002A3CD101220220198801F44151C9
:10F7000041F445710A4302431A809A8B22F4006245
:10F710001204120C9A8307221A821A8892B242F0BB
:10F7200040021A80F8BD164AD1680B43D360A4E7A3
:10F73000134A11690B4313619FE7124A93420AD19E
:10F7400002F5EC32116941F480411161116921F433
:10F7500080411161CBE70C4A9342C8D102F5EA32ED
:10F76000116941F400411161116921F40041F0E790
:10F7700000221046C1E700BFBC0C00200030014051
:10F780000010024000380040003C004010B5427AB2
:10F79000044632B1036800F10A014068984700232B
:10F7A000637210BD2DE9F341056906460F46002D31
:10F7B0003BD1D0F80080C8F3090373B300234FF4A2
:10F7C0000050D6F800800193FDF73CFC042821D1BD
:10F7D0002A4C4FF40050236943F001032361BBB26C
:10F7E000A8F80030FDF72EFC04283CD108F10203F4
:10F7F0000193019B3F0C1F804FF40050FDF722FC4A
:10F800002369042823F001034FEAC3434FEAD3439B
:10F8100023612FD06FF0010507E04FF43020FDF792
:10F8200011FC042805D04FF0FF35284602B0BDE892
:10F83000F081124C4FF43020236943F0020323611E
:10F84000C4F81480236943F040032361FDF7FAFBF9
:10F850002369042823F002034FEAC3434FEAD3434A
:10F860002361ABD0DFE7236923F00103DB04DB0C6A
:10F870002361CFE7336804333360D6E700200240CA
:10F88000F8B504460D4600278E18B54201D120690F
:10F89000F8BDE368591CE16015F8012B23440429E5
:10F8A0001A72F2D1A1682046FFF77CFFE760206161
:10F8B000EBE770B50D46064644880021C4F30B04FF
:10F8C000224628460AF021FB33690A4A934209D3AB
:10F8D000094A934206D222462846BDE8704019469E
:10F8E00007F0E2BE23B121462846BDE87040184724
:10F8F00070BD00BFF4E301088BE40108064B074923
:10F900008B4202D30023184670471A88C2F30B02B9
:10F910009042F8D01433F3E770E00108F4E30108F3
:10F92000024A136823EA000010607047A8220020F2
:10F93000F8B51A4D2B789F2B2ED16B78BE2B2BD17F
:10F9400005221749A81C0AF023FB28BB07222946D9
:10F950004FF6FF7002F0DEFB124FEC1D22884AB119
:10F96000A618BE4218D2052A16D9214602F0D2FBAB
:10F970003446F3E72146022202F0CCFB0222A11812
:10F9800002F0C8FB0634084B641B1C8041F60F5381
:10F99000C31A58425841F8BD0020F8BD00F80108CC
:10F9A0003BBE0108000002087E2000202DE9F8433C
:10F9B00002780346202A00F10100F9D0092AF7D085
:10F9C0002D2A4BD10346444D1C460026DFF80C81FE
:10F9D000234614F8012BA2F13007F9B2092943D9C3
:10F9E0002E2A09D127463D4CA0463B4617F8010B6D
:10F9F0003038C2B2092A44D91A7802F0DF02452A07
:10FA000063D15A782D2A4CD10127023300240A20D1
:10FA1000013B13F8012F303AD1B2092947D9B4F587
:10FA20009A7F28BF4FF49A744FF07E50A046DFF8BB
:10FA3000B090B8F1070F3DD8DFF8A08004F00704BC
:10FA4000002C3DD1002F42D00146304607F08AF904
:10FA50000146284607F0D2F8BDE8F8832B2A08BFF4
:10FA600003464FF07E55AFE74146304607F0C6F8F3
:10FA70000646384607F06EF8314606F0B7FF0646F0
:10FA8000A6E707F067F8214607F06CF90146304613
:10FA900006F0ACFF41460646204607F0AFF80446A4
:10FAA000A3E72B2A14BF013302330027AEE700FB84
:10FAB0000424AEE7494607F0A1F8A8F10808B8E722
:10FAC000414607F09BF8013CBAE74FF07E500146F3
:10FAD000304607F093F8BBE7000080BF00002041EC
:10FAE00020BCBE4C002330B50C4687B00021054633
:10FAF00000930193029307F03DFA294900283DD075
:10FB0000284606F073FF274907F078F807F052FA05
:10FB1000054680EAE07003A9A0EBE57005F016F851
:10FB2000002DACBF20232D2303A88DF8003006F054
:10FB3000A1FA012826D130238DF801308DF802304A
:10FB40008DF8033003A968460AF005FA684606F006
:10FB500091FA0338C5B22A46694620460AF051FA9E
:10FB600000231149635520460AF0F5F90DEB050114
:10FB700020460AF0F0F9204607B030BD284606F0CE
:10FB800033FFC0E7022805D130238DF801308DF80E
:10FB90000230D7E7032804BF30238DF80130D1E7C6
:10FBA0006F12033A00007A44CCCB010870B50646C8
:10FBB000B6FBF2F40846154614B12046FFF7F6FFEF
:10FBC00005FB1464024B1B5D00F8013B70BD00BFD8
:10FBD000D8D8010870B50124B0FBF4F58D4202D2EB
:10FBE0001CB91C7070BD4C43F6E7B0FBF4F6092E4F
:10FBF0000BDD002A14BF37255725354404FB1600BA
:10FC000003F8015BB4FBF1F4EAE73025F5E702689D
:10FC100010B51146531C036011F8024BD31C016050
:10FC20005178036093781B0443EA0123111D01609E
:10FC3000D078234343EA006010BD03685A1C026079
:10FC40001A4612F8021B0260587841EA00207047F9
:10FC500038B504461546006807F026FD22682A4498
:10FC6000226038BD03685A1C0260197003685A1C70
:10FC700002600A0A1A7003685A1C02600A0C1A70A1
:10FC80000368090E5A1C02601970704703685A1CF9
:10FC9000026019700368090A5A1C026019707047E3
:10FCA0000FB437B50B4906AB0B4853F8042B096862
:10FCB0000068019302F045F90446084D286802F0F7
:10FCC000BBFF0028FAD0204603B0BDE8304004B0A6
:10FCD000704700BF200B0020240B0020B03900200B
:10FCE00010B50E22002104460AF00FF90A232380E2
:10FCF00000236381A381A380E380238110BD037867
:10FD00008B4286BF024B33F811000020704700BFC2
:10FD100018360020034B187E10B1002201201A76FD
:10FD2000704700BF18360020F0B5002541F22107CA
:10FD30002B46224A517E8E1EECB2B44217DB0144A0
:10FD40008C1E013914441144A47E897E01EB0421E8
:10FD500089B28B420AD100244FF4AF6692F83D502D
:10FD60000130E3B29D4216D801231376F0BD04445E
:10FD70001444A47E83EA0423082413F4004F04F1FE
:10FD8000FF344FEA430318BF7B4014F0FF049BB2DB
:10FD9000F3D10135D0E700EB4303D9B25318013159
:10FDA00011449F7E8B7E03EB07239BB273431B138F
:10FDB00003F5487322F814300134D2E718360020D6
:10FDC00007298FBF0020034B03EB8101086C80B231
:10FDD000704700BF183600202DE9F041174D95F807
:10FDE000602012B90020BDE8F081002285F8602073
:10FDF00095F86120A82AF5D195F87440002CF1D12E
:10FE00000F4F104E05F16108403508EB0403D87818
:10FE10001B7903EB002006F099FE394606F0EEFE52
:10FE2000314606F0E1FD07F0EBF845F81400023426
:10FE3000102CEAD10120BDE8F08100BF1836002067
:10FE40000000203E0080BB43034B03EB4101B1F8AF
:10FE50007600C008704700BF183600201F4BF0B571
:10FE600093F8962019460AB90020F0BD002093F8B7
:10FE70009740B3F8986003EB440595F89D7095F8AA
:10FE80009E2083F8960042EA07229642ECD193F82E
:10FE90009B30012B02D0812B14D0F0BD1846102CC2
:10FEA00088BF10234FF0000288BF81F897300C4BB9
:10FEB00091F89740A3F12705D1B28C4203F10203D8
:10FEC00002D8F0BD0320EAE713F8026C13F8011C16
:10FED00041EA062125F812100132EDE7183600201C
:10FEE000B536002003788B420CD9074B890093F874
:10FEF000BF200B44D3F8C00002B1400800F5777072
:10FF000080B270470020704718360020054B03EB85
:10FF10008101D1F8F00000EB8000C00800F55C70B2
:10FF200080B27047183600205E4B10B593F8380148
:10FF3000002800F0B680002293F83B4193F83C0182
:10FF400083F8382193F83A2104F0070142EA0122AC
:10FF500000F03F01490141EAD401C3F8F02093F8D1
:10FF60003D21C3F8F41093F83E11920093F83F41FD
:10FF700042EA901201F0010042EA8022C3F8F82020
:10FF800093F8400104F00F02D20142EA510200F05E
:10FF90007F01C3F8FC20090193F8412141EA1411C3
:10FFA00093F842415200C3F8001142EAD01204F023
:10FFB000030193F8430142EA4122C3F8042193F874
:10FFC000442100F01F018901D20041EA940142EA74
:10FFD000501293F8464193F84701C3F80C2193F867
:10FFE0004521C3F8081104F0070142EA012200F09C
:10FFF0003F01490141EAD401C3F8102193F8482197
:020000040801F1
:10000000C3F8141193F84911920093F84A4142EA57
:10001000901201F0010042EA8022C3F8182193F8FF
:100020004B0104F00F02D20142EA510200F07F01BD
:10003000090141EA1411C3F82011C3F81C2193F8F7
:100040004C2193F84D41520004F0030142EAD012D2
:1000500042EA4122C3F8242193F84F2193F84E013C
:10006000D20042EA501200F01F01C3F82C2193F88D
:100070005021890141EA9401D407C3F828114CBFEB
:1000800040F21471AD21C3F8301191074CBF40F21A
:100090001471AD2112F0080F14BF03200120C3F822
:1000A000341110BD1836002008B5084B03EB810150
:1000B000D1F8540106F04AFD054906F09FFD0549B7
:1000C00006F094FC06F09CFF80B208BD18360020B4
:1000D00001F11F3F00405C446B4B30B593F8942115
:1000E0000AB9002030BD002283F8942193F89721AB
:1000F000162AF6D1082112F0800F4FEA420218BFEB
:1001000082F0D5020139D2B2F5D193F896015F4D54
:1001100002388142C0F2A78093F8AE119142E0D13B
:10012000182293F8994193F89A0183F8962193F84D
:10013000982104F0070142EA012200F03F01490141
:10014000C3F8542141EAD40193F89B21C3F8581114
:1001500093F89C11920093F89D4142EA901201F0AD
:10016000010042EA8022C3F85C2193F89E0104F06A
:100170000F02D20142EA510200F07F01C3F8602170
:10018000090193F89F2141EA141193F8A04152000C
:10019000C3F8641142EAD01204F0030193F8A101FC
:1001A00042EA4122C3F8682193F8A22100F01F011E
:1001B0008901D20041EA940142EA501293F8A44125
:1001C00093F8A501C3F8702193F8A321C3F86C112B
:1001D00004F0070142EA012200F03F014901C3F89F
:1001E000742141EAD40193F8A621C3F8781193F859
:1001F000A711920093F8A84142EA901201F0010081
:1002000042EA8022C3F87C2193F8A90104F00F028E
:10021000D20142EA510200F07F01090141EA1411C2
:10022000C3F88411C3F8802193F8AA2193F8AB4155
:10023000520004F0030142EAD01242EA412293F84C
:10024000AC01C3F8882193F8AD2100F01F018901AA
:10025000D20042EA501241EA9401C3F88C11C3F86B
:100260009021012030BD6C18E4786240082412F01F
:10027000800F4FEA420218BF82F0D502013CD2B291
:10028000F5D1013145E700BF18360020AD37002019
:1002900070B5304E054633782F4C3BB1D4F8BC31A5
:1002A00083429EBF0023337084F8C0312B4B1B6800
:1002B00013F001021CD094F8C12194F8C23193428A
:1002C0000CD00123002184F8C031254B84F8C221D1
:1002D0001970D4F8C4312B44C4F8BC3194F8E0311F
:1002E00073BBD4F8F001854234BF0020012070BDFB
:1002F00013F4005308D013461A4A32F8131009BBFE
:1003000001330C2BF9D1E9E784F8E031D4F8EC3172
:100310009847C307E2D5012300F00200002814BF6C
:100320001A46002284F8E0310D4B5A700CBF0123AD
:1003300000233370D4F8C4312B44C4F8BC31CDE76A
:10034000012070BD0123002284F8C031044B1A70D3
:10035000F0E700BF311B002018360020601B002092
:10036000E4030020E03700200020704700207047A1
:100370000023032BCCBF012200220CBF05211E212C
:1003800000F8132000EB43020133122B5170F0D11F
:10039000704710B500234FF47A744FF4FA61C452D9
:1003A000C2180433102B5180F9D110BD70B5054629
:1003B00002F082FB324CD4F8F431C4F8F401C31AD1
:1003C000B3F5FA5F82BF002384F8F83184F8F9317D
:1003D00094F8F83133B9A12D1ED1012284F8F92106
:1003E0001B22627694F8F9212AB1E218EDB20133AA
:1003F000957684F8F83194F8F851637EAB420AD1CF
:1004000094F8FA31052B0ED0062B0FD0002384F878
:10041000F93184F8F83170BDA22DE3D1012284F8BE
:10042000F9212322DDE70020FFF77EFCE37E1E2B6F
:10043000ECD100200246013DC3B2AB4207DB2544AC
:10044000AB7E9A42E2D10320FFF76EFCDEE7082183
:1004500023449B7EDBB282EA030616F0010F4FEACB
:10046000530301F1FF310CBFDBB283F08C0311F0B9
:10047000FF01C2F34702EED101301A46DCE700BFAC
:100480001836002010B5044602F016FB41F2883100
:100490000D4BD3F8FC21C3F8FC01821A8A4284BFB9
:1004A000002283F8002293F80022142A03EB0201B1
:1004B0000CBF0122013281F8614014BF83F8002291
:1004C00083F8602010BD00BF1836002010B5044628
:1004D00002F0F2FA254BD3F80422C3F80402821A80
:1004E000B2F57A6F84BF002283F8082293F80822BD
:1004F0004AB9A82C38D183F89620A3F898209918E7
:1005000081F89A4006E0022A02D183F89740F6E784
:10051000242AF4D993F8971001320231D2B249005B
:100520008A4283F8082216DA082241F22101B3F840
:100530009800E4B280EA042010F4004F02F1FF3288
:100540004FEA400018BF484012F0FF0280B2F3D1DA
:10055000A3F8980010BD01318A4201BF002283F840
:100560000822012283F8962010BD00BF1836002013
:10057000F8B5434C94F81002002859D0002384F8B1
:10058000103294F8113294F8125205EB032502F060
:1005900093FA3C4BADB2B0FBF3F0D4F82432002B0D
:1005A00047D1A4F82852C4F824020322D4F82C32EC
:1005B00094F82B521E7894F82A0294F83072511E47
:1005C000631893F811322B4103F00F03B34212D298
:1005D0000B2B10D808B183420DD0214491F811E2C1
:1005E000A11891F811120EEA070E04EB830301EB38
:1005F0000E21C3F8C0100232112AE0D194F8313232
:10060000ABB194F8323293B194F813321B060ED585
:1006100002F052FAD4F80C321B4964301BB15A680C
:10062000121A002A28DB194AD36004320A6001201A
:10063000F8BD9842B9D0C31A012BB2D194F82A223E
:10064000002AAED0B4F8283294F8BF1092002244A9
:10065000EB1A49B16FF01301DB0293FBF1F303F5E1
:100660000063C2F8C0309CE76FF013019B0293FB5C
:10067000F1F303F58063F4E703F108019B68CDE72C
:100680001836002020A1070024380020E4030020B1
:1006900010B5044602F010FA41F288310E4BD3F83F
:1006A0003422C3F83402821A8A4284BF002283F8BB
:1006B000382293F838220F2A0DD8511CC9B21A4497
:1006C0001029E4B282F8114214BF0022012283F8FB
:1006D000381283F8102210BD1836002010B50446D9
:1006E00002F0EAF940F6AC51104BD3F83C22821AE2
:1006F0008A42C4BF002283F8402293F840228AB97C
:100700000F2C11D1C3F83C02511CC9B21A4419294B
:1007100082F8394114BF0022012283F8401283F885
:10072000382101E0182AEFD910BD00BF183600208B
:1007300010B5044602F0C0F9124BD3F8442202F57A
:100740007A72904284BF002283F8482293F84812BC
:1007500019B9C3F84402052204E00229FBD993F831
:10076000962102328A420CDD481CC0B28242CCBFC4
:1007700000220122194483F8480281F8954183F848
:10078000942110BD1836002010B5074C94F8322281
:1007900042B104F24921D4F8600202F05CFA00236D
:1007A00084F8323210BD00BF183600202DE9F04128
:1007B000884600240C4B93E8E000054406440744B7
:1007C000444501DBBDE8F08137F9142036F91430D7
:1007D00035F914001344022293FBF2F3C01A05F01A
:1007E00041FA0134ECE700BFC8160020064B1A6836
:1007F0004FF47A73B3FBF2F3C3EB431203EB8203C0
:10080000DB000380704700BFFC3F002002392DE968
:10081000F843426804460368806806290DD8DFE87B
:1008200001F0040873767B7E810022605B42636086
:1008300003E05B425242236062603C4B1B7C002B16
:1008400060D1206806F086F98046606806F082F97B
:100850000746A06806F07EF9354D0646D5F86412C5
:10086000404606F0CBF9D5F870128146384606F0BE
:10087000C5F90146484606F0B9F8D5F87C1281461C
:10088000304606F0BBF90146484606F0AFF807F0DF
:1008900071F8D5F868122060404606F0AFF9D5F837
:1008A00074128146384606F0A9F90146484606F01A
:1008B0009DF8D5F880128146304606F09FF9014632
:1008C000484606F093F807F055F8D5F86C126060CA
:1008D000404606F093F9D5F878128046384606F07F
:1008E0008DF90146404606F081F8D5F88412074696
:1008F000304606F083F90146384606F077F807F0EF
:1009000039F8A060BDE8F883524222608FE75B426D
:1009100023604042A06090E722606360F9E75242A2
:100920006260F6E7524222605B42F6E7E403002091
:10093000183600202DE9F04105460F460446094EC1
:1009400006F10808217809B9BDE8F081054809F0E9
:1009500011FB20B140453EBF801B631B3B5401345B
:10096000F0E700BFFABA0108094A92F888325BB989
:10097000084B92F8E41193F822300433DBB28B4237
:1009800028BF0B4682F8883292F88802704700BF71
:100990001836002034190020124B03EB400393F863
:1009A00089222AB1022A12D00F4B33F81000704767
:1009B000022809D90328F7D10C4B1B6813F4805F78
:1009C0000B4B02D1D88C7047094B188B704793F8AA
:1009D0008A0200EB800000EB800000F2EE2080B283
:1009E000704700BF18360020EC1E0020601B00205E
:1009F0003419002008B502F05FF80222064B83F894
:100A0000B422C3F8B002054B1A68054B9A60012264
:100A100083F8212008BD00BF183600204C3A002082
:100A2000641B002008B502F047F80222074B00F5CE
:100A3000B71083F8B422064A00F55870C3F8B00224
:100A4000936803F2DC53936008BD00BF18360020A2
:100A5000641B0020037903F00C03042B05D0082B42
:100A60000FD0BBB9B0F80B0070470B4BB0F80B00C0
:100A70001B7803EBC30203EB820300EB430080B25D
:100A80007047054BB0F80B005B7803EB430300EBBA
:100A90008300F4E7002070475820002010B4447A07
:100AA000631CDBB204444372A172027A9A4202D8F8
:100AB00010BCFEF76BBE10BC704720B10078B0FAD6
:100AC00080F0400970470120704708B5202109F0E7
:100AD00051FA034618461BB102780133202AF9D097
:100AE00008BD2DE9F8430D4616468146002440F620
:100AF00034074FF019084846FFF7E7FF814690B1E9
:100B000006F0AAFDB842A8BF3846B0F5617FB8BF6D
:100B10004FF46170A0F5617090FBF8F04CB928704B
:100B20003378013333700134022CE4D14846BDE8F8
:100B3000F8836870F4E710B50446B0F80900FEF7D2
:100B4000DDFE01462046FFF785FF4B68184410BDC7
:100B500038B505460C46FFF7EEFF2B7903F003038B
:100B6000012B00D001D2047038BD048038BD0FB411
:100B700013B5084C04AB53F8042B074920680193C4
:100B800001F0DFF92068FEF701FE02B0BDE8104079
:100B900004B07047482B00209D0A0108074B1B68D2
:100BA000597A4A1CD2B219445A728872197A9142FF
:100BB00002D81846FEF7EABD704700BF482B002058
:100BC00038B50B4C451E15F8011F206819B9BDE852
:100BD0003840FEF7DBBD427A531CDBB2024443725D
:100BE0009172027A9A42EED8FEF7D0FDEBE700BF91
:100BF000482B00202DE9F8430379044603F0300028
:100C000020280D46164617D10E46DFF87C80DFF807
:100C100084906379771BBB4201DCBDE8F88316F84A
:100C2000011B4046FFF7A3FF6379013BBB42F0DDA8
:100C30004846FFF7C5FFECE703F00303012B06D09E
:100C400008D2097848B1102813D0BDE8F88391F98B
:100C50000010F7E7B1F90010F4E70B48FFF787FF42
:100C600086B1B4F90720B4F905100848BDE8F84387
:100C70007DE76279064B53F8323053F82100BDE826
:100C8000F8439DE7BDE8F8832AD901083FCC010865
:100C90007CB80108C6CB010838B50D460446FFF7FD
:100CA0004AFF2A4601462046BDE83840A2E70148EF
:100CB00086E700BFBECC010810B5064C0B460246C5
:100CC0000549206801F03DF92068FEF75FFDBDE8A9
:100CD0001040ECE7482B00209D0A01080FB407B52F
:100CE00004A951F8040B0191FFF7E6FF03B05DF88A
:100CF00004EB04B0704713460A4601460048EDE78E
:100D0000FDD80108F8B5037903F03003102B0AD0A1
:100D1000202B23D03BBBBDE8F840B0F90720B0F949
:100D200005101148DAE700244579104E1048FFF706
:100D300047FF06EBC5031F79BC4202D3BDE8F8406C
:100D4000B5E714B10B48FFF73BFF56F835300A48BA
:100D500053F82410FFF70BFF0134EDE74179BDE8AC
:100D6000F8400648BAE7F8BD16D901087CB8010872
:100D70002DD90108C6CB010884CB01083DD9010853
:100D80002DE9F74F314C824689460025A04601F0F7
:100D9000100301932E4B1868FEF7F8FC277907F033
:100DA0000C0353450DD10D2303FB058BBBF8090044
:100DB000FEF7A4FD064660B9DBF800102548FFF7F2
:100DC0008DFF0135AA2D04F10D04E3D103B0BDE878
:100DD000F08F2046FFF73EFE07F00307012F834602
:100DE000B26871682CD02ED2175C0A5CBB1A5F42C5
:100DF0005F41019B0BB1002FE3D119F0200F0FD001
:100E000077B90D2202FB058213481168FFF7AFFE88
:100E100071683A4659442046FFF7ECFEFFF747FF5A
:100E20000D2202FB05820D481168FFF7A0FEB16894
:100E3000002259442046FFF7DDFEFFF738FFC0E7E8
:100E400017560A56D2E7175E0A5ECFE7D8AF0108F9
:100E5000482B00204ED901085DD901085ED9010850
:100E60000CB407B510F0200009D069B92320FFF7B2
:100E700095FE05A904980191FFF71EFF012003B01C
:100E80005DF804EB02B070470020F8E70CB4C3062D
:100E900007B500D551B905A904980191FFF70CFFDA
:100EA000012003B05DF804EB02B070470020F8E7C2
:100EB0002DE9F04F814690460C461646334FDFF839
:100EC000D4A087B002F1280B002394F90220304906
:100ED0005956914254D00C333C2BF8D108365E451C
:100EE00004F10804F0D107B0BDE8F08F96F90230A4
:100EF00071799A42328841D1208890423ED1E5787A
:100F0000F07885423AD125793079854236D1A57974
:100F1000B079854232D16579681A4542454157F822
:100F2000211048460491B17957F821100391317985
:100F300057F821100291F178009257F8211052468B
:100F400001912946FFF78CFF627994F9023057F836
:100F5000222029460492A279484657F8222003927B
:100F6000227957F822200292E27857F82220019243
:100F7000228800925246FFF789FFAFE70025CEE7AF
:100F8000B8F1000FB2D14546DEE700BF90A40108DA
:100F90003C40002068D901082DE9F04F8146904679
:100FA0000C46154600261927DFF8A8A085B0B8F131
:100FB000000F4CD028782378834246D162786B7832
:100FC0009A4242D1A278AB789A423ED1E178EB784E
:100FD000CB1A594259418B46FBF786F998B1EB7809
:100FE00052467B4303F561730393AB7859467B43C9
:100FF00003F5617302936B780193037A484600937B
:101000003346FFF72DFF2078FBF76EF998B1E378B0
:1010100052467B4303F561730393A37859467B43A0
:1010200003F56173029363780193037A4846009352
:101030003346FFF72BFF0136142E04F1040405F1AB
:101040000405B4D105B0BDE8F08F0021C3E7C34665
:10105000D9E700BF85D90108F7B50746FFF72DFD91
:10106000044630B1002229490120FFF795FF03B063
:10107000F0BD384606F0F0FA1328054635DC860048
:10108000781C8DF80740FFF720FD074668B106F091
:10109000E3FA0C211E4AC0B201FB042393F808E0D6
:1010A000864528D00134242CF6D13846FFF70DFDB3
:1010B000164C074650B106F0CFFA0D2806D8A319F2
:1010C00058709DF8073001338DF80730B11C0DF1D1
:1010D000070221443846FFF704FD9DF80730042B32
:1010E000C5D0002344F82530C1E713222146094822
:1010F000FFF701FEBBE71A78044B03F825209DF8A3
:10110000073001338DF80730CFE700BFBC22002045
:1011100010BB010881C5010808B5FFF751FDBDE806
:101120000840C4E50048F7E798D901082DE9F341E4
:101130000346FFF7C2FC044630B1002201203649C5
:1011400002B0BDE8F041B3E60090019018465E1C85
:1011500006F082FA304B40B203EBC40595F9022049
:10116000824255D00134052CF6D100252C4630465C
:10117000FFF7ABFC074628B106F06EFA0134ADF874
:101180000000E4B20026DFF894803846FFF79DFCAB
:10119000074600B306F060FA002258F82210D3B2D6
:1011A000884203D00132102AF7D1002358F82320B7
:1011B000904210D1022E19D0032E1CD05A1E012E9F
:1011C000D2B20ED00B2A03D88DF803300134E4B22A
:1011D0000136042ED9D1052C13D802B0BDE8F04158
:1011E000A0E7042AF4D88DF80430EFE7052BEFD8F8
:1011F0008DF80630EAE79A1E0D2AE9D88DF80530F9
:10120000E4E76B4603CB2860696002B0BDE8F0817B
:101210008DF802000124AAE70E40002090A40108E6
:10122000F7B50646FFF749FC054658B1002401A969
:10123000204603F08BFC0134FFF7F2FF122CF6D1AD
:1012400003B0F0BD304606F007FAC4B2112C5DD8E9
:10125000701CFFF73AFC304D0746B8B92F4B13F816
:1012600014108A1E514251412C4B13F81420AA5CD1
:10127000002946D003EB4403597819234B432848EF
:1012800003F2EE232146FFF729FDD9E7017828462E
:1012900008F070FE60B1032C8CBF03220022214BAA
:1012A000401BC0B21344184490F8B061032E02D121
:1012B000FFF738FFC4E73846FFF707FCF0B1022E0E
:1012C000F6D106F0C9F940F6CA0280B29042A8BF32
:1012D000104640F2EE229042B8BF10461922A0F20A
:1012E000EE2090FBF2F00D4B03EB44035870B31E5D
:1012F00059425941094B03F81460B5E7022EF6D163
:10130000D6E721460848FFF7E9FC99E7112229466C
:101310000648FFF7F0FC93E738A90108A138002040
:1013200060C6010810BB010870C60108CBD10108D6
:10133000002310B5074A9C5C9918844203D18C782D
:10134000C9788C4204D30433502BF4D1002010BD53
:10135000012010BDBC22002010B50C7849788C42C9
:101360001CD20F4B043033F9102040F633039A425D
:10137000A8BF1A461923B2F5617FB8BF4FF4617256
:101380005C4304F28334944208DA03FB01F000F278
:1013900083309042B4BF0020012010BD002010BD5A
:1013A000EC1E00200146014801F03DB8B4160020B3
:1013B00008B51C20FFF7F6FF20B9034B1868C0F3EF
:1013C000805008BD012008BD601B002038B50F4BC0
:1013D0000F4D1B680F4C13F4805F11D01D20FFF7D9
:1013E000E1FF68B90C4A238BD288B5F90600991A37
:1013F000884209DD13449842B4BF0020012038BD63
:10140000B5F90600638BF6E7012038BD601B0020AC
:10141000EC1E002034190020303900201FB5084B85
:101420009B784BB100238DF8040002910D2001A997
:101430008DF80530F7F7B0FB05B05DF804FB00BF91
:101440008C410020F0B500210A25154884680A3037
:10145000E27897B2CB1B1BB2002B1EDDC2F16402F7
:10146000D2B203FB03F694F804E052430EFB06F6F7
:1014700096FBF2F2CEF1640E7244534393FBF5F304
:1014800007EB87070A3103EB470389B203F57A7349
:10149000782920F8023FDBD1F0BD08BF0122E0E748
:1014A0003039002070472DE9F0412D4D2C68228AFB
:1014B000D2B9267A042E17D12A480378012B0FD1EE
:1014C000294B1968294B89B221F007010B445B00B5
:1014D0001A603023027043802B681E72BDE8F081D1
:1014E000102307264380F7E7B4F81480A369424528
:1014F0008CBF02260426904528BF90461FFA88F725
:10150000384698470021184B08F101021B68521019
:101510009BB223F0070303F1005303F540535B0034
:101520001B689BB203F1005303F540535B008A42F2
:1015300010D139460020FBF787FC3022238ADB1BC1
:101540002382638A1F44074B67825A804FF44052BC
:101550009A80C1E730F802EB23F821E00131E6E799
:10156000443A00205C390020505C004002300020EA
:1015700008B50B4B002093F82C10FBF743FC094BEC
:101580001B68187A082805D14FF48052064B9A80C0
:1015900010225A80A0F109035842584108BD00BFEB
:1015A00030040020443A00205C3900207047704726
:1015B0007047FEE7FEE7FEE77047202938B50C4686
:1015C0001DD8D1B1631C124AA1B25B100432C3B959
:1015D0000120FBF739FC0F4A1368234413600E4ABD
:1015E000136823F4E04323F040039BB283F03003FD
:1015F00043F4004343F080031360204638BD2024A9
:10160000E0E730F8025B013B22F8045CDEE700BF54
:1016100080610040503A0020045C0040002330B557
:101620001D46DCB2A24200D830BD040F092C94BF85
:101630003034373401F8134001EB43040001657086
:101640000133EEE770B5002240F60F7648F28005D0
:1016500002F1805303F5B8539B00196842EA050470
:10166000314001322143042A1960F1D1024B40F08C
:101670008000186070BD00BF4C5C00402DE9F3474E
:10168000994D9A4C2B689A4E9BB2E380E38832883E
:101690001340980506D54FF6FF532B60237A01338C
:1016A000DBB22372E3881A40110440F11382002355
:1016B00048F60F788F4FDFF85092ADF802302B6864
:1016C0009AB21904E28040F10582E38803F00F0327
:1016D0006372002B40F0FD82D9F800309BB2A380EA
:1016E000A38803F030036380A38803F44053A380EE
:1016F000D9F8003023F4804323F040031B041B0C73
:1017000083F4005383F0200343F4004343F0800349
:10171000C9F80030E38813F0100FD9F8003028D151
:1017200023F4E14323F070031B04734F1B0CC9F82F
:1017300000303B681A7A022A01D0042A06D1FFF74A
:10174000B2FE3B681B7A3A6813729CE1062A0ED1FE
:101750005A78052A08D11A78520605D1D878FFF7A9
:1017600071FFE3681B6A984723699B6898470823C1
:10177000E9E79BB2ADF80230BDF80230180540F140
:101780001982D9F800305D4923F070031B051B0D49
:10179000C9F800300A685A4B92B222F0070213448B
:1017A000554F5B001A683B688846187A092817D09D
:1017B00092B2520002F1804202F5C04211781970D3
:1017C000517859709088C1B2090241EA10215980BC
:1017D0001089C1B2090241EA102199809289DA8008
:1017E00001221A72DA8893F80190002A40F0DC8016
:1017F0001A7812F07F0258D1B9F1090F16D1DA78B0
:10180000012A08D9236948465B699847032840F0B4
:10181000C780092397E799780029F3D1998800298F
:10182000F0D19A72E3685B6898470FE0B9F1050F51
:101830001AD193F90320002A99DB9A78002A96D1CD
:101840009A88002A93D19B7A002B90D1D8F8002057
:101850002C4B92B222F00702134400225B001A6064
:101860003023638006236EE7B9F1030F0CD1DA78D9
:10187000012AC7D19A88002AC4D15A7A42F020029C
:101880005A72E368DB69CFE7B9F1010FBAD1DA78B0
:10189000012AB7D19A88002AB4D15B7A9906B1D5CA
:1018A00005F06AFD0028D1D0ACE7012A2ED1B9F1AC
:1018B0000B0FA7D12269D9789269587990473B6874
:1018C0009A7A002A9ED000289CD11A79002A99D1B0
:1018D0009B78002B96D1E368DB6898473B685A7980
:1018E000DA72DA781A73B1E7445C00405C390020A0
:1018F00084410020C8BC0108443A0020505C0040EC
:101900000430002002300020005C0040022A7FF4F6
:1019100079AFB9F1010FC3D0B9F1030F7FF472AF02
:10192000587920F0800E4FEA8E0202F1804101F5D5
:10193000B841096840B20028B4BF01F0300101F499
:101940004051BEF1030F3FF65DAFB3F802E0BEF1C8
:10195000000F7FF457AF00293FF454AF9B7A002B60
:101960003FF450AF02F1804202F5B84213680028FC
:10197000B5BF23F4E04323F4804323F0400323F076
:101980007003B5BF9BB29BB283F0100383F4805306
:1019900043F4004343F080031360E3689B6943E72B
:1019A00000287FF4E4AE51E7B9F1060F13D11A789D
:1019B00052065ED19B78012B03D12369DB69FBB909
:1019C00057E0022B02D123691B6AF8E7032B50D1A1
:1019D00023695B6AF3E7B9F1000F40F09D805988F5
:1019E000002946D15A6822F47F42B2F5003F40D127
:1019F0001A7812F07F0219D19B88002B39D1A84B9D
:101A00004FF000083A684046A2F812809361984768
:101A100040464FF6FF713B681A8A8A4231D002284D
:101A200002D0002A40F09C8008222BE0012A09D134
:101A30002269587992699047D8B93B689B7A002B04
:101A4000DDD116E0022A14D15A7902F00F018B0081
:101A500003F1804303F5B8431B6812F0800F14BFF5
:101A600003F0300303F44053032902D812F0700F3F
:101A7000E5D03A68236950781B6998470328C8D194
:101A80003B6809221A72FFF773FD864B1B68A28818
:101A900023F4804323F04003D1044FEA0343A28898
:101AA0004FEA134348BF83F480539204628848BFCF
:101AB00083F40053D706628848BF83F01003900672
:101AC00048BF83F0200343F4004343F08003754A8A
:101AD0009BB213603288E38813405A0505D54FF650
:101AE000FF332B60704B5B689847E3883288134064
:101AF000DB0440F128814EF6FF732B600023237531
:101B0000237D052B00F21481DFE813F00E0117018D
:101B1000200124012D013801B9F1080F04D11B78EF
:101B20005B06A6D1614B6BE7B9F10A0FA1D11A7818
:101B300002F07F02012A9CD19A7A002A99D0598812
:101B4000002996D15A6822F47F42B2F5803F90D1A5
:101B5000226958799269904700288AD1544B4FE7FF
:101B600093F9001000291FDAD98801910198824267
:101B700008D9019A1A82226992F82C209A82FFF7DA
:101B800092FC80E78A42F6D2216991F82C008242C9
:101B900002D200222270EEE792FBF0F100FB11224C
:101BA000002AE8D10122F5E703221A724FF44053CC
:101BB000A38068E7BDF8023018047FF580ADD9F83E
:101BC00000303C4A23F070031B051B0D1768C9F851
:101BD00000303B7A9146022B79D0042B77D0032B2F
:101BE00001D0052B6ED1BB693A8AC3B93B8A43B198
:101BF00000214FF440530846A380FBF725F930231A
